:100000000C9410210C9441210C9441210C94412119
:100010000C9441210C9441210C9441210C944121D8
:100020000C9441210C9441210C9441210C944121C8
:100030000C9441210D940E380C9441210C944121D3
:100040000C9441210C944CD80C9441210C944121E6
:100050000C9441210C9441210C9413D50D94C43778
:100060000C9441210C94404C0C94364C0C9441213E
:100070000C9441210C9441210C9441210C94412178
:100080000C9441210C9441210C9441210C94412168
:100090000C9441210C9441210C9441210C94412158
:1000A0000C9441210C9441210C9441210C94412148
:1000B0000C9441210C9441210C9441210C94412138
:1000C0000C9441210C9441210C9441210C94412128
:1000D0000C9441210C9441210C9441210C94412118
:1000E0000C944121084AD73B3BCE016E84BCBFFD36
:1000F000C12F3D6C74319ABD56833DDA3D00C77FF8
:1001000011BED9E4BB4C3E916BAAAABE0000008090
:100110003F05A84CCDB2D44EB93836A9020C50B91F
:10012000918688083CA6AAAA2ABE000000803F004B
:100130000C943E7F0C9406850C94B27A0C94AD4CD2
:100140000C94E3AF0C94044D0C9490C80C9413865B
:100150000C9436C30C9416860C9409A70D940532A2
:100160000C949B830C940F850C9441780C943079FB
:100170000C94D1AF0C9419820C94ACC90D9430310D
:100180000C94C37C0C94FBAF0D94B4310C94CE7ED4
:100190000C942BBD0D9449310C94BF7C0C949D782C
:1001A0000C94337D0D943C310C94A97A0C94B3AF2C
:1001B0000C948A7A0C94EFC80C9476810C94EA4CD7
:1001C0000C94B99E0C94D64C0C94CB4C0C944C22B1
:1001D0000D94E7310D943C320D9434310C946FC87A
:1001E0000C94C17C0C9410BC0C9443210C94469646
:1001F0000C94D4C80C94C5AF0D94E3120C944BB37B
:100200000D944F310C94E7330C94BC4C0C94189D16
:100210000C9482810C94DDAF0C9401BD0D94F131EE
:100220000D9442130C9465820C9473790C941D8682
:100230000C9407860C944B760C9462810C9405B058
:100240000C94FCB00C94787E0C946E810C946DC967
:100250000D9446320C9423860C94B0820C949782B1
:100260000C9450A00D9444440C9441B30C9476CA61
:100270000C94B6780C945C790C940CC50C940D8697
:100280000C94F5AF0C9429820D941E310C943A7A9B
:100290000C9451250D9465310C94558E0C94D7AF68
:1002A0000C94E24C0D9428320C94A1BC0C94B9C36C
:1002B0000C9446B30C9455380C94F4980D94143265
:1002C0000C943E830C94287B0C942FBC0C94DC780B
:1002D0000D941E320C94BFAF0C94AD7A0C94462151
:1002E0000C94BC970C94C0210C9431820C94137B19
:1002F0000C94BB7C0D9445310C94CA7E0C941D76F5
:100300000C9426970D94DF310C9486810C94EA822C
:100310000D94F1430C9404860C945A780C947C86CA
:100320000C943AA80C94EFAF0C94398D0C94FC4CBF
:100330000C94CBAF0D9462440C9428250C940E7948
:100340000C94C17A0C943D7B0C941B860C94C9824E
:100350000C94D68B0D9419310C94E64C0C94767C4D
:100360000C94967A0C942C7C0C9434220C94A179E5
:100370000C940B830C94D1990C94AB7A0C94DAC73F
:100380000C94B9AF0C94BD7C0C94D24C0C9482BCF0
:100390000C9440760C94F8880C9420860D946F3160
:1003A0000C94F7900C94B77C0C94257B0C94DB7B1D
:1003B0000D94CD310C94FE840C9473780C9422A28D
:1003C0000D94C3310D946B310C948A790C946D7C2F
:1003D0000C94227B0D94D7310C94DDB30C94E2BCC9
:1003E0000C94BC940C94C67E0C94C9780C947281C5
:1003F0000D9439140D943F310C9450B30C94F7C7FD
:100400000D9432320C940A860C9436B70D946131F7
:100410000C9468B30C941D790C945B980C94B325E0
:100420000C94DE4C0C9466810C94467B0C945C849A
:100430000C94F14C0C94427B0C94C39E0C947FC999
:100440000D9453310C94BC7A0C946A810C94978669
:100450000C94B8C30D9410130C94D4820C9482782D
:100460000C947E810C942B7B0C9410860C94F97A5E
:100470000C94B97C0D945D310C945BC70C94E9AF7E
:100480000C94B77A0C94BA920C94429B0C94B87961
:100490000C94B57C0C94817A0C941A850C9421A54B
:1004A0000D9438310D94B9310C948A760C94CB8A22
:1004B0000C947E820C94BEAC0C94F5780D94FB31B8
:1004C0000C947E4C0C94F6850C9443790D94573122
:1004D0000C9455830C94F8840C947A810C9417B482
:1004E0000C94DA4C0C94A3760C94B1760C946C7E3C
:1004F0000D94AC310C9479860C941D7C0C9401867F
:100500004E414E494E495459494E46CDCCCC3D0AF8
:10051000D7233C17B7D13877CC2B329595E6241FDB
:10052000B14F0A000020410000C84200401C462094
:10053000BCBE4CCA1B0E5AAEC59D7400407A10F367
:100540005A00A0724E18090010A5D4E80000E87601
:1005500048170000E40B54020000CA9A3B00000058
:10056000E1F505000080969800000040420F000071
:1005700000A08601000000102700000000E8030032
:100580000000006400000000000A000000000001FC
:1005900000000000002C76D888DC674F0823DFC1FC
:1005A000DFAE59E1B1B796E5E3E453C63AE65199B7
:1005B0007696E8E6C28426EB898C9B62ED407C6FE0
:1005C000FCEFBC9C9F40F2BAA56FA5F490055A2A97
:1005D000F75C936B6CF9676DC11BFCE0E40D47FEA3
:1005E000F520E6B500D0ED902E0300943577050098
:1005F00080841E080000204E0A000000C80C33331F
:1006000033330F986E12831141EF8D2114893BE62D
:100610005516CFFEE6DB18D1844B381BF77C1D90B6
:100620001DA4BBE424203284725E228100C9F1241F
:10063000ECA1E53D27434F4D4D554E4943415449AB
:100640004F4E0044525952554E004552524F52534C
:1006500000494E464F004543484F004572726F7245
:100660002077726974696E6720746F204545505217
:100670004F4D210A0053544F505045442E200050F6
:1006800072696E7465722073746F70706564206433
:10069000756520746F206572726F72732E204669C3
:1006A0007820746865206572726F7220616E6420B4
:1006B000757365204D39393920746F2072657374F4
:1006C0006172742E202854656D7065726174757244
:1006D000652069732072657365742E2053657420DC
:1006E00069742061667465722072657374617274D6
:1006F000696E67290A004E6F20436865636B7375E6
:100700006D2077697468206C696E65206E756D6206
:1007100065722C204C617374204C696E653A200020
:100720004E6F20436865636B73756D2077697468DD
:10073000206C696E65206E756D6265722C204C614F
:100740007374204C696E653A2000636865636B734F
:10075000756D206D69736D617463682C204C6173D5
:1007600074204C696E653A20004C696E65204E75A8
:100770006D626572206973206E6F74204C617374B2
:10078000204C696E65204E756D6265722B312C2090
:100790004C617374204C696E653A20004D313130E4
:1007A0000053657269616C20737461747573206D98
:1007B00069736D617463680A00776169740A005334
:1007C000442072656164206572726F720A00486F1E
:1007D00074656E642049646C652054696D656F753D
:1007E0007400486F74656E642049646C65205469B8
:1007F0006D656F75740A002121204B494C4C2063B4
:100800006175736564206279204B494C4C20627598
:1008100074746F6E2F70696E0A002121204B494C51
:100820004C2063617573656420627920746F6F205A
:100830006D75636820696E6163746976652074699B
:100840006D65202D2063757272656E7420636F6D07
:100850006D616E643A20007061757365004D3630CD
:1008600030002066696C616D656E745F72756E6FC5
:100870007574200066696C616D656E745F72756E6B
:100880006F757420540046696C616D656E745275A5
:100890006E6F75742054004D656469612052656DFA
:1008A0006F766564004D6564696120496E73657299
:1008B000746564004D313030305300627573793A9D
:1008C0002070617573656420666F7220696E707543
:1008D000740A00627573793A2070617573656420DB
:1008E000666F7220757365720A00627573793A20BB
:1008F00070726F63657373696E670A00506C65612F
:100900007365205265736574005052494E544552C8
:100910002048414C5445440025533A20255300704B
:100920006F7765726F6666004B494C4C45442E20CC
:10093000005072696E7465722068616C7465642E13
:10094000206B696C6C28292063616C6C6564210ADA
:10095000006563686F3A004572726F723A000A4D23
:100960006561737572656420706F696E74733A0A9D
:1009700000357835206D6573682E205A206F6666C5
:100980007365743A20005072696E74696E67204F07
:10099000626A656374002553202569002F2F616307
:1009A00074696F6E3A0073746172740070726F6D67
:1009B00070745F00656E6400486F74656E642074C7
:1009C0006F6F20636F6C640A0053656E64204D3155
:1009D000303820746F20726573756D650A00496E3A
:1009E000736572742066696C616D656E7420616EEA
:1009F000642073656E64204D3130380A005265689A
:100A000065617420446F6E65005265686561746944
:100A10006E672E2E2E005265686561740048656110
:100A20007465722054696D656F75740053656E64EA
:100A3000204D31303820746F2068656174206E6FEE
:100A40007A7A6C650A004E6F7A7A6C652050617212
:100A50006B656400706175736564005061757365E2
:100A600000726573756D656400526573756D696EAE
:100A700067004732362043616E63656C65640047EA
:100A800032362048656174696E67204E6F7A7A6CE1
:100A900065004732362048656174696E672042659B
:100AA000640057616974696E6720666F72206865BB
:100AB000617475702E0A004669786564204C656E15
:100AC000677468205072696D6500446F6E652050D0
:100AD00072696D696E67004D616E75616C20707230
:100AE000696D696E672E2E2E004C656176696E67A2
:100AF00020473236003F537065636966696564203C
:100B0000582C5920636F6F7264696E617465206F31
:100B10007574206F6620626F756E64732E0A003FD5
:100B200028522965706561742076616C7565206E48
:100B30006F7420706C61757369626C653B206D75B4
:100B40007374206265206174206C65617374203158
:100B50002E0A003F537065636966696564206E6F95
:100B60007A7A6C652074656D7065726174757265F2
:100B7000206E6F7420706C61757369626C652E0AEB
:100B8000003F5370656369666965642066696C61DE
:100B90006D656E742073697A65206E6F7420706C59
:100BA00061757369626C652E0A003F5370656369F5
:100BB00066696564207072696D65206C656E677426
:100BC00068206E6F7420706C61757369626C652E3D
:100BD0000A003F537065636966696564206E6F7AC9
:100BE0007A6C652073697A65206E6F7420706C6111
:100BF000757369626C652E0A003F52657472616399
:100C000074696F6E204D756C7469706C69657220C3
:100C10006D757374206265207370656369666965BC
:100C2000642E0A003F5370656369666965642052EB
:100C3000657472616374696F6E204D756C74697050
:100C40006C696572206E6F7420706C617573696277
:100C50006C652E0A003F53706563696669656420A0
:100C60006C6179657220686569676874206E6F745D
:100C700020706C61757369626C652E0A0043292EC1
:100C80000A003F5370656369666965642062656444
:100C90002074656D7065726174757265206E6F7415
:100CA00020706C61757369626C65202834302D008A
:100CB000473236207374617274696E672E2E2E0A65
:100CC000004F46460A0046616465204865696768CA
:100CD000742000426564204C6576656C696E6720FF
:100CE000004661696C656420746F20656E61626C9A
:100CF0006520426564204C6576656C696E670A0004
:100D00004D65736820426564204C6576656C20648F
:100D10006174613A0A00496E76616C6964206D65A0
:100D200073682E0A00206E6F7420656E746572659C
:100D3000642E0A0050726F62696E6720506F696E90
:100D4000740025532025692F256900206F66200037
:100D50004D424C2047323920706F696E7420002953
:100D60000A004A206F7574206F662072616E676595
:100D70002028302D00290A0049206F7574206F66E5
:100D80002072616E67652028302D004732384C3064
:100D9000004D6573682070726F62696E6720646FC2
:100DA0006E65004D6573682070726F62696E6720B2
:100DB000646F6E652E0A005374617274206D6573E2
:100DC000682070726F62696E67207769746820228C
:100DD000473239205331222066697273742E0A001B
:100DE0004732395332004732384C300A4732395390
:100DF0003200686173206E6F20646174612E0A0096
:100E00004D65736820426564204C6576656C696E3B
:100E100067200053206F7574206F662072616E67C3
:100E2000652028302D35292E0A004D657368207005
:100E30006F696E74206F7574206F662072616E67C3
:100E4000650A004D34323120696E636F72726563DA
:100E50007420706172616D6574657220757361676D
:100E6000650A004F4646004F4E0020204D61783AFB
:100E70002000200020204D696E3A2000536F6674D8
:100E800020656E6473746F70733A20004D323420A5
:100E900053256C642054256C64004739322E392068
:100EA00045257300473120462564004739322E39E5
:100EB000205A2573004731205A3020463230300006
:100EC0004731205825732059257320463330303060
:100ED000004D34323020532569205A2573004D319E
:100EE00030362050256920532569004D323030209E
:100EF0004425730047323852305859004739322E52
:100F000039204530205A300A47315A2573004D3177
:100F1000303920532569004D31393020532569007F
:100F20004D343230205330205A300020496E7661E3
:100F30006C6964206578747275646572200047324C
:100F40002F47332062616420706172616D65746542
:100F500072730A00536C6565702E2E2E004D6573FA
:100F60006820706F696E74206F7574206F662072D0
:100F7000616E67650A004D302053746F70004D310B
:100F80002053746F7000436C69636B20746F205240
:100F90006573756D652E2E2E004E6F204D6F766534
:100FA0002E00456E642066696C65206C6973740A56
:100FB00000426567696E2066696C65206C697374B0
:100FC0000A004E6F206D656469610A005265737591
:100FD0006D696E6720534400286E6F2066696C65EA
:100FE000290043757272656E742066696C653A20DB
:100FF000005072696E742074696D653A20000A535E
:10100000746174733A2046696C616D656E74207505
:101010007365643A20002C204C6F6E6765737420F2
:101020006A6F623A2000546F74616C2074696D6558
:101030003A200053746174733A20002C2046616991
:101040006C65643A20002C2046696E69736865649B
:101050003A20005072696E74733A200053746174C0
:10106000733A2000436F6F6C696E672E2E2E004816
:10107000656174696E672E2E2E0045202553006F22
:101080006B006F666600560651064A064306350633
:1010900044454255473A004D3131332053004265B3
:1010A0006420436F6F6C696E672E2E2E004265645C
:1010B0002048656174696E672E2E2E00544D3344AE
:1010C00020435231305632204F46462E002F2F00FB
:1010D0004D31343520533C696E6465783E206F7520
:1010E00074206F662072616E67652028302D31296B
:1010F0000A00205200416363656C65726174696F18
:101100006E3A2050005741524E494E4721204C6FB5
:1011100077205A204A65726B206D6179206C656179
:101120006420746F20756E77616E746564207061E1
:10113000757365732E0A004D3230362058004652C2
:101140003A0020466C6F773A20004D424C204164B3
:101150006A757374205A0020643A0020693A0020AE
:10116000703A00496E76616C6964206578747275B6
:101170006465720A0020643A0020693A0020703ADF
:101180000064697300656E0043290A0061626C6542
:101190006420286D696E2074656D702000436F6C4B
:1011A00064206578747275646573206172652000CF
:1011B00046696C616D656E742072756E6F75742012
:1011C00064697374616E636520286D6D293A20002F
:1011D00046696C616D656E742072756E6F757420F2
:1011E000004F666673657473204170706C69656446
:1011F000004572723A20546F6F206661722100546C
:101200006F6F206661722066726F6D207265666511
:1012100072656E636520706F696E740A0045455093
:10122000524F4D204F4B0A00506F7765722D6C6FF7
:101230007373207265636F7665727920004D383460
:1012400000446F6E65207072696E74696E67206607
:10125000696C650A004D3737004D333100436170CA
:101260003A004D4541545041434B00434F4F4C458C
:10127000525F54454D5045524154555245004348E4
:10128000414D4245525F54454D504552415455528F
:101290004500424142595354455050494E47004140
:1012A000524353004D4F54494F4E5F4D4F444553A9
:1012B00000544845524D414C5F50524F54454354A1
:1012C000494F4E004C4F4E475F46494C454E414DAD
:1012D00045004155544F5245504F52545F53445F5F
:1012E0005354415455530053445F57524954450099
:1012F00052455045415400534443415244005052DA
:101300004F4D50545F535550504F525400454D452A
:101310005247454E43595F50415253455200434155
:1013200053455F4C494748545F4252494748544EE1
:1013300045535300544F47474C455F4C4947485429
:101340005300534F4654574152455F504F574552F3
:10135000004255494C445F50455243454E54004C61
:101360004556454C494E475F44415441005A5F50F1
:10137000524F42450052554E4F5554004155544F1F
:101380004C4556454C005052494E545F4A4F42001E
:1013900050524F4752455353004155544F524550B8
:1013A0004F52545F54454D5000564F4C554D455487
:1013B00052494300454550524F4D0042494E41521B
:1013C000595F46494C455F5452414E534645520081
:1013D00053455249414C5F584F4E5F584F46460067
:1013E0004649524D574152455F4E414D453A4D6138
:1013F000726C696E20322E302E375F4457372E3391
:1014000020544D33442053534D444E4E20284170B8
:101410007220323420323032312032323A32303A95
:1014200032302920534F555243455F434F44455F67
:1014300055524C3A68747470733A2F2F6769746808
:1014400075622E636F6D2F496E73616E6974794199
:1014500075746F6D6174696F6E2F4D61726C696E1A
:101460002F747265652F437265616C697479447776
:10147000696E5F322E302050524F544F434F4C5FB5
:1014800056455253494F4E3A312E30204D41434834
:10149000494E455F545950453A544D3344204352C8
:1014A000313056322045585452554445525F434FCF
:1014B000554E543A3120555549443A636564653276
:1014C0006132662D343161322D343734382D396232
:1014D00031322D6335356336326633363766660A08
:1014E0000043616E6E6F74206F70656E207375625D
:1014F00064697220002569730025696D2025697370
:10150000002569682025696D2025697300256964B7
:10151000202569682025696D202569730025697972
:1015200020256964202569682025696D2025697357
:101530000023646566696E652044454641554C54F8
:101540005F00626564004B6420004B6920004B70B3
:101550002000504944204175746F74756E65206693
:10156000696E6973686564212050757420746865BC
:10157000206C617374204B702C204B6920616E6469
:10158000204B6420636F6E7374616E747320667297
:101590006F6D2062656C6F7720696E746F20436F8A
:1015A0006E66696775726174696F6E2E680A0050A5
:1015B0004944204175746F74756E65206661696C6D
:1015C0006564212074696D656F75740A0050494423
:1015D000204175746F74756E65206661696C656411
:1015E000212054656D706572617475726520746F29
:1015F0006F20686967680A00204B643A2000204B1E
:10160000693A2000204B703A200020436C617373CC
:10161000696320504944200A00204E6F206F766590
:101620007273686F6F740A002054753A2000204B63
:10163000753A2000206D61783A2000206D696E3A7D
:10164000200020643A200020626961733A20005033
:101650004944204175746F74756E652073746172AE
:10166000740A00504944204175746F74756E65208A
:101670006661696C6564212054656D706572617482
:1016800075726520746F6F20686967680A00504939
:1016900044204175746F74756E6500504944204153
:1016A00075746F74756E65206661696C6564212060
:1016B000426164206865617465722069640A00454E
:1016C00072723A207574663820666F6E74206E6F81
:1016D0007420696E697469616C697A65642E00456D
:1016E00072723A207574663820666F6E74206E6F61
:1016F0007420696E697469616C697A65642E00454D
:1017000072723A207574663820666F6E74206E6F40
:101710007420696E697469616C697A65642E000071
:101720000C0F00FE07022503BB017FFE08FE08FE2A
:1017300005080806000040F0C88888987810050859
:1017400008060000C0F88888888888F8050505061E
:1017500000012030F830200508080600002070F84D
:1017600020202020E00509090600FF2070A8A8B865
:1017700088887020070505070001D86C366CD805ED
:1017800009090600FFF8A88888888888A8F8050A4B
:101790000A0600FE205050505088A8A88870030305
:1017A0000306000340A040FFFFFFFFFFFFFFFFFF16
:1017B000FFFFFFFFFFFFFFFFFFFFFFFFFF00000036
:1017C0000605FF01070706020080808080800080F8
:1017D000030303060105A0A0A005060606000050AD
:1017E000F85050F8500509090600FF2070A8A070B5
:1017F00028A87020050707060000C8C810204098D8
:101800009805070706000040A0A040A890680103C3
:10181000030602058080800309090601FF2040407D
:101820008080804040200309090601FF804040205D
:10183000202040408005070706000020A870207087
:10184000A8200505050600012020F820200203033A
:101850000601FFC04080050101060003F8020202F4
:10186000060100C0C0050707060000081010204050
:101870004080050707060000708898A8C888700394
:10188000070706010040C040404040E0050707064A
:101890000000708808102040F8050707060000F8CF
:1018A00008103008887005070706000010305090B7
:1018B000F81010050707060000F880F00808887087
:1018C000050707060000304080F08888700507078C
:1018D000060000F808101020202005070706000069
:1018E00070888870888870050707060000708888EF
:1018F00078081060020505060100C0C000C0C002E3
:1019000006060601FFC0C000C040800305050601B1
:10191000012040804020050303060002F800F80380
:1019200005050601018040204080050707060000EC
:10193000708810202000200507070600007088B876
:10194000A8B88070050707060000708888F88888A6
:1019500088050707060000F04848704848F005076A
:1019600007060000708880808088700507070600E1
:1019700000F04848484848F0050707060000F8808E
:1019800080F08080F8050707060000F88080F0806E
:1019900080800507070600007088808098887005A1
:1019A0000707060000888888F888888803070706E4
:1019B0000100E04040404040E005070706000038D5
:1019C0001010101090600507070600008890A0C056
:1019D000A09088050707060000808080808080F83E
:1019E00005070706000088D8A888888888050707A3
:1019F0000600008888C8A8988888050707060000A0
:101A000070888888888870050707060000F0888835
:101A1000F080808005070706000070888888A890FD
:101A200068050707060000F08888F0A09088050781
:101A30000706000070888070088870050707060098
:101A400000F82020202020200507070600008888B5
:101A5000888888887005070706000088888888506D
:101A6000502005070706000088888888A8A8500528
:101A70000707060000888850205088880507070659
:101A8000000088885020202020050707060000F865
:101A90000810204080F80309090601FFE0808080DB
:101AA00080808080E005070706000080404020100D
:101AB00010080309090601FFE02020202020202033
:101AC000E00503030600052050880501010600FE1D
:101AD000F803030306010580402005050506000004
:101AE00070087888780507070600008080F08888ED
:101AF00088F00505050600007080808870050707DE
:101B00000600000808788888887805050506000022
:101B10007088F08070050707060000304840E040FC
:101B200040400507070600FE708888887808700521
:101B300007070600008080F088888888030707066A
:101B400001004000C0404040E00409090601FE10C9
:101B5000003010101010906005070706000080800C
:101B60008890E09088030707060100C0404040408D
:101B700040E0050505060000D0A8A8A8A8050505B1
:101B8000060000B0C8888888050505060000708832
:101B90008888700507070600FEF0888888F0808036
:101BA0000507070600FE7888888878080805050577
:101BB000060000B0C880808005050506000078801A
:101BC0007008F00507070600002020F820202018E4
:101BD0000505050600008888889868050505060043
:101BE0000088888850200505050600008888A8A878
:101BF0005005050506000088502050880507070697
:101C000000FE88888850204080050505060000F801
:101C1000102040F80309090601FF204040408040A1
:101C20004040200109090602FF808080808080807A
:101C300080800309090601FF804040402040404069
:101C40008005030306000248A890FF554E4C4F4103
:101C5000442046494C414D454E54004C4F41442090
:101C600046494C414D454E540046494C414D454E28
:101C700054204348414E47450042656400456E6329
:101C80006C6F73757265002568753A25303268751A
:101C90000025303268753A253032687500202020E2
:101CA000202020200020202020001FE020102010D5
:101CB0002010102010202010201030300840048008
:101CC00003001FE03FF03FF03FF01FE01FE03FF058
:101CD0003FF03FF00FC0078003003FFFF038007077
:101CE00030FC3020FC102078102030102C00D02E3A
:101CF00031D02F7BD02F7BD02E31D02C00D0203074
:101D00001020781020FC1030FC303800703FFFF0BD
:101D10003FFFF03800703186302387102787902FDF
:101D200087D02F03D020301020781020781020305A
:101D3000102F03D02F87D02787902387103186302C
:101D40003800703FFFF01FFFF81FFFF8041040023B
:101D50000820020820041040082080104100104193
:101D6000000820800410400000001FFFF81FFFF84B
:101D7000FFFFFF8000018E00E19F01F19381399FF9
:101D800081F99F81F99FB9F98F28F180380180008E
:101D9000019FFFF99174999B06A99B54A99B56A991
:101DA0009B54999FFFF9FFFFFF6E6F74696669632B
:101DB0006174696F6E200063616E63656C005072C0
:101DC000696E742041626F72746564004469736D5A
:101DD0006973730055492041626F72746564004DE8
:101DE000323520500A4D323400526573756D6500EE
:101DF00055492050617573650050617573696E6750
:101E00002E2E2E00726573756D65004D32340052B2
:101E1000756E6F75742044697374206D6D004C6F1E
:101E20006164206D6D00556E6C6F6164206D6D0096
:101E300046696C2E204469612E004520696E206D34
:101E40006D5E33004D3330332055312045256920F8
:101E500053256900504944204175746F74756E654F
:101E6000202A005049442D44202A005049442D493D
:101E7000202A005049442D50202A00200820466185
:101E80006374002008204D6178002008204D696EA1
:101E9000004F6666004F6E004175746F74656D701B
:101EA000005654726176204D696E00566D696E0061
:101EB000566D6178204500566D6178205A00566D48
:101EC0006178205900566D6178205800416D617825
:101ED000204500416D6178205A00416D617820599C
:101EE00000416D6178205800412D54726176656C17
:101EF00000412D5265747261637400416363656CC7
:101F00000056652D4A65726B00565A2D4A65726BF4
:101F10000056592D4A65726B0056582D4A65726BF2
:101F200000452073746570732F6D6D005A205374D3
:101F30006570732F6D6D00592053746570732F6D2C
:101F40006D00582053746570732F6D6D0041647679
:101F5000616E6365642053657474696E6773003FD6
:101F60000043616E63656C00496E6974004D3432E4
:101F70003800496E697469616C697A65204545501D
:101F8000524F4D0046696C616D656E740054656D0D
:101F900070657261747572650053746570732F6D2E
:101FA0006D004A65726B00416363656C65726174B4
:101FB000696F6E0056656C6F636974790053657460
:101FC00020486F6D65204F66667365747300436FBC
:101FD0006E66696775726174696F6E003F004E6569
:101FE000787420506F696E7400446F6E65004E65A2
:101FF0007874004C6576656C696E6720446F6E6519
:1020000021004D6F7665205A004732395332004E19
:1020100065787420506F696E74002569202F202523
:102020007500473239533100473239533200436C1F
:1020300069636B20746F20426567696E00486F6D3D
:10204000696E672058595A005A2056616C756500B0
:10205000496E646578205900496E6465782058009F
:1020600053746F72652053657474696E6773004CA6
:102070006F61642053657474696E6773004C657694
:10208000656C20436F726E65727300426564205AFE
:10209000004661646520486569676874004F66663C
:1020A000004F6E00426564204C6576656C696E6712
:1020B0000045646974204D657368004C6576656CF5
:1020C00020426564004D6F74696F6E003F0043618C
:1020D0006E63656C204F626A656374004E4F0059F1
:1020E00045530043616E63656C204F626A6563749B
:1020F000203D004D61696E00426564004E6F7A7A42
:102100006C650046616E20537065656400436F6EB8
:1021100066696775726174696F6E004C6F616420E7
:1021200053657474696E677300526573746F72657A
:102130002044656661756C74730053746F7265201A
:1021400053657474696E6773005072656865617475
:10215000202420436F6E6600506F776572204F75A4
:1021600074616765004F6666004F6E0052756E6F52
:1021700075742053656E736F7200416476616E638F
:1021800065642053657474696E6773004D61696E90
:10219000004D37303220542564004D363030204217
:1021A0003020542564004D373032203B2564004DEB
:1021B00037303120542564004D373032004D3730F0
:1021C00031004D363030204230004D61696E0043A1
:1021D0006F6E74696E7565004F6666004F6E0052D3
:1021E000756E6F75742053656E736F7200507572E3
:1021F0006765206D6F726500524553554D45204F00
:102200005054494F4E533A005052494E5420504179
:10221000555345440020204E6F7A7A6C653A200071
:102220005061726B696E672E2E2E00000057616937
:102230007420666F720066696C616D656E742063F0
:1022400068616E676500746F207374617274005703
:1022500061697420666F720066696C616D656E7489
:1022600020756E6C6F616400004E6F7A7A6C652029
:1022700068656174696E6700506C6561736520778D
:102280006169742E2E2E0000507265737320627582
:1022900074746F6E00746F2068656174206E6F7A5D
:1022A0007A6C650000496E736572742066696C61B2
:1022B0006D656E7400616E64207072657373206268
:1022C0007574746F6E00746F20636F6E74696E75D1
:1022D00065005761697420666F720066696C616D94
:1022E000656E74206C6F61640000507265737320BA
:1022F000427574746F6E00746F20726573756D65CE
:10230000207072696E7400005761697420666F7284
:10231000207072696E7400746F20726573756D65DC
:102320002E2E2E00005761697420666F7200666958
:102330006C616D656E7420707572676500003E207B
:1023400000256C642E25696D00457874727564658E
:102350006420546F74616C003E20004C6F6E6765A2
:102360007374204A6F622054696D65003E200054EA
:102370006F74616C205072696E742054696D6500D1
:10238000436F6D706C65746564003A20005072692B
:102390006E7420436F756E74003A20003135300042
:1023A00035004245443A20415443203130344754AB
:1023B0002D320052756E61776179205761746368C0
:1023C0003A204F4E004D61782054656D70003331D6
:1023D00035004D696E2054656D7000350045313A09
:1023E000204550434F53203130304B00505355005F
:1023F00047656E657269630050726F746F636F6CCE
:1024000000312E300042617564003235303030309A
:1024100000437265616C69747933442052414D50B8
:1024200053004D657368204C6576656C696E670076
:1024300045787472756465727300310074696E79E1
:102440006D616368696E657333642E636F6D0054EC
:102450004D33442043523130563200323032312D28
:1024600030342D313800322E302E375F4457372E1E
:1024700033004D61726C696E005072696E746572E2
:1024800020537461747300546865726D6973746F5E
:10249000727300426F61726420496E666F00507201
:1024A000696E74657220496E666F004D61696E00D9
:1024B0004D313030300053746F70205072696E743B
:1024C00000526573756D65205072696E7400506FAF
:1024D000776572204F7574616765003F00426163E4
:1024E0006B0053746F70005072696E742066726F67
:1024F0006D204D65646961004368616E6765204DBC
:1025000065646961004D32310041626F757420501D
:1025100072696E746572004368616E676520466912
:102520006C616D656E7400436F6E6669677572618C
:1025300074696F6E0054656D706572617475726553
:10254000004D6F74696F6E00486F7374205374612F
:10255000727400526573756D65205072696E7400F7
:102560004E6F204D656469610043616E63656C2048
:102570004F626A6563740054756E650053746F70C2
:10258000205072696E7400506175736520507269D5
:102590006E7400496E666F2053637265656E003F0E
:1025A000005374617274205072696E740043616EDE
:1025B00063656C005072696E740043616E6E6F7477
:1025C00020656E746572207375626469723A2000CA
:1025D000022E2E004D61696E002100486F74656EF9
:1025E0006420746F6F20636F6C64004261636B00E2
:1025F00050726F63656564004F6666004F6E0053EE
:102600006F667420456E6473746F7073004D6F74E1
:10261000696F6E0044697361626C65205374657004
:1026200070657273004D383400426564204C6576E5
:10263000656C696E6700486F6D65205A00473238D7
:102640005A00486F6D652059004732385900486F6D
:102650006D6520580047323858004175746F204826
:102660006F6D6500473238004D61696E00507265CC
:1026700068656174202420456E6400507265686549
:1026800061742024204265640054656D7065726138
:102690007475726500436F6F6C646F776E00507273
:1026A000656865617420240046616E20537065651D
:1026B00064207E00426564004E6F7A7A6C65004D3E
:1026C00061696E004261627973746570205A0046D8
:1026D0006C6F770046616E205370656564207E00E4
:1026E000426564004E6F7A7A6C6500426564205AD8
:1026F000005370656564004D61696E00486F6D69D7
:102700006E67204661696C6564006F70656E005489
:102710005249474745524544003A200066696C617A
:102720006D656E74007A5F6D696E00795F6D696EBC
:1027300000785F6D696E005265706F7274696E67C4
:1027400020656E6473746F70207374617475730A9E
:102750000020746F6F206C6F6E67206578747275DF
:1027600073696F6E2070726576656E7465640A00B9
:1027700020636F6C6420657874727573696F6E2066
:1027800070726576656E7465640A00000000000072
:10279000000000000000005761726E696E673A2009
:1027A000486F6D696E672042756D70204469766967
:1027B000736F72203C20310A0002020400809D43A6
:1027C00000009B430000C84300000041000000419E
:1027D0000000004000000001000000010000800037
:1027E000555555000000400033333300AAAA2A0093
:1027F0004992240000002000C7711C00999919001B
:10280000D1451700555515003BB11300244912005E
:1028100011111100000010000F0F0F00E3380E001F
:1028200043790D00CCCC0C00C3300C00E8A20B00A7
:1028300064210B00AAAA0A00703D0A009DD8090075
:10284000427B090092240900DCD308008888080034
:102850001042080000000800F0C107008787070049
:1028600075500700711C07003EEB0600A1BC060076
:102870006990060066660600703E06006118060054
:1028800017F4050074D105005BB00500B290050097
:10289000627205005555050078390500B81E05001F
:1028A000050505004EEC040087D40400A1BD04001A
:1028B00090A7040049920400C17D0400EE69040061
:1028C000C7560400444404005C320400082104009C
:1028D00041100400000004003FF00300F8E0030092
:1028E00026D20300C3C30300CCB503003AA80300FB
:1028F0000A9B0300388E0300C08103009F7503000C
:10290000D0690300505E03001D53030034480300E8
:10291000913D03003333030016290300381F0300E1
:1029200097150300300C0300030303000BFA0200A9
:1029300049F10200BAE802005CE002002DD8020072
:102940002DD0020059C80200B0C0020031B9020007
:10295000DAB10200AAAA0200A0A30200BC9C0200F5
:10296000FA9502005C8F0200DF880200828202007A
:10297000457C02002776020027700200436A0200AD
:102980007C640200D05E02003F590200C85302007E
:10299000FFFDFCFAF8F6F4F2F0EEECEAE9E7E5E325
:1029A000E1E0DEDCDAD9D7D5D4D2D0CFCDCBCAC8DE
:1029B000C7C5C3C2C0BFBDBCBAB9B7B6B4B3B2B065
:1029C000AFADACAAA9A8A6A5A4A2A1A09E9D9C9AC1
:1029D00099989795949392908F8E8D8B8A898887FA
:1029E0008684838281807F7E7D7B7A797877767515
:1029F00074737271706F6E6D6C6B6A69686766650F
:102A000064636261605F5E5D5C5B5A5958585756FB
:102A1000555453525150504F4E4D4C4B4A4A4948D1
:102A2000474646454443424241403F3E3E3D3C3B93
:102A30003B3A393838373635353433323231303045
:102A40002F2E2E2D2C2B2B2A2929282727262525EA
:102A500024232322212120201F1E1E1D1C1C1B1B82
:102A60001A1919181817161615151413131212110E
:102A700011100F0F0E0E0D0D0C0C0B0A0A09090890
:102A80000807070606050504040303020201000007
:102A900000809D4300009B430000C84300000000ED
:102AA000000000000000000053657474696E6773D5
:102AB0002053746F72656400454550524F4D204954
:102AC0006E697469616C697A65640A003B20002054
:102AD000204D363033200020440020204D34313248
:102AE00020530046696C616D656E742072756E6F5F
:102AF00075742073656E736F723A002055004C0038
:102B000046696C616D656E74206C6F61642F756EC3
:102B10006C6F6164206C656E677468733A00202086
:102B20004D343133205300506F7765722D4C6F73E5
:102B300073205265636F766572793A0020440020F5
:102B4000490020204D3330342050002044002049DB
:102B50000020204D3330312050005049442073650F
:102B60007474696E67733A00204600204800202084
:102B70004D3134352053004D6174657269616C20AC
:102B800068656174757020706172616D65746572DD
:102B9000733A002020473239205334205A00204A0B
:102BA00000202047323920533320490020204D3463
:102BB00032302053004D65736820426564204C65B7
:102BC00076656C696E673A0020204D3230362058A9
:102BD00000486F6D65206F66667365743A00205813
:102BE0000020530020204D323035204200416476D1
:102BF000616E6365643A20423C6D696E5F73656720
:102C00006D656E745F74696D655F75733E20533CCE
:102C10006D696E5F66656564726174653E20543CE3
:102C20006D696E5F74726176656C5F66656564720E
:102C30006174653E20583C6D61785F785F6A6572AB
:102C40006B3E20593C6D61785F795F6A65726B3EBF
:102C5000205A3C6D61785F7A5F6A65726B3E2045F1
:102C60003C6D61785F655F6A65726B3E0020540061
:102C700020520020204D32303420500041636365E3
:102C80006C65726174696F6E2028756E6974732F3C
:102C90007332293A20503C7072696E745F616363CD
:102CA000656C3E20523C726574726163745F61634F
:102CB00063656C3E20543C74726176656C5F616341
:102CC00063656C3E0020204D3230312058004D614C
:102CD00078696D756D20416363656C6572617469B7
:102CE0006F6E2028756E6974732F7332293A002035
:102CF000204D3230332058004D6178696D756D205C
:102D00006665656472617465732028756E69747395
:102D10002F73293A005374657073207065722075A3
:102D20006E69743A0020440020204D323030205328
:102D3000002044697361626C65640A0046696C61D5
:102D40006D656E742073657474696E67733A0020E4
:102D5000204D3134392043203B20556E6974732057
:102D6000696E2043656C736975730A0020286D6D68
:102D700029002020473231202020203B20556E6939
:102D8000747320696E206D6D000000FA430000FA34
:102D90004300002041000096420000A0420000A035
:102DA000420000C8430000BA42DC050000DC050018
:102DB00000640000004B00000024F4D43050C38EA7
:102DC00020C2A24017828B7011127A910D816CD9AA
:102DD0000AA861E108C7586607615143061E4B5DAA
:102DE00005C145A7041A411104093D980371393101
:102DF000034036DB0265339102D4305402802E1D2D
:102E000002632CEE01752AC501B028A001102781AC
:102E1000018F2564012B244B01E0223401AC211FDA
:102E2000018D200D01801FFC00841EED00971DDF29
:102E300000B81CD200E61BC600201BBC00641AB2FE
:102E400000B219A8000A19A0006A189900D11791B8
:102E50000040178B00B516840031167E00B315793B
:102E6000003A157300C7146F0058146A00EE136619
:102E7000008813630025135E00C7125B006C1257B5
:102E80000015125400C111510070114F0021114B57
:102E900000D61049008D1047004610440002104231
:102EA00000C00F4000800F3E00420F3C00060F3B69
:102EB00000CB0E3800930E37005C0E3500270E3421
:102EC00000F30D3200C10D3100900D3000600D2E69
:102ED00000320D2D00050D2C00D90C2B00AE0C2955
:102EE00000850C29005C0C2700350C27000E0C26F1
:102EF00000E80B2400C40B2400A00B23007D0B234F
:102F0000005A0B2100390B2100180B2000F80A1F72
:102F100000D90A1E00BB0A1E009D0A1D00800A1D62
:102F200000630A1C00470A1B002C0A1B00110A1A26
:102F300000F7091A00DD091900C4091900AB0919C5
:102F400000920917007B091800630917004C091645
:102F50000036091600200916000A091500F50815A3
:102F600000E0081400CC081400B8081400A40814E9
:102F700000900813007D0812006B08130058081217
:102F8000004608120034081100230811001208112D
:102F90000001081100F0071000E0071000D0071032
:102FA00000C0071000B0070F00A107100091070E26
:102FB0000083070F0074070F0065070E0057070E08
:102FC0000049070E003B070D002E070E0020070DDD
:102FD0000013070D0006070D00F9060C00ED060DA5
:102FE00000E0060C00D4060C00C8060C00BC060C61
:102FF00000B0060C00A4060B0099060C008D060B11
:103000000082060B0077060B006C060B0061060AB7
:103010000057060B004C060A0042060A0038060A52
:10302000002E060A0024060A001A060A00100609E5
:103030000007060A00FD050900F4050900EB050973
:1030400000E2050900D9050900D0050900C70509F6
:1030500000BE050900B5050800AD050800A5050975
:10306000009C050800940508008C050800840508EC
:10307000007C050800740508006C0507006505085C
:10308000005D050700560508004E050700470507C7
:10309000004005080038050700310507002A05072C
:1030A00000230507001C050600160507000F05078D
:1030B000000805060002050700FB040600F50407EA
:1030C00000EE040600E8040600E2040700DB040644
:1030D00000D5040600CF040600C9040600C3040698
:1030E00000BD040600B7040600B1040500AC0406E8
:1030F00000A6040600A00405009B04060095040534
:1031000000900406008A040500850405008004067A
:10311000007A04050075040500700405006B0405C1
:103120000066040500610405005C04050057040501
:1031300000520405004D0405004804050043040541
:10314000003E0404003A0405003504050030040480
:10315000002C04050027040400230405001E0404B9
:10316000001A04040016040500110404000D0404F0
:1031700000090405000404040000040400FC030426
:1031800000F8030400F4030400F0030400EC03045B
:1031900000E8030400E4030400E0030400DC03048B
:1031A00000D8030400D4030400D0030400CC0304BB
:1031B00000C8030300C503030024F404D9201BC482
:1031C0000C5C0E9804C4095F0265077101F405F9EF
:1031D00000FB04B30048048700C10369005803558D
:1031E0000003034500BE023A008402310053022A64
:1031F000002902250004022000E4011C00C8011976
:1032000000AF011700980114008401130071011030
:10321000006101100051010E0043010D0036010B49
:10322000002B010B0020010B00150109000C010906
:103230000003010800FB000800F3000800EB000792
:1032400000E4000600DE000600D8000600D20006FA
:1032500000CC000500C7000500C2000500BD000449
:1032600000B9000400B5000400B1000400AD000482
:1032700000A9000400A5000300A20003009F0004B1
:10328000009B0003009800030095000200930003D8
:1032900000900003008D0002008B000300880002F4
:1032A000008600020084000300810002007F00020B
:1032B000007D0002007B000200790002007700011F
:1032C000007600020074000200720001007100022A
:1032D000006F0002006D0001006C0002006A000136
:1032E000006900020067000100660001006500013E
:1032F0000064000200620001006100010060000142
:10330000005F0002005D0001005C0001005B000145
:10331000005A000100590001005800010057000147
:103320000056000100550001005400010053000048
:103330000053000100520001005100010050000143
:10334000004F0001004E0000004E0001004D000142
:10335000004C0001004B0000004B0001004A00013E
:10336000004900010048000000480001004700013A
:103370000046000000460001004500000045000135
:10338000004400010043000000430001004200002F
:103390000042000100410000004100010040000126
:1033A000003F0000003F0001003E0000003E000121
:1033B000003D0000003D0001003C0000003C00001A
:1033C000003C0001003B0000003B0001003A00000F
:1033D000003A000100390000003900010038000007
:1033E00000380000003800010037000000370001FD
:1033F00000360000003600000036000100350000F5
:1034000000350000003500010034000000340000E9
:1034100000340001003300000033000000330001DD
:1034200000320000003200000032000100310000D4
:1034300000310000003100010030000000300000C9
:1034400000300001002F0000002F0000002F0000BE
:10345000002F0001002E0000002E0000002E0001B1
:10346000002D0000002D0000002D0000002D0001A7
:10347000002C0000002C0000002C0000002C00019B
:10348000002B0000002B0000002B0000002B00018F
:10349000002A0000002A0000002A0000002A000183
:1034A0000029000000290000002900000029000078
:1034B000002900010028000000280000002800006A
:1034C000002800000028000100270000002700005D
:1034D0000027000000270000002700010026000050
:1034E0000026000000260000002600000026000143
:1034F0000025000000250000002500000025000038
:103500000025000000250001002400000024000028
:10351000002400000024000000240001002300001B
:10352000002300000023000000230000002300000F
:103530000023000000230001002200000022000000
:1035400000220000002200000022000000220001F2
:1035500000210000002100000021000000210000E7
:1035600000210000002100000021000100200000D7
:1035700000200000002000000020000000200000CB
:10358000002000000020000000200001001F0000BB
:10359000001F0000001F0000001F0000001F0000AF
:1035A000001F0000001F0001001E0000001E0000A0
:1035B000001E0000001E000000393000003325000E
:1035C0000087190000B00F0000DB080000BD0400F8
:1035D00000740200003F01000020436F756E7420EC
:1035E000583A0042656400453100626564002C2051
:1035F00073797374656D2073746F707065642120C6
:103600004865617465725F49443A20004865617499
:10361000696E67204661696C65640048656174691C
:103620006E67206661696C6564004D3131322053EC
:10363000687574646F776E001000C90210012C0168
:103640004001220170011801B0010E01F0010401D6
:103650005002FA00B002F0003003E600D003DC00B4
:103660009004D2007005C800A006BE000008B40097
:10367000B009AA00D00BA000600E960060118C006B
:103680000015820020197800C01D6E00A022640081
:10369000B0275A00902C500000314600E0343C0026
:1036A00010383200903A2800603C1E00A03D140003
:1036B000803E0A00203F0000544845524D414C20B6
:1036C00052554E4157415900546865726D616C20E6
:1036D00052756E61776179004572723A204D41589A
:1036E00054454D50004D415854454D502074726919
:1036F000676765726564004572723A204D494E54A1
:10370000454D50004D494E54454D502074726967E7
:10371000676572656400202F002042403A00204017
:103720003A0020573A0020573A00496E76616C699A
:10373000642065787472756465720A007C3C3E5E34
:103740002B3D3F2F5B5D3B2C2A225C0043616E6E5C
:103750006F74206F70656E207375626469722000EB
:1037600041425300504C4100534420496E6974203B
:103770004661696C0053442063617264206F6B0A78
:10378000006F70656E526F6F74206661696C65645E
:103790000A00766F6C756D652E696E6974206661BE
:1037A000696C65640A004E6F205344206361726443
:1037B0000A000A4D3234004D3233202573002E0AA0
:1037C000006F70656E206661696C65642C204669C7
:1037D0006C653A200046696C652073656C6563749E
:1037E00065640A002053697A653A200046696C6571
:1037F000206F70656E65643A2000454E4420535535
:1038000042524F5554494E450A002220706F7300B2
:103810002220706172656E743A2200535542524FF5
:103820005554494E452043414C4C207461726765A4
:10383000743A220053756263616C6C204F76657236
:10384000666C6F77004578636565646564206D61BB
:103850007820535542524F5554494E452064657067
:1038600074683A002E0A0044656C6574696F6E20B6
:103870006661696C65642C2046696C653A20004677
:10388000696C652064656C657465643A0053442016
:103890007072696E74696E67206279746520004E7B
:1038A0006F74205344207072696E74696E670A00E9
:1038B0002F6175746F25632E670057726974696E86
:1038C0006720746F2066696C653A200066726573C4
:1038D0006800646F696E67002066696C653A200055
:1038E0004E6F77200002FD55555555555FFFFFFF80
:1038F000FFFFFFFFFFFFFE00000000003FFFFFFF94
:10390000FFFFFFFFFFFFFD000007FFFFFFFFFFFFBF
:10391000FFFFFFFFFFFFFE07C00555555555555FDB
:10392000FFFFFFFFFFFFFC0A200600000000003F32
:10393000FFFFFFFFFFFFFE141005000007FFFFFF62
:10394000FFFFFFFFFFFFFC28080607C00555555580
:1039500055555FFFFFFFFE5404040A2006000000D7
:1039600000003FFFFFFFFC60040614100500000785
:10397000FFFFFFFFFFFFFE50040428080607C005F5
:1039800055555555555FFC6004065404040A20063D
:1039900000000000003FFE54041C600406141005E3
:1039A00000000000001FFC28082E50040428080610
:1039B00007C00001F03FFE141054600406540404D4
:1039C0000A200002081FFC0A206654041C6004063A
:1039D00014100005043FFE07C05428082E500404AC
:1039E0002808000A021FFC00002E14105460040670
:1039F00054040015013FFE00001C0A206654041CFC
:103A000060040018011FFC00000607C05428082E9F
:103A100050040014013FFE00000400002E14105456
:103A200060040018011FFCFFFFFE00001C0A206656
:103A300054041C15013FFED5555400000607C05420
:103A400028082A0A021FFC84104600000400002EE9
:103A500014105105043FFEC41044FFFFFE00001C7B
:103A60000A206102881FFC841046D55554000006C8
:103A700007C05101F03FFE8410448410460000044A
:103A800000002A00001FFCC41046C41044FFFFFEC3
:103A900000001C00003FFE841044841046D555549D
:103AA00000000000001FFCD55556841044841046C9
:103AB00000000000003FFCFFFFFCC41046C410449F
:103AC000FFFFFFFFFF9FFE000006841044841046A6
:103AD000D555555555BFFD555554D55556841044AB
:103AE00084104104109FFFFFFFFCFFFFFCC4104641
:103AF000C410410411BFFFFFFFFE00000684104404
:103B000084104104109FFFFFFFFD555554D55556B5
:103B100084104104109FFFFFFFFFFFFFFCFFFFFC2D
:103B2000C410410411BFFFFFFFFFFFFFFE000006AE
:103B300084104104109FFFFFFFFFFFFFFD55555408
:103B4000D555555555BFFFFFFFFFFFFFFFFFFFFC9A
:103B5000FFFFFFFFFF9FFFFFFFFFFFFFFFFFFFFED6
:103B600000000000003FFFFFFFFFFFFFFFFFFFFD22
:103B700055555555555FFFFFFFFFFFFFFFFFFFFF47
:103B8000FFFFFFFFFFFFFFFFFFFFFFFFFFFFFFFF45
:103B9000FFFFFFFFFFFFFFFFFFFFFFFFFFFFFFFF35
:103BA000FFFFFFFFFFFFFFFFFFFFFFFFFFFFFFFF25
:103BB000FFFFFFFFFFFFE02EFB7DFBFBCFC1DFBB65
:103BC0003EC0E1FE3C1FFDEE7B39F9F3CF9EDFBB2B
:103BD0003EDFDEFCDDE7FDEE3BBBF9EBD7BF5FBBB5
:103BE0005EDFDEFDEDF7FDEEBBD3FAEBB73FDFBBEB
:103BF0004EDFDFFFCDF3FDEEDBC7FAEBBB7FC03B53
:103C00006EC0E3FF1DF3FDEECBEFFADBBB7FDFBB46
:103C100066DFF8FFCDF3FDEEEBEFFB5B033F5FBB31
:103C200076DFFE7FEDF3FDEEF3EFFB5B79BEDFBBEE
:103C30007ADFDE7DEDF7FDEEF3EFFBBAFD9EDFBB35
:103C40007CDFDEFDCDE7FDEEFBEFFBBAFDC1DFBBA8
:103C50007EC0E0FE1C1F6D61726C696E66772E6F10
:103C6000726700322E302E375F4457372E33001FD5
:103C7000FFFFFFFFFFFF600000000001FF400000AA
:103C8000000000FF8000000000007F83CF00000CD8
:103C9000303F87FF80000C301F867980000C000FBA
:103CA0008C30C7838C30E78C30CFC7CC31F38C306D
:103CB000DCECEC33B98C30D86C6C33198C30D06CB4
:103CC0000C33198C30D86C0C33198C30DC6C0E3BF7
:103CD000198C30CF7C079F198C30C77C038F19401B
:103CE000000000000002600000000000061FFFFF4F
:103CF000FFFFFFF870012C0190012701B0012201A4
:103D0000C0011D01F00118011002130130020E0163
:103D10006002090190020401C002FF000003FA00E2
:103D20004003F5008003F000D003EB002004E60020
:103D30007004E100E004DC004005D700C005D200BB
:103D40004006CD00D006C8008007C3003008BE0082
:103D5000F008B900C009B400B00AAF00B00BAA0067
:103D6000D00CA500000EA000500F9B00C0109600C4
:103D70005012910000148C00C0158700B01782000B
:103D8000B0197D00D01B7800001E730040206E002B
:103D900090226900F024640040275F0090295A00B7
:103DA000E02B5500102E500020304B001032460002
:103DB000E033410090353C00103737007038320056
:103DC000A0392D00B03A2800A03B2300603C1E0023
:103DD000103D1900903D1400103E0F00703E0A0087
:103DE000C03E0500003F0000403FFBFF803FF6FF64
:103DF000C03FF1FF2020506C616E6E6572427566A7
:103E000066657242797465733A2000204672656572
:103E1000204D656D6F72793A2000436F6D70696C4B
:103E200065643A2041707220323420323032310AD7
:103E300000204C61737420557064617465643A208D
:103E4000323032312D30342D3138207C20417574A0
:103E5000686F723A2054696E794D616368696E6566
:103E60007333440A00322E302E375F4457372E33D7
:103E70000A004D61726C696E0020536F6674776141
:103E800072652052657365740A0020576174636817
:103E9000646F672052657365740A002042726F7701
:103EA0006E206F75742052657365740A0020457822
:103EB0007465726E616C2052657365740A00506F90
:103EC00077657255700A0073746172740A00473224
:103ED000385859004D31303031006572726F7220A0
:103EE00077726974696E6720746F2066696C650A01
:103EF00000446F6E6520736176696E672066696C39
:103F0000652E0A004D323900456E6473746F70730C
:103F10000025532025632025632025632025630089
:103F2000205A3A0020593A0020583A00656E6473CE
:103F3000746F7073206869743A200000000A0B02E5
:103F4000090C0D0E0807030401000000000000002A
:103F50000000000000000000000000000000000061
:103F6000000000000000001211100000000000001E
:103F70000000000000000000000000000000000041
:103F800000004D6F76652025736D6D004D6F766571
:103F900020302E316D6D004D6F766520316D6D00D6
:103FA0004D6F76652031306D6D004D6F7665204127
:103FB000786973004578747275646572004D6F7628
:103FC00065205A004D6F76652059004D6F7665204B
:103FD0005800643760374368616E67652046696CD6
:103FE000616D656E7400556E6C6F61642046696C1E
:103FF000616D656E74004C6F61642046696C616D23
:10400000656E7400507265686561742043757374E1
:104010006F6D0050726568656174202400426163B1
:104020006B00FFFFFF486F6D6520257325732573B7
:104030002046697273740073686F770062757474D8
:104040006F6E00626567696E0044697361626C65DA
:1040500052756E6F75740050757267654D6F72653D
:104060000050617573656400436F6E74696E7565A9
:10407000004C6F61642046696C616D656E742054FC
:1040800000496E736572742066696C616D656E744B
:1040900020616E642073656E64204D3130380A00F3
:1040A000220A00556E6B6E6F776E20636F6D6D61C7
:1040B0006E643A2022002042002050006F6B0054B2
:1040C0004D33442043523130563220526561647979
:1040D0002E005072696E74696E672E2E2E0050721B
:1040E000696E742050617573656400204500205A24
:1040F00000205900204D393220580020453A002038
:104100005A3A0020593A00583A0020746F6F206CD8
:104110006F6E6720657874727573696F6E20707248
:104120006576656E7465640A0020636F6C64206553
:104130007874727573696F6E2070726576656E74CF
:1041400065640A00526573656E643A20006E6F7490
:10415000696669636174696F6E2000000022002542
:104160000028002B002E0031003400020100000561
:104170000108010B0100002100240027002A002D66
:10418000003000330001010000040107010A0105AD
:10419000050505070508080808020202020A0A08C0
:1041A00008040404040101010101010101030303E6
:1041B0000303030303040707070C0C0C0C0C0C0C83
:1041C0000C0202020206060606060606060B0B0B8A
:1041D0000B0B0B0B0B0102102020080810204010C5
:1041E00020408002010201080402010102040810BB
:1041F00020408080402010080402018004020180D9
:104200004020100804020108040201010204081001
:104210002040800102040810204080009A013201F1
:1042200011241FBECFEFD1E2DEBFCDBF00E00CBF37
:1042300013E0A0E0B2E0EAE1F5EB02E00BBF02C060
:1042400007900D92A836B107D9F728E1A8E6B3E0A8
:1042500001C01D92AF30B207E1F711E2CFE0D1E229
:1042600000E006C021970109802FFE010F94E3565C
:10427000CE30D10780E00807A9F70F9495450D943B
:104280007B5A0C940000FC0184910895FC0180810C
:1042900008951198000000009091020187FD90950B
:1042A000917090930001119A00000000000000003E
:1042B0001198000000009091020186FD9095917088
:1042C00090930001119A0000000000000000119876
:1042D000000000009091020185FD909591709093EF
:1042E0000001119A00000000000000001198000079
:1042F00000009091020184FD9095917090930001CF
:10430000119A000000000000000011980000000059
:104310009091020183FD9095917090930001119A04
:1043200000000000000000001198000000009091C3
:10433000020182FD9095917090930001119A000006
:1043400000000000000011980000000090910201A0
:1043500081FD9095917090930001119A00000000EA
:10436000000000001198000000008091020181709F
:1043700080930001119A00000000000000000895E1
:1043800090E080E00895CF93DF93DB01F9019C91E9
:104390009130C1F0943080F094509C938830D1F4E7
:1043A00080819181009771F0019791838083480FFC
:1043B000591FEA01188206C08C3539F49C5F9C9322
:1043C000943041F4DF91CF9108958B3339F781E038
:1043D0008C93F8CF20813181B9016F5F7F4F71835A
:1043E0006083420F531FEA018883808191818F355A
:1043F00091056CF7E7CF0F931F9381E00091D815DB
:104400001091D9152091DA153091DB154091D41512
:104410005091D5156091D6157091D71504171507D1
:104420002607370708F480E01F910F91089590E068
:1044300080E00895282F90916308833021F495FD42
:104440000FC094FD0FC0892F90E0B0E0A0E004C041
:10445000B695A795979587952A95D2F78170089577
:1044600081E0089580E0089510924A0880915102F9
:1044700090915202A0915302B09154028093390658
:1044800090933A06A0933B06B0933C060895129A87
:104490000895269A2E9A0895AF92BF92CF92DF92F6
:1044A000EF92FF920F931F93CF93DF936B01E9017C
:1044B0004A3009F4C1C0453109F073C0DB011296DE
:1044C000ED91FC91F280C681D781809102018095A7
:1044D00082708093000188E28A950000E9F7BF2C82
:1044E000B29420EFB22230E1A32EAF0C48E2E42ECA
:1044F00088EF0E9449218E2D8A950000E9F7BFE1DF
:10450000BF1508F485C08F2D807780680E944921EF
:104510008B2D0E9449218E2D8A950000E9F780E8B5
:104520000E94492180E00E9449218E2D8A95000039
:10453000E9F78AEF0E9449218E2D8A950000E9F75C
:104540008E01005F1F4F8881807F0E9449218991E1
:104550008295807F0E944921C017D107A1F78E2D37
:104560008A950000E9F7F394E0E1BE0EFA10C0CF9F
:1045700080910201827080930001D6011296CD9144
:10458000DC91CE010F94AD38811147C2DF91CF91FC
:104590001F910F91FF90EF90DF90CF90BF90AF9061
:1045A0000895FB0102811381423309F4F1C108F43B
:1045B000F5C1463409F4E2C1473409F4E5C14B338F
:1045C00029F589812B81D80112966C911297139647
:1045D0004C91213009F438C2233009F002C238EF7F
:1045E000380F582F91E0431708F490E041E053173B
:1045F00008F040E031E0561708F430E0592F542B12
:10460000352309F016C2942309F013C281E0BECF0E
:1046100080EE8F0D8068807F0E9449218F2D8295CA
:10462000807F0E9449218E2D8A950000E9F780E85D
:104630000E94492180E877CF8091010182608093B8
:10464000010180910201827080930001809101013B
:10465000816080930101809102018170809300014B
:10466000099A119A809102018095827080930001CD
:1046700088E28A950000E9F788E790E0CEE9DFE07C
:10468000FE013197F1F70197D9F788EF0E94492190
:1046900018E2812F8A950000E9F780E20E94492103
:1046A00080E00E944921812F8A950000E9F780E08F
:1046B0000E94492180E80E944921812F8A950000AB
:1046C000E9F780E00E94492180E10E944921812F81
:1046D0008A950000E9F7CE010197F1F7CE01019725
:1046E000F1F7CE010197F1F7CE010197F1F7CE0175
:1046F0000197F1F7CE010197F1F7CE010197F1F79C
:10470000CE010197F1F7CE010197F1F7CE010197A4
:10471000F1F7CE010197F1F7CE010197F1F7CE0144
:104720000197F1F7CE010197F1F72197F1F780E2B8
:104730000E94492180E40E944921812F8A9500002E
:10474000E9F780E20E94492180E60E9449211A95FA
:104750000000E9F710E0D0E0C8E28D2F8077806894
:104760000E944921812F0E9449218C2F8A950000A7
:10477000E9F780E80E94492180E00E9449218C2FBE
:104780008A950000E9F78AEF0E9449218C2F8A95CB
:104790000000E9F790E2119800000000809102010A
:1047A000817080930001119A000000000000000059
:1047B0001198000000008091020181708093000137
:1047C000119A000000000000000011980000000095
:1047D00080910201817080930001119A0000000015
:1047E000000000001198000000008091020181701B
:1047F00080930001119A0000000000000000119851
:104800000000000080910201817080930001119AE4
:1048100000000000000000001198000000008091DE
:104820000201817080930001119A000000000000D5
:1048300000001198000000008091020181708093B7
:104840000001119A00000000000000001198000013
:10485000000080910201817080930001119A000094
:10486000000000000000119800000000809102018B
:10487000817080930001119A000000000000000088
:104880001198000000008091020181708093000166
:10489000119A0000000000000000119800000000C4
:1048A00080910201817080930001119A0000000044
:1048B000000000001198000000008091020181704A
:1048C00080930001119A0000000000000000119880
:1048D0000000000080910201817080930001119A14
:1048E000000000000000000011980000000080910E
:1048F0000201817080930001119A00000000000005
:1049000000001198000000008091020181708093E6
:104910000001119A00000000000000001198000042
:10492000000080910201817080930001119A0000C3
:104930000000000000008C2F8A950000E9F79150DC
:1049400009F029CF88EF0E9449218C2F8A95000019
:10495000E9F7DF5F105FD03209F0FFCE80E00E9400
:10496000492180EC0E944921CA950000E9F7809115
:10497000020182708093000181E008CED801159673
:104980008C91888381E002CEF80181818883FACFFF
:10499000B901C8010F94CA3881E0F8CD443171F0F3
:1049A000473109F033CE1882F801828189838581ED
:1049B00081508A8383818B8381E0E8CDD80115966D
:1049C0004C91159750E0440F551F70E060E016962B
:1049D0008D919C910F941C5AC8010F94C33881E0AB
:1049E000D5CD481708F412CE861708F40FCEFA80FA
:1049F000E12CD12C243070F41DC0BE01C8010F94ED
:104A0000CA38898198819D0D98838E0D8983FF0C0A
:104A100009F4FCCDF7FEF6CFF0CF4D8150E0440F06
:104A2000551F70E060E08E819F810F941C5A81E0D9
:104A3000ADCDFA8030E0F901ED55FD4FD080215623
:104A40003D4FF901E080E6CF58E0580F382FCACD2E
:104A5000EF92FF920F931F93CF93DF93EC018B01A3
:104A60007A018A859B858617970731F0888199811D
:104A70000F94A33A1B870A87B701888199810F9405
:104A8000922C2E813F81820F932F911D9F838E83C5
:104A900090E080E0DF91CF911F910F91FF90EF9018
:104AA00008959F92AF92BF92CF92DF92EF92FF92C2
:104AB0000F931F93CF93DF93EC018B01942EA52EC0
:104AC0008A859B858617970731F0888199810F9495
:104AD000A33A1B870A8788859985019649F5BC808A
:104AE0000A818E81080FC880D980D6015596ED9134
:104AF000FC91C6011995B80EE92CFA2C10E0F701CB
:104B000021917F01211127C08E819F81810F911DED
:104B10009F838E8390E080E0DF91CF911F910F9172
:104B2000FF90EF90DF90CF90BF90AF909F9008954F
:104B30000E811F81692D7A2D888199810F94922C85
:104B4000800F912F911D288539852817390738F650
:104B500081E090E0E1CF4B2D602FC6010F94FB3A2E
:104B6000080F180FCCCFDF92EF92FF920F931F9395
:104B7000CF93DF93EC01D62E1CAD0BAD7C0184E00E
:104B8000E80EF11CE98DFA8DC7011995412F480FE8
:104B90002D2D602FC7010F94FB3A9BAD890F8BAF72
:104BA00081E090E0DF91CF911F910F91FF90EF9006
:104BB000DF900895AB01BC014093D8155093D915EF
:104BC0006093DA157093DB158FE397E10C943FCF78
:104BD000809323028032B8F590910405891724F060
:104BE00091E0980F909304054091000550910105C4
:104BF0006091020570910305082E04C076956795B3
:104C0000579547950A94D2F7417040939B0F87FDC3
:104C10001DC0282F082E000C330B3F938F9386E87E
:104C200099E09F938F9386E999E09F938F931F92CA
:104C30000E947EB38DB79EB707960FB6F8949EBFBD
:104C40000FBE8DBF089510929B0FE1CF0D941B40B6
:104C50000F931F93CF93DF9300D01F92CDB7DEB792
:104C60009C0101E318E090E1E6EEFFE0D80101903D
:104C70000D929A95E1F7F9012081318142815381AA
:104C8000F80160857185828593850F94EC56F80153
:104C9000608771878287938780E090E0A0EAB0E424
:104CA00089839A83AB83BC83CE0101960E94D8F797
:104CB0000F900F900F900F90DF91CF911F910F9158
:104CC00008952F923F924F925F926F927F928F92B0
:104CD0009F92AF92BF92CF92DF92EF92FF921F937B
:104CE000CF93DF93CDB7DEB72C970FB6F894DEBF26
:104CF0000FBECDBF7A011901DC012D913D914D917F
:104D00005C912D833E834F835887FB014080518007
:104D1000628073808090E60F9090E70FA090E80F7C
:104D2000B090E90FA50194016D817E818F819885F6
:104D30000F94FA4F81110EC011E0A301920160910E
:104D4000EA0F7091EB0F8091EC0F9091ED0F0F94A3
:104D5000FA4F811110E0D1012D913D914D915C915F
:104D600029873A874B875C87F701C080D180E28032
:104D7000F3802091090230910A0240910B02509178
:104D80000C02C701B6010F94FA4F882309F44EC0F4
:104D9000C0920902D0920A02E0920B02F0920C0239
:104DA0008091F20F9091F30FA091F40FB091F50F55
:104DB0004091EA0F5091EB0F6091EC0F7091ED0F65
:104DC0008092310890923208A0923308B092340851
:104DD000409335085093360860933708709338082D
:104DE000C0923908D0923A08E0923B08F0923C0811
:104DF00080933D0890933E08A0933F08B0934008ED
:104E000020E030E040E05FE36091C90F7091CA0F8D
:104E10008091CB0F9091CC0F0F94605069837A836F
:104E20008B839C83CE0101960E94D8F72D813E8111
:104E30004F815885209331083093320840933308CE
:104E400050933408409235085092360860923708E3
:104E500070923808D1012D913D914D915C916091F6
:104E60003D0870913E0880913F08909140080F9452
:104E7000EC5660933D0870933E0880933F089093F2
:104E8000400811112FC020E030E0A90169857A8522
:104E90008B859C850F94FA4F811133C060E070E0E0
:104EA00088EC92E469837A838B839C83CE0101969C
:104EB0000E94D8F72C960FB6F894DEBF0FBECDBF78
:104EC000DF91CF911F91FF90EF90DF90CF90BF9037
:104ED000AF909F908F907F906F905F904F903F909A
:104EE0002F9008952AEF3EE74AE25FE36091CD0FED
:104EF0007091CE0F8091CF0F9091D00F0F94605092
:104F0000D1CF60E070E080EA91E4CCCF8091BB0427
:104F10009091BC04009731F04AE050E070E060E00E
:104F20000D94154E60E070E0CB01089580915C090E
:104F300082FF0BC063E682E79AE00E9499B30F9468
:104F4000B7320E9464BA81E0089580E008958091AC
:104F5000BB049091BC04009731F04AE050E070E04F
:104F600060E00D94E74C60E070E0CB010895AF92F3
:104F7000BF92CF92DF92EF92FF920F931F93CF9346
:104F8000DF93EC015B018A01FB01199587FD16C0D7
:104F9000C82ED12CF12CE12C2196F801C082D182AF
:104FA000E282F382CE01DF91CF911F910F91FF90AA
:104FB000EF90DF90CF90BF90AF900895982F907EA4
:104FC000903CA9F48F7190E0B0E0A0E06C017D010D
:104FD00056E0CC0CDD1CEE1CFF1C5A95D1F7CE011F
:104FE0000196F50119958F73C82A2296D6CF982F6E
:104FF000907F903E11F58F7090E0B0E0A0E06C01E2
:105000007D0136E0CC0CDD1CEE1CFF1C3A95D1F77F
:10501000CE010196F50119958F73C82A46E0CC0C94
:10502000DD1CEE1CFF1C4A95D1F7CE010296F5015E
:1050300019958F73C82A2396B0CF982F987F903FE9
:1050400079F5877090E0B0E0A0E06C017D0186E02A
:10505000CC0CDD1CEE1CFF1C8A95D1F7CE0101960D
:10506000F50119958F73C82A96E0CC0CDD1CEE1C57
:10507000FF1C9A95D1F7CE010296F50119958F7311
:10508000C82A26E0CC0CDD1CEE1CFF1C2A95D1F7AB
:10509000CE010396F50119958F73C82A24967DCF0A
:1050A000982F907C903841F4807C803869F4219668
:1050B000CE01F5011995F8CF8E7F8D3F28F021960E
:1050C000CE01F5011995F8CFC12CD12C760165CF11
:1050D0009CE0899F802D112491E0980F9093050505
:1050E0002CE0280F20932B0830E02E5F3F4F40919B
:1050F000A2154217130619F014F080E008952091CC
:10510000A4159217D0F7662341F08E5F0F94BD3936
:1051100080912B088E5F0F94BD3980912B08909160
:10512000A215891750F32091A41590910505291710
:1051300020F31092A5158093A61581E00895CF93D2
:105140008091F704811154C01092A5151092A615F4
:105150001092A71510927315109272151092751572
:10516000109274151092771581E08093761582E283
:105170008093781510927D1510927C15E1E9F5E188
:105180002FE935E18FEF81932E173F07E1F7C1E05B
:10519000C0938E1520E131E0309384152093831560
:1051A000C0938515109286151092871590E4909300
:1051B0008815109289152AE232E03093A0152093C9
:1051C0009F1526E132E0309371152093701597E119
:1051D0009093951591E19093961590E19093931586
:1051E00080939215809391150F94E438C093F7043F
:1051F00081E08093F8048FE197E190930F158093FD
:105200000E151092111510921015CF91089520913E
:10521000F604022E000C330B8217130641F0809324
:10522000F6046FE177E18EE695E10D94A33A0895D7
:10523000CF92DF92EF92FF920F931F93CF93DF9362
:10524000CDB7DEB72C970FB6F894DEBF0FBECDBF3B
:105250006F3F71058105910509F0D0F48AE695E16B
:105260000E94B325E0917215F091731531968491E7
:1052700090E02C960FB6F894DEBF0FBECDBFDF9145
:10528000CF911F910F91FF90EF90DF90CF900895F5
:10529000F090A515E090A6152091F80421110FC0FB
:1052A0004FEF56E16E2D8F2D0F94673B90E080E01D
:1052B000F80EF092A515E092A6159927DACFC090C6
:1052C0007215D09073152EE635E13A8329832F2D80
:1052D00030E03C832B832E2D30E03E832D831886D7
:1052E0001F822FEF3FEF3A8729871C861B8601E537
:1052F00015E29E012F5F3F4FAB01BC01C6010F9429
:105300003524B6018EE695E10F94A33A8F819885F6
:10531000CFCFCF93DF93FC0125AD211104C021E055
:1053200025AF0F94E438C0917015D0917115E091BC
:105330009F15F091A01582E01995E0919F15F091CD
:10534000A01581E0199530E020E044E1BE018EE631
:1053500095E10F94E03821EA35E147E1BE018EE6A0
:1053600095E10F94E038E0919F15F091A01580E051
:10537000DF91CF911994CF92DF92EF92FF920F932A
:105380001F93CF93DF93CDB7DEB72C970FB6F8946A
:10539000DEBF0FBECDBFF090A515E090A615209101
:1053A000F80421111DC04FED56E16E2D8F2D0F9485
:1053B000673B90E080E0F80EF092A515E092A6150C
:1053C00099272C960FB6F894DEBF0FBECDBFDF91A4
:1053D000CF911F910F91FF90EF90DF90CF900895A4
:1053E000C0907215D09073152EE635E13A8329836B
:1053F0002F2D30E03C832B832E2D30E03E832D83F8
:1054000018861F827A8769871C861B8601E515E24C
:105410009E012F5F3F4F43E451E2BC01C6010F9450
:10542000F924B6018EE695E10F94A33A8F81988511
:10543000C2CF6FEF7FEF0C94BB29CF92DF92EF9238
:10544000FF920F931F93CF93DF93CDB7DEB72C97C7
:105450000FB6F894DEBF0FBECDBFF090A515E0905B
:10546000A6152091F80421111DC04FEB56E16E2DB9
:105470008F2D0F94673B90E080E0F80EF092A51519
:10548000E092A61599272C960FB6F894DEBF0FBEB2
:10549000CDBFDF91CF911F910F91FF90EF90DF90E3
:1054A000CF900895C0907215D09073152EE635E117
:1054B0003A8329832F2D30E03C832B832E2D30E03F
:1054C0003E832D8318861F827A8769871C861B86F8
:1054D00001E515E29E012F5F3F4F46E451E2BC011A
:1054E000C6010F94F924B6018EE695E10F94A33A14
:1054F0008F819885C2CFBF92CF92DF92EF92FF92B9
:105500000F931F93CF93DF938B01F42EE90141FB9F
:10551000662760F90E946828882309F45AC0B12CD4
:105520000115110521F0C8010E9435BBB82EE12CF0
:10553000209721F0CE010E9420BDE82E80E8C82EE1
:10554000D12CF0FE1EC085E190E08B199109B7FCCB
:1055500093958E199109E7FC939597FD0196959582
:105560008795F82E30E8C32ED12CFA94F7FC09C0A9
:1055700060E270E080E090E00E941829C81AD90A21
:10558000F4CFBB2099F0C60166E070E00F94BB56E3
:10559000262F40912D0850912E0860912C08C801AB
:1055A0000E9475BA96E0899F60011124EE2031F0C7
:1055B000B601CE010E941D2AC81AD90A87E0C81672
:1055C000D10438F060E270E080E090E00E94182999
:1055D000F3CFDF91CF911F910F91FF90EF90DF906C
:1055E000CF90BF9008956FEF7FEF0C941D2AAF927C
:1055F000BF92CF92DF92EF92FF920F931F93CF93C0
:10560000DF935C016B010E9435BBE82EC6010E944E
:1056100020BDF12C03E110E0081B1109C5E20E15B5
:105620001F050CF4CFE18C2F90E09C012E5F3F4FC3
:105630004091A2154217130609F0CCF50997209165
:10564000A415281719069CF140912D0850912E0899
:1056500060912C081092A515C093A61525E1C501EF
:105660000E9475BAD1E0C114D104B1F06AE370E0D0
:1056700080E090E00E9418290E151F05D4F4C45F45
:105680008091A215C81740F02091A4154C2F4950C5
:10569000550B241715067CF4DF91CF911F910F91C4
:1056A000FF90EF90DF90CF90BF90AF900895D0E043
:1056B000DACFDD2389F3802F880F080F000F0093C6
:1056C000A515C093A61560E270E080E090E00E940E
:1056D0001829C601DF91CF911F910F91FF90EF9094
:1056E000DF90CF90BF90AF900C94F32A8F929F924F
:1056F000AF92BF92CF92DF92EF92FF920F931F93E0
:10570000CF93DF93CDB7DEB72C970FB6F894DEBFFB
:105710000FBECDBF982F862F5A017901D02E692F49
:105720000E946828882309F489C0C701002391F1E9
:105730000E9435BBC82E8090721590907315809191
:10574000F804811145C01FEF23E12C1940912D0869
:1057500050912E0860912C08C5010E9475BACC208A
:1057600009F46CC0B6E08B9F500111246AE370E02D
:1057700080E090E00E94182957E0A516B10408F4D3
:1057800044C060E270E080E090E00E941829A81A0E
:10579000B90AF2CF0E9420BDC82E80907215909059
:1057A00073158091F804882371F2FE0133968AE024
:1057B000DF011D928A95E9F78EE695E19A83898348
:1057C00008E215E29E012F5F3F4F46E451E212C00E
:1057D000FE0133968AE0DF011D928A95E9F78EE695
:1057E00095E19A83898308E215E29E012F5F3F4F7E
:1057F00043E451E2B701C4010F94F924B4018EE6E9
:1058000095E10F94A33A1F819FCF40912B08212F40
:1058100030E0A6E0CA9EC00111242E5F3F4F28173A
:1058200039070CF49C0180E8821B8093A5154093F6
:10583000A615C701DD20A9F00E94192A2C960FB6E3
:10584000F894DEBF0FBECDBFDF91CF911F910F91B6
:10585000FF90EF90DF90CF90BF90AF909F908F9090
:1058600008950E94F32AEACFEAE6F5E183AF64AF38
:10587000CA010C94F32A2F923F924F925F926F923B
:105880007F928F929F92AF92BF92CF92DF92EF92D0
:10589000FF920F931F93CF93DF93D62FC72FFC0157
:1058A00080809180A280B380C501B40120E831E5F9
:1058B00041E050E00F943E56C9016DE671E00F944F
:1058C000BB566B017C01C501B40120E13EE040E024
:1058D00050E00F943E56CA01B90128E130E040E0A3
:1058E00050E00F943E56362E272E062F172F8CE3AE
:1058F000482E512C612C712CC501B401A3019201D9
:105900000F943E56B62EA72ECA01B901A3019201EB
:105910000F943E56CB01C114D10479F1AF92BF92DE
:105920007F936F932F923F92FF92EF92DF92CF92ED
:105930008DE195E19F938F93CF93DF930F94914FD8
:105940008DB79EB70E960FB6F8949EBF0FBE8DBF53
:105950008D2F9C2FDF91CF911F910F91FF90EF9092
:10596000DF90CF90BF90AF909F908F907F906F907F
:105970005F904F903F902F900895E114F104C9F08B
:10598000AF92BF927F936F932F923F92FF92EF92CD
:105990008DE095E19F938F93CF93DF930F94914F79
:1059A000EDB7FEB73C960FB6F894FEBF0FBEEDBF45
:1059B000CFCF012BB9F0AF92BF927F936F932F920D
:1059C0003F9281E095E19F938F93CF93DF930F9464
:1059D000914F8DB79EB70A960FB6F8949EBF0FBE33
:1059E0008DBFB6CF892BA9F0AF92BF927F936F93F3
:1059F00089EF94E19F938F93CF93DF930F94914F0F
:105A0000EDB7FEB738960FB6F894FEBF0FBEEDBFE8
:105A10009FCFAF92BF9285EF94E19F938F93CF93E7
:105A2000DF930F94914F0F900F900F900F900F9066
:105A30000F908ECF8F929F92AF92BF92CF92DF92B4
:105A4000EF92FF920F931F93CF93DF931092F50481
:105A50001092F4042FE32093F3041092F2041092B6
:105A6000F1041092F0041092EC041092ED041092E4
:105A7000EE041092EF049C01F90190812F5F3F4FDB
:105A80009032D1F39E34C9F4818190ED980F9A3011
:105A900020F08D3211F08B3281F432969F012F5F0E
:105AA0003F4F808180538A3008F47BC09F012F5F75
:105AB0003F4F8081803209F476C0F0935008E09324
:105AC0004F088F010F5F1F4FC0816AE270E0C8016D
:105AD0000F94415A009731F0FC0131978081803258
:105AE000E1F31182CD3429F0C43519F0C73409F03F
:105AF0004BC0F80180810F5F1F4F8032D1F380537C
:105B00008A3008F041C0C093F30430E020E04AE05E
:105B1000DF011196429FC001439F900D11249C010B
:105B2000205331098081280F311D87FD3A958181ED
:105B300090ED980F9A30C8F13093F2042093F1045D
:105B40008E3261F4329690E04AE0DF0131968C911A
:105B500050ED580F5A3058F19093F004CD01DC010C
:105B600001964C914032D9F3CD3489F52E3131056F
:105B700039F018F52731310519F02C31310539F597
:105B8000B093F504A093F404DF91CF911F910F918E
:105B9000FF90EF90DF90CF90BF90AF909F908F904D
:105BA0000895F9017BCFF90181CFFD01B1CF949F19
:105BB000800D112490ED980FC8CF2537310538F0AE
:105BC00027373105E8F2203A83E03807C9F2D0914F
:105BD0004F0840E050E0BA0110E000E0C12CD12CA9
:105BE0007601C394FD0131968C91882309F47FC01E
:105BF0008132E1F4CD34D1F420323105B9F440934F
:105C0000EC045093ED046093EE047093EF04F09372
:105C1000F504E093F40463E270E0CF010F94415A7D
:105C2000009709F4B1CFFC011082AECF81548A31C4
:105C300008F058C0DF019D91903291F0A0EDA90FBE
:105C4000AA30E8F09E3271F4918190539A30B8F006
:105C50000115110519F48F010150110990E013C0CD
:105C6000FD01E8CF9D3211F09B3291F79181A0EDBB
:105C7000A90FAA3020F09E3259F79281E6CF9E2FCD
:105C80009D1B309759F3A82FB0E04601570104C07F
:105C9000880C991CAA1CBB1C8A95D2F74829592943
:105CA0006A297B29AE52BB4F9C9380818154DF01CE
:105CB0008A3108F497CFDF018191882309F492CFCC
:105CC00090ED980F9A30B8F393ED980F923098F3C7
:105CD0008B3289F3CD010196EC91E03209F082CF4D
:105CE000DC01F8CF0115110501F78D01DECF10930E
:105CF000F5040093F4044093EC045093ED04609396
:105D0000EE047093EF0440CF9B01AC01485F5F4FFE
:105D1000BC016C5F7F4F0C9461260F931F93CF9350
:105D2000DF9300D000D01F921F92CDB7DEB7FC01E9
:105D30008B0183A5811112C081E083A784819581A5
:105D4000A681B781B05889839A83AB83BC83BE0197
:105D50006F5F7F4F81E398E00E94842E1D821E8238
:105D60001F82188620E030E040E05FE36091EE0F94
:105D70007091EF0F8091F00F9091F10F0F94EC560E
:105D800069837A838B839C839E012B5F3F4FAE0197
:105D90004F5F5F4F6AEE7FE086EE9FE00E946126D4
:105DA0001D821E821F82188620E030E040E05FE303
:105DB000F80160857185828593850F94EC5669831F
:105DC0007A838B839C83B8016C5F7F4F9E012B5F2E
:105DD0003F4FAE014F5F5F4FC8010E94612628967A
:105DE0000FB6F894DEBF0FBECDBFDF91CF911F91EC
:105DF0000F9108952F923F924F925F926F927F92F0
:105E00008F929F92AF92BF92CF92DF92EF92FF92CA
:105E10000F931F93CF93DF93CDB7DEB7A2970FB643
:105E2000F894DEBF0FBECDBF8C011B015E834D8396
:105E30004090E60F5090E70F6090E80F7090E90FE8
:105E40008090EA0F9090EB0FA090EC0FB090ED0FC8
:105E5000DB018D919D910D90BC91A02D8F87988B2A
:105E6000A98BBA8B9C01AD01C301B2010F94EB5613
:105E70006B017C01D10114968D919D910D90BC9187
:105E8000A02D8B8B9C8BAD8BBE8B9C01AD01C50176
:105E9000B4010F94EB566F8B788F898F9A8FAD81F9
:105EA000BE818D919D910D90BC91A02D8F8398877F
:105EB000A987BA879C01AD01C301B2010F94EB56CB
:105EC0006B8F7C8F8D8F9E8FAD81BE8114968D914F
:105ED0009D910D90BC91A02D8B879C87AD87BE872F
:105EE0009C01AD01C501B4010F94EB566F8F78A3EF
:105EF00089A39AA3A7019601C701B6010F94605028
:105F00006B017C012F89388D498D5A8DCA01B901E9
:105F10000F9460509B01AC01C701B6010F94EC5681
:105F20004B015C012F85388949895A896F817885B1
:105F300089859A850F94EB562B013C012B893C896E
:105F40004D895E896B857C858D859E850F94EB568A
:105F50006B017C01A3019201C301B2010F94605057
:105F60002B013C01A7019601C701B6010F946050B7
:105F70009B01AC01C301B2010F94EC560F949A59E6
:105F80006B017C012B8D3C8D4D8D5E8DCA01B9015D
:105F90000F9460502B013C012F8D38A149A15AA1CB
:105FA000CA01B9010F9460509B01AC01C301B20159
:105FB0000F94EC569B01AC01C501B4010F944C59F0
:105FC0001816B4F520E030E0A901C701B6010F941E
:105FD0004C5987FF2AC0C701B601905820E030E035
:105FE00040EA50E40F944C59181614F5A1016D8144
:105FF0007E81C8010E94FA2EA2960FB6F894DEBFE9
:106000000FBECDBFDF91CF911F910F91FF90EF9009
:10601000DF90CF90BF90AF909F908F907F906F90C8
:106020005F904F903F902F900895C701B601D6CF53
:1060300020E030E040E050E4C501B4010F944C5939
:10604000181624F4B101C8010E948D2E19821A82FB
:106050001B821C82BE016F5F7F4FC1010E94842E94
:106060002DEC3CEC4CEC5CE3C701B6010F946050A6
:106070009B01AC01F80160817181828193810F9451
:10608000605069837A838B839C83C8010F94C42BEF
:10609000BE016F5F7F4F8D819E810E94842EACCFA9
:1060A0004F925F926F927F929F92AF92BF92CF92E8
:1060B000DF92EF92FF920F931F93CF93DF93CDB7B1
:1060C000DEB768970FB6F894DEBF0FBECDBFFB01F9
:1060D0009080342F390D353008F026C1E180022F31
:1060E0000E0D053008F020C1EE2DF0E0EE54FB4F10
:1060F0004080512C712C612C092C04C0769467943B
:10610000579447940A94D2F740FE0EC110E0F8016C
:10611000EE54FB4F4080512C712C612CC32ED12C9E
:1061200004C076946794579447943A95D2F740FE0A
:10613000FBC0F22E642F5C01660F770B072E000C5C
:10614000880B990B0F9401502B013C01892D94E091
:106150008902F0011124E354FA4EA30192016081F7
:106160007181828193810F94EC566D877E878F8732
:10617000988BF601EE0FFF1FEE0FFF1FE354FA4E50
:10618000A301920160817181828193810F94EB560A
:1061900069837A838B839C836F2D660F770B072E21
:1061A000000C880B990B0F9401502B013C018E2D94
:1061B00094E08902F0011124E755FA4EA3019201FF
:1061C00060817181828193810F94EC56698B7A8B07
:1061D0008B8B9C8B000F111F000F111FF801E755CF
:1061E000FA4EA301920160817181828193810F94A3
:1061F000EB566D837E838F839887F501808591852B
:10620000A285B38589879A87AB87BC878D8B9E8B48
:10621000AF8BB88F45E351E061E070E0CE0141966D
:106220000E9416D645E351E061E070E0CE0105968C
:106230000E9416D64AE351E061E070E0CE010D966F
:106240000E9416D64AE351E061E070E0CE0101966B
:106250000E9416D6C988DA88EB88FC8827E137EBDC
:1062600041ED58EBC701B6010F944C5987FD5CC056
:1062700023E030E04BE953E4C701B6010F94FA4F35
:1062800018160CF451C0CD84DE84EF84F88827E121
:1062900037EB41ED58EBC701B6010F944C5987FD20
:1062A00043C023E030E84DE953E4C701B6010F9441
:1062B000FA4F1816CCF1CD80DE80EF80F88427E10C
:1062C00037EB41ED58EBC701B6010F944C5987FDF0
:1062D0002BC023E030E04BE953E4C701B6010F9433
:1062E000FA4F18160CF1C980DA80EB80FC8027E1A8
:1062F00037EB41ED58EBC701B6010F944C5987FDC0
:1063000013C023E030E84DE953E4C701B6010F9410
:10631000FA4F18164CF0AE014F5F5F4FBE01635F3E
:106320007F4FC5010E94FA2E68960FB6F894DEBF23
:106330000FBECDBFDF91CF911F910F91FF90EF90D6
:10634000DF90CF90BF90AF909F907F906F905F90C5
:106350004F9008958C38910514F08CE890E090935C
:106360006F0880936E080C945BC70E94A72797FD67
:106370000CC00E94A7276F3F71058105910509F0A8
:1063800034F40E94A727862F089580E008958FEFA8
:1063900008958091BB049091BC04892B41F00E9428
:1063A000B53191E0811101C090E0892F089591E00D
:1063B000FCCF0E94A727CB0108950F931F93CF9383
:1063C0008091BB049091BC040097E9F0FC018F011F
:1063D000C1912C2F2F7D81F0C53411F0C536B9F74E
:1063E000F801108270E060E00F94894BF801C083DF
:1063F000CF911F910F91089570E060E0CF911F91B0
:106400000F910D94894B60E070E0CB01F1CF2FEB41
:10641000280F2A3108F047C0E22FF0E08091EC0409
:106420009091ED04A091EE04B091EF0404C0B695F4
:10643000A795979587952A95D2F780FD02C0817020
:106440000895EE52FB4FE081EE2341F180914F0819
:1064500090915008E80FF92FF11D808190ED980F71
:106460009A3030F08E3251F4818180538A3098F422
:10647000F093BC04E093BB0481E008958D3211F0E9
:106480008B3249F4818190ED980F9A3088F38E32E7
:1064900011F48281EACFF0E0E0E0EACF1092BC0490
:1064A0001092BB04E9CF80E008950E940732882350
:1064B00041F081E02091BB043091BC04232B09F40E
:1064C00080E00895CF93DF93EB010E94553288233B
:1064D00019F00E94A727EB01CE01DF91CF9108951B
:1064E000CF92DF92EF92FF926A017B010E945532B8
:1064F000882331F0FF90EF90DF90CF900C94DD3146
:10650000C701B601FF90EF90DF90CF9008954F92B2
:106510005F926F927F928F929F92AF92BF92CF9233
:10652000DF92EF92FF921F93CF93DF9300D01F92E1
:10653000CDB7DEB719821A821B821C82CE0101966A
:106540004C0186EEC82E8FE0D82E91E3E92E98E01C
:10655000F92E2CE4A22E29E0B22E10E088E5810F5E
:106560000E945532F40181934F01882341F00E942B
:10657000DD312B013C0180919B0F882359F0F601FE
:1065800080819181A281B381F70180839183A2836D
:10659000B38314C0812F0E941A22882309F4D0C02B
:1065A000F6012081318142815381C301B2010F94F0
:1065B000EC56F70160837183828393831F5FF4E05D
:1065C000CF0ED11C84E0E80EF11C94E0A90EB11CA2
:1065D000133021F685E40E9455328C83882309F418
:1065E000B9C00E94DD316B017C0183E00E941A2258
:1065F000882371F02091F20F3091F30F4091F40F46
:106600005091F50FC701B6010F94EC566B017C0158
:10661000C0923D08D0923E08E0923F08F0924008B8
:106620008091CB05882359F18091DC1582FF27C02A
:106630008C81882321F18981811103C08A8188237B
:10664000F1F02DEC3CEC4CE45DE36091A30870911B
:10665000A4088091A5089091A6080F94EC569B0180
:10666000AC016091EE0F7091EF0F8091F00F90915F
:10667000F10F0F944C59181614F40F947C3C40E021
:1066800050E0BA0186E40E94703220E030E0A901B7
:106690000F944C59181684F40E94DD3120E030E04C
:1066A00040E752E40F94E6576093740270937502CA
:1066B000809376029093770280919C0F83FD2CC08B
:1066C00080919B0F811128C08091AB07882321F115
:1066D0002091F20F3091F30F4091F40F5091F50F8C
:1066E00060913D0870913E0880913F08909140086C
:1066F0000F94EB562091B8073091B9074091BA0733
:106700005091BB070F94EC566093B8077093B9078C
:106710008093BA079093BB070F900F900F900F9044
:10672000DF91CF911F91FF90EF90DF90CF90BF90BE
:10673000AF909F908F907F906F905F904F90089553
:10674000F5012081318142815381C301B2010F944F
:10675000EB562FCF8091F20F9091F30FA091F40F91
:10676000B091F50F80933D0890933E08A0933F08A9
:10677000B093400855CFCF93DF93EB010E94553281
:10678000882321F0DF91CF910C94D931CE01DF9194
:10679000CF910895CF93DF93C82FD62F0E94553203
:1067A000882321F0DF91CF910C94C9318C2F0E9466
:1067B0000732811101C08D2FDF91CF910895EAE951
:1067C000F8E082EBDF011D928A95E9F70895809148
:1067D000CB05811104C00E94DF330D94203F8091CE
:1067E000DC1582FD0D947C3C089580919A088823E5
:1067F00061F090914B09891308C08091DC1583FFEB
:1068000004C088ED98E00D942B3F80E00895FC01D2
:10681000238121110C94EBD20895CF92DF92EF9255
:10682000FF920F931F93CF9390912402913009F41C
:1068300061C0662351F010929E0410929A04109247
:106840009B0410929C0410929D04C82F0F947E32DA
:10685000C0909A04D0909B04E0909C04F0909D041A
:106860009B01AC012C193D094E095F0969017A01B0
:10687000F7FC40C020919E04C7FD15C04C2F0C2E84
:10688000000C550B4C5F5F4FE22F022E000CFF0BEC
:106890004E175F077CF144EFC42EDD24D394E12C26
:1068A000F12C2C1734F438EEC32E33E0D32EE12C28
:1068B000F12CC60ED71EE81EF91EC0929A04D09283
:1068C0009B04E0929C04F0929D04022F017010E062
:1068D00084E2809FB001819F700D701B112460596C
:1068E0007C4F82E390E00E94847E80919E048F5FC3
:1068F00080939E04CF911F910F91FF90EF90DF90B6
:10690000CF9008950F931F9301E010E020E030E056
:10691000082E04C0000F111F221F331F0A94D2F744
:1069200040910005509101056091020570910305A9
:10693000402B512B622B732B409300055093010584
:10694000609302057093030590912302891303C09D
:1069500081E080939B0F1F910F9108951092300654
:10696000109231061092320610923306ECECF5E0EC
:1069700084E6DF011D928A95E9F708959091E50F6D
:106980009817B1F00E94FADC8091E50F882341F05E
:1069900086EE9FE00E941DDD1092E50F0C94E8F05A
:1069A00081E08093E50F86EE9FE00E944FDCF6CFFA
:1069B00008954F925F926F927F928F929F92AF92C3
:1069C000BF92CF92DF92EF92FF921F93CF93DF930C
:1069D000EC01162F209164083091650840916608FB
:1069E00050916708688179818A819B810F94FA4F61
:1069F000882309F4AEC0B090E50F80E00E94BE3459
:106A0000C880D980EA80FB8020E030E0A901C7017E
:106A1000B6010F944C5918161CF0C12CD12C7601DC
:106A2000C0926408D0926508E0926608F092670808
:106A30002DEB37E346E855EBC701B6010F944C59EF
:106A400087FD0BC02DEB37E346E855E3C701B601E0
:106A50000F94FA4F18160CF078C0A701960160E069
:106A600070E080E89FE30F94E6576093AF05709362
:106A7000B0058093B1059093B20580EF9FEFA9E731
:106A8000B4EC8093B3059093B405A093B505B0938F
:106A9000B605BB2009F45DC04090E60F5090E70FAB
:106AA0006090E80F7090E90F8090EA0F9090EB0FE4
:106AB000A090EC0FB090ED0FC090EE0FD090EF0FC4
:106AC000E090F00FF090F10F81E00E94BE341123AE
:106AD00009F43FC02091E60F3091E70F4091E80F95
:106AE0005091E90FC301B2010F94FA4F81111CC0FC
:106AF0002091EA0F3091EB0F4091EC0F5091ED0F88
:106B0000C501B4010F94FA4F81110EC02091EE0F10
:106B10003091EF0F4091F00F5091F10FC701B60186
:106B20000F94FA4F8823A9F0DF91CF911F91FF9026
:106B3000EF90DF90CF90BF90AF909F908F907F901D
:106B40006F905F904F900C9490F960E070E0CB01F3
:106B50008CCFDF91CF911F91FF90EF90DF90CF907E
:106B6000BF90AF909F908F907F906F905F904F906D
:106B70000895EF92FF920F931F93CF93DF930CEC46
:106B800015E0C5E07801D5E0F7016191719181913F
:106B900091917F0120E030E0A9010F94FA4F81111B
:106BA0000EC0D15089F7C1500C5E1F4FC111EACF02
:106BB000DF91CF911F910F91FF90EF90089581E0A9
:106BC000F7CFEFE6F0E080818260808308958091C6
:106BD000450890914608892B79F480914508909159
:106BE0004608892B49F4209145083091460881E0F8
:106BF000232B19F480E0089581E00895CF92DF926D
:106C0000EF92FF926B017C0183E3C816D104E1048B
:106C1000F10470F082E3C81AD108E108F10862E3D8
:106C200070E080E090E00F944B320E94EAF0ECCFED
:106C3000C701B6010F944B32FF90EF90DF90CF90D9
:106C40000C94EAF080912B0781110AC080916208B0
:106C5000813041F08091DC1582FB882780F908950E
:106C600080E0089581E008955F9A8091BF078E7F4C
:106C70008093BF078A9A8091BF078D7F8093BF075B
:106C80008091080180958170809306018091BF07F3
:106C90008B7F8093BF070C9447229091DC1593FB68
:106CA000882780F993FF06C081E0909142179111E7
:106CB00001C080E0089580912B07811110C0809160
:106CC0006208823061F00E944D36882349F080913D
:106CD000DC1582FB882780F991E08927089581E0FF
:106CE00008950E945B3681110DC01092000510922C
:106CF00001051092020510920305109204058FEF12
:106D00000E94E8250C94DFFCE6E8F9E0108211828D
:106D1000089581E008958F929F92AF92BF92CF9293
:106D2000DF92EF92FF920F93CF93DF931F92CDB735
:106D3000DEB75C017B0149016B01C40ED51EF50174
:106D4000808191810F9418568983002311F0F701F7
:106D50008083BE016F5F7F4FC4010F941F24F50134
:106D600080819181019691838083FFEFEF1AFF0A62
:106D7000EC14FD0421F780E00F90DF91CF910F918B
:106D8000FF90EF90DF90CF90BF90AF909F908F904B
:106D900008959091C00095FFFCCF8093C6000895A0
:106DA000CF93DF93EC018991882319F00E94C936B3
:106DB000FACF8DE00E94C9368AE0DF91CF910C9422
:106DC000C936CF92DF92EF92FF92CF936B017C0195
:106DD000C42F4A3069F4F7FE0BC0F094E094D094CD
:106DE000C094C11CD11CE11CF11C8DE20E94C9366B
:106DF0004C2FC701B601CF91FF90EF90DF90CF905D
:106E00000D94DE3BCF93DF93EC01FE01849121963C
:106E1000882319F00E94C936F8CFDF91CF910895E9
:106E20000F931F93CF938C01C62F8DE592E10E94A3
:106E30000237C8010E9402378AE30E94C93680E304
:106E40008C0F0E94C9368AE0CF911F910F910C944C
:106E5000C93680EE93E10E94023760E080ED93E155
:106E60000E94103760E08BEB93E10E94103761E0E5
:106E700084EB93E10E94103761E089EA93E10E947C
:106E8000103761E089E993E10E94103760E080E902
:106E900093E10E94103761E086E893E10E94103789
:106EA00060E08CE793E10E94103761E085E793E1B1
:106EB0000E94103760E08DE693E10E94103761E098
:106EC0008FE593E10E94103761E081E593E10E9434
:106ED000103760E082E493E10E94103760E084E3C1
:106EE00093E10E94103760E08EE193E10E94103739
:106EF00061E08DE093E10E94103761E08EEF92E156
:106F00000E94103761E087EF92E10E94103760E045
:106F100080EF92E10E94103761E087EE92E10E94DB
:106F2000103761E082ED92E10E94103761E084EC5D
:106F300092E10E94103761E081EB92E10E941037EC
:106F400060E084EA92E10E94103761E08FE992E10B
:106F50000E94103761E082E992E10E94103760E000
:106F60008EE792E10E94103760E08BE692E10E948A
:106F7000103760E08EED95E10E941722682F617056
:106F800082E692E10C9410370E94C93685E29DE0BA
:106F90000C9402370F931F93CF938C01C62F8CE96B
:106FA00099E00E940237C8010E940237CC2331F0D9
:106FB0008AE0CF911F910F910C94C936CF911F9108
:106FC0000F9108950F931F93CF938C01C62F60E00C
:106FD0008CEA99E00E94CA37C8010E940237CC238C
:106FE00031F08AE0CF911F910F910C94C936CF9167
:106FF0001F910F91089561E084EB99E00C94E237C2
:10700000EF92FF920F931F93CF937C018B01C42FBC
:1070100060E08CEA99E00E94CA37C7010E940237FB
:1070200080E20E94C936C8010E940237CC2319F0C1
:107030008C2F0E94C9368AE0CF911F910F91FF904B
:10704000EF900C94C936DF92EF92FF920F931F934B
:10705000CF93DF93D82E7B018A01E9010E94FB3791
:10706000D092490840E0B70183E490E40E940038E0
:107070000115110531F040E0B8018CE390E40E9465
:107080000038209731F040E0BE018CE390E40E948C
:10709000003861E087E390E4DF91CF911F910F9179
:1070A000FF90EF90DF900C94E23761E086EA99E080
:1070B0000C94CA37AF92BF92CF92DF92EF92FF92B9
:1070C0000F931F93CF93DF9381E799E00E940237DC
:1070D00060913006709131068091320690913306AE
:1070E00045E00F945F078EE599E00E940237C0E00B
:1070F000D9E0D15021F080E20E94C936FACF8C2F1E
:107100000F94453CCF5FC53099F78AE00E94C9369D
:107110000CEC15E0C0E080E20E94C9368C2F0F9481
:10712000453C5801D5E080E20E94C936F501C08097
:10713000D180E280F380A7019601C701B6010F94C8
:10714000DE5981112CC020E030E0A901C701B60151
:107150000F944C5987FD03C08BE20E94C93645E06D
:10716000C701B6010F945F07D15084E1A80EB11C8E
:10717000D111D9CF8AE00E94C936CF5F0C5F1F4F73
:10718000C53049F68AE0DF91CF911F910F91FF90B2
:10719000EF90DF90CF90BF90AF900C94C936F12C58
:1071A00080E20E94C936F3948DE3F8E0FF12F9CF34
:1071B000DBCF811107C083E69EE00E9402378AE0A0
:1071C0000C94C93687E69EE0F8CFCF93DF93EB01AE
:1071D0000E940237CE01DF91CF910D944C3CCF93AA
:1071E000C62F0E9402378C2FCF910D94453CCF9231
:1071F000DF92EF92FF926A017B010E94023742E028
:10720000C701B601FF90EF90DF90CF900D945F071C
:10721000CF92DF92EF92FF926A017B010E940237C8
:107220004AE0C701B601FF90EF90DF90CF900C9439
:10723000E1362F923F924F925F926F927F928F92A0
:107240009F92AF92BF92CF92DF92EF92FF920F93F5
:107250001F93CF93DF93CDB7DEB7C654D1090FB6D6
:10726000F894DEBF0FBECDBF70E060E085E40E9401
:10727000BB33182F8F3F09F483C08823E9F08BE9D3
:1072800096E1CA5BDF4F0FB6F894DEBF0FBECDBFED
:10729000DF91CF911F910F91FF90EF90DF90CF90F2
:1072A000BF90AF909F908F907F906F905F904F9026
:1072B0003F902F900C94023724EB30E03A832983DF
:1072C00083E50E945532882321F00E94D9319A83A8
:1072D000898365E070E083E40E94BB338AA760E0A5
:1072E00085E50E94CA3325968FAF259760E08EE82A
:1072F00096E10E9499B3A981BA81BD01BB0F880BA9
:10730000990B0F9401506D837E838F8327969FAFD7
:1073100027970F947E32688B798B8A8B9B8B1F3FCC
:1073200009F045C420E030E04CE053E46D817E81FB
:107330008F8127969FAD27970F944C5918160CF004
:10734000AAC183E696E10E940237CA5BDF4F0FB6FF
:10735000F894DEBF0FBECDBFDF91CF911F910F918B
:10736000FF90EF90DF90CF90BF90AF909F908F9065
:107370007F906F905F904F903F902F900D941B40A7
:1073800046E450E05A8349839BCF1FAEAFC1249699
:10739000EEADFFAD2497808383C2FBEE4F2E512CC0
:1073A000612C712C04C384E190E0A0E0B0E08C8BF0
:1073B0009D8BAE8BBF8BE4E14E2E512C612C712C3A
:1073C00004C34C8A5D8A6E8A7F8AFFC22496EEAD22
:1073D000FFAD24978083D4C389819A81AB81BC811E
:1073E00029A93AA94BA95CA9821B930BA40BB50B45
:1073F000B7FD59C08FAD0F9403088AE00E94C936CB
:1074000089819A81AB81BC818053984FAF4FBF4F28
:1074100089AB9AABABABBCAB9DA9911177C02EA940
:107420003FA948AD59ADB101802F26969FAD269753
:107430000F944C5918160CF053C020E030E040E097
:1074400050E4B101802F26969FAD26970F94EC56FD
:107450006EAB7FAB88AF99AF2CA53DA54EA55FA5C0
:1074600089819A81AB81BC81280F391F4A1F5B1F1C
:107470002AAF3BAF4CAF5DAF20E030E040EC50E4D2
:107480006D817E818F8127969FAD27970F94EB5654
:107490009101402F26965FAD26970F94FA4F881FD3
:1074A0008827881F8DAB88899989AA89BB89C816C6
:1074B000D906EA06FB0610F4D701C60129813A81F4
:1074C0004B815C81281B390B4A0B5B0BDA01C9012C
:1074D00081389F44A241B105A8F18FEA95E10EC21F
:1074E00089819A81AB81BC812AAD3BAD4CAD5DAD4C
:1074F000821B930BA40BB50B4CE056E36BE176E3D8
:10750000B7FDD1CF812F0E9458D6CDCF20E030E0FB
:1075100040EF51E46D817E818F8127969FAD279743
:107520000F94EB569B01AC01B101802F26969FADC5
:1075300026970F94FA4F87FFB6CF48EB56E368ECD7
:1075400076E3E0CF4AA55BA5888D998D481759074A
:107550000CF09EC003970CF49BC082E595E10E945D
:1075600002371F3F09F076C0A2E4B5E1BA83A983D0
:1075700081E395E10E94023789819A810E94023756
:10758000488559856A857B858EE495E10E94F738A8
:107590008AE00E94C93681E395E10E940237898121
:1075A0009A810E94023749A15AA16BA17CA18AE469
:1075B00095E10E94F7388AE00E94C93681E395E19F
:1075C0000E94023789819A810E940237B501A40185
:1075D00086E495E10E94F7388AE00E94C936259634
:1075E000FFAD2597FF2391F12CEA35EC47E25EE3EE
:1075F00069A17AA18BA19CA10F9460506B017C01C1
:107600002CEA35EC47E25EE3C501B4010F94E6577E
:10761000288539854A855B851F3F09F520937108C8
:10762000309372084093730850937408C0927508A1
:10763000D0927608E0927708F09278086093790803
:1076400070937A0880937B0890937C0881E0809304
:107650005D027BCEE1E8FFE3FA83E98389CF2093E3
:107660002115309322154093231550932415C09271
:107670002515D0922615E0922715F09228156093D3
:10768000291570932A1580932B1590932C15DECF16
:107690000E94A5B780C08FE496E10E9402370E9445
:1076A0004BD58FE78093700824EB30E0A8EEB3E071
:1076B0000F9492566CA77DA78EA79FA7288939891A
:1076C0004A895B89260F371F481F591F2AAF3BAFD6
:1076D0004CAF5DAF10925D0281E080936C0232E0AE
:1076E000310F3EAF323008F450CE1FAFC888D98872
:1076F000EA88FB88C9AADAAAEBAAFCAA812C912CF9
:10770000540189A29AA2ABA2BCA288869986AA86B5
:10771000BB868FE790E0A0E0B0E08C8B9D8BAE8BBA
:10772000BF8B1C8690E49A8FACE1AB8FB6E4BC8F24
:107730001D8E1E8E1F8E18A23FE7432E512C612CEA
:10774000712C1DAA8EAA9FAAA8AEB9AE1EA21FA216
:1077500018A619A6E1E0EDA3198E188E212C312C64
:1077600000E026961FAE2697F5E11F02C001112406
:107770009C01285E3A4E22963FAF2EAF2297285F9B
:107780003F4F24963FAF2EAF24974AA5042E000CFE
:10779000550B5BA74AA780916C02882309F4B0C0FF
:1077A0000F947E3269837A838B839C8350914D063C
:1077B00058AB552309F48BC00E94FED560916C082C
:1077C00070916D081F3F39F02296AEADBFAD229784
:1077D00014966D917C91072E000C880B990B0F94D9
:1077E00001501B01082F26969FAF26972D8D3E8DA9
:1077F0004F8D58A126969FAD26970F944C59181679
:107800003CF42D8E3E8E0F8F2696BFAD2697B8A3E3
:107810002C853A8D4B8D5C8DB101802F26969FADC6
:1078200026970F94FA4F87FF07C02C863A8E0B8F4E
:107830002696EFAD2697EC8FFDA19101402F26965D
:107840005FAD26976D817E818F8127969FAD2797AB
:10785000FF2309F45AC00F94FA4F87FF38C04981BB
:107860005A816B817C814C195D096E097F09DB01AE
:10787000CA0188589341A109B109B7FD28C08C8974
:107880009D89AE89BF8984199509A609B709B5955F
:10789000A795979587951F3F09F079CD809370083C
:1078A0004EA35FA368A779A7FD81FD8F2E812E8F40
:1078B0003F813F8F27964FAD279748A389819A81B3
:1078C000AB81BC81888B998BAA8BBB8B1DA220E0DE
:1078D00030E040EF51E46D817E818F8127969FAD2E
:1078E00027970F94EC569101402F26965FAD26976F
:1078F0000F94FA4F87FF70CD8DEC95E10E9402370F
:1079000010926C020E944BD5A1CE0F944C591816C0
:10791000F4F689819A81AB81BC81288939894A89A9
:107920005B89821B930BA40BB50BAC01BD014858BE
:1079300053416109710977FDCACF488D598D452B97
:1079400009F40DC1CEA0DFA0E8A4F9A4C80ED91E89
:10795000EA1EFB1E2EA13FA148A559A5281B390BE5
:107960004A0B5B0BC301B2010F942E56A70196017F
:107970000F9460564C885D886E887F88420E531E37
:10798000641E751E54E145165104610471040CF423
:107990000ACD8CEE48165104610471040CF0FDCC44
:1079A00090E849165104610471040CF40ACD4C8A24
:1079B0005D8A6E8A7F8A2EEF30E040E050E0241925
:1079C00035094609570929013A014C895D896E89B3
:1079D0007F8987E496E10E940839B301A20182E41D
:1079E00096E10E9408394C855A8D6B8D7C8D8BE316
:1079F00096E10E94F7384D8D5E8D6F8D78A184E3FE
:107A000096E10E94F738A88DB98D13970CF4A7C0A2
:107A1000C301B2010F94015020E030E040E850E48F
:107A20000F9460504B015C012C853A8D4B8D5C8D21
:107A30006D8D7E8D8F8D98A10F94EB562BED3FE0D1
:107A400049E450E40F94605020E030E040E05FE310
:107A50000F9460509B01AC01C501B4010F94E6572F
:107A60006C877D878E879F87C701B6010F94015071
:107A70002FE632E143E85AE30F9460506B017C013A
:107A80001E3F59F02AE939E949E15FE3812C912C45
:107A9000A12C6EE3B62E1F3F59F42DEC3CEC4CE4C8
:107AA0005EE37BEA872E7AEA972EA92C7EE3B72E37
:107AB0006C857D858E859F850F946050688779875A
:107AC0008A879B879B01AC010F94EC56A701960116
:107AD0000F94E65769A37AA38BA39CA328853985C5
:107AE0004A855B85C701B6010F946050A5019401DA
:107AF0000F9460504B015C014C855D856E857F85E0
:107B00008EE296E10E94F738B701A60188E296E17D
:107B10000E94F7388AE00E94C936BEAD89E196E13D
:107B2000B23010F08AE096E10E940237488559850C
:107B30006A857B8584E096E10E94F73849A15AA1C5
:107B40006BA17CA18EEF95E10E94F738B501A401ED
:107B500088EF95E10E94F7388AE00E94C9368C8947
:107B60009D89AE89BF89840D951DA61DB71DB5954C
:107B7000A795979587951F3F09F028CC80937008AB
:107B8000288D398D2F5F3F4F398F288F3D813C875E
:107B90004E814A8F5F815B8F27968FAD27978C8FA1
:107BA000C980DA80EB80FC8098A99DA390CEE12E5D
:107BB000012E000CFF08F70183E0EE0FFF1F8A95EE
:107BC000E1F7EC59FD4F668177816F507109072EFF
:107BD000000C880B990B0F9401509B01AC016D8137
:107BE0007E818F8127969FAD27970F944C59181649
:107BF0000CF4A7CB8FE496E10E9402370E944BD58C
:107C000085E18E9DF0018F9DF00D1124E85EFA4E06
:107C10008FE7808722E330E049CDCF93DF93EB01FC
:107C20000E940237CE01DF91CF910D94D6252F927D
:107C30003F924F925F926F927F928F929F92AF92FC
:107C4000BF92CF92DF92EF92FF920F931F93CF9349
:107C5000DF93CDB7DEB7C058D1090FB6F894DEBFB9
:107C60000FBECDBF80EB9CE00E9402370F943D40D9
:107C700081118FC084E50E945532882329F00E942B
:107C8000D93181110E9401D580E090E0A0E8BFE3E6
:107C900089839A83AB83BC838D839E83AF83B887AC
:107CA0008DEC9CECACE4BEE389879A87AB87BC87FC
:107CB00080E090E0A0E2B1E48D879E87AF87B88B2B
:107CC0008CE390E09A8B898B8DEC90E09C8B8B8B76
:107CD0008DEC9CECACECBEE38D8B9E8BAF8BB88FA8
:107CE00080E090E0A0EEBFE3898F9A8FAB8FBC8FCE
:107CF0001BA61CA64AE959E969E97EE38FE40E94C4
:107D000070326D8F7E8F8F8F98A360E083E40E9426
:107D1000CA3389A360E08BE40E94CA338AA389E452
:107D20000E94553210E0F12CE12C8823C1F00E9412
:107D3000B53190E01816190614F481E090E011E0D6
:107D4000180F212F2150330BC90126E0289FF00185
:107D5000299FF00D1124EB5FF74FE280F38082E45E
:107D60000E945532882319F00E94D9317C01E11418
:107D7000F10459F1C70188978536910520F16CE827
:107D800070E082E89CE00E940D3E8DE79CE00E943E
:107D90000237C058DF4F0FB6F894DEBF0FBECDBF1D
:107DA000DF91CF911F910F91FF90EF90DF90CF90D7
:107DB000BF90AF909F908F907F906F905F904F900B
:107DC0003F902F900895FA8AE98A8CE40E945532F8
:107DD0008823E1F00E94DD316B017C01C986DA86DF
:107DE000EB86FC8620E030E0A9010F944C5987FD1A
:107DF0000AC020E030E040E050E4C701B6010F9433
:107E0000FA4F18161CF485E59CE0C1CF81E50E946D
:107E10000732882331F18091BB049091BC04892BF7
:107E2000E9F00E94DD316B017C01CD82DE82EF82C0
:107E3000F8862DEC3CEC4CE45DE30F944C5987FD47
:107E40000AC020E030E040E751E4C701B6010F94DA
:107E5000FA4F181634F484E29CE099CF89EF9BE046
:107E600096CF83E50E9455328823E9F00E94DD31E8
:107E70006B017C01CD8ADE8AEF8AF88E2DEC3CEC1A
:107E80004CEC5DE30F944C5987FD0AC020E030E0D4
:107E900040E050E4C701B6010F94FA4F18161CF4E5
:107EA00082ED9BE074CF80E50E940732882341F089
:107EB0008091BB049091BC04892B29F58FEF8BA78F
:107EC00086E40E945532882309F43DC00E94DD31CA
:107ED0006B017C01C98EDA8EEB8EFC8E20E030E0E7
:107EE00040E85FE30F944C5987FD0AC020E030E082
:107EF00040E850E4C701B6010F94FA4F18161CF57C
:107F000081E89BE044CF8BA58F5F8BA70E94DD317A
:107F10006B017C01CD86DE86EF86F88A20E030E0BA
:107F2000A9010F944C5987FD0BC020E030E048ECCC
:107F300051E4C701B6010F94FA4F18160CF0C0CFE8
:107F40008AEA9BE024CFC98CDA8CEB8CFC8C8D8880
:107F50009E88AF88B88CA7019601C701B6010F941F
:107F600060509B01AC0160E070E084E490E40F9409
:107F7000E65729813A814B815C810F9460502B0137
:107F80003C01A5019401C501B4010F946050A70103
:107F900096010F9460502CEE31E548EB5DE30F94B1
:107FA000E6579B01AC01C301B2010F946050698395
:107FB0007A838B839C83112309F1412F4150550B08
:107FC00026E0249FF001259FF00D1124EB5FF74F71
:107FD0000081118188E40E945532882319F00E94A3
:107FE000D9318C010115110571F0C801855A91092B
:107FF0008838910530F083E59BE0C9CE10E000E0C1
:10800000E9CF1C8B0B8B85E50E9407328823C9F0D2
:108010000F947E32611571058105910511F00F9461
:10802000804B8091BB049091BC04892BC9F00E94C5
:10803000DD316093B7047093B8048093B9049093D2
:10804000BA046AE170E082E50E94BB33E5969FAF17
:108050008EAFE5971816190644F08FE19BE097CE96
:1080600060E070E088E492E4E4CF89E50E94553254
:10807000882309F40AC10E94DD3120915009309112
:10808000510940915209509153090F94EB564B01FD
:108090005C0188E50E945532882309F4FFC00E94E4
:1080A000DD3120914C0930914D0940914E0950919C
:1080B0004F090F94EB566B017C01CBA2DCA2EDA221
:1080C000FEA28FA298A6A9A6BAA627E137EB41ED9A
:1080D00058EBC501B4010F944C5987FDE8C023E06B
:1080E00030E04BE953E4C501B4010F94FA4F181680
:1080F0000CF4DDC027E137EB41ED58EBC701B601C9
:108100000F944C5987FDD3C023E030E84DE953E488
:10811000C701B6010F94FA4F18160CF4C8C084E4D6
:108120000E94073211E081270E94BE3480E090E077
:10813000A0EAB0E48DA79EA7AFA7B8ABCE018D96FD
:108140000F94692B50918108EC965FAFEC971092D9
:1081500081080E940CC582EA9AE00E940237898950
:108160009A894A970CF0A6C063E68FE79AE00E94CE
:1081700099B30F94B7328B899C890E947CDC41E0D3
:1081800061E080E00F94FB09882309F4A6C00F94F6
:108190001B400F94B7321092F20F1092F30F10920F
:1081A000F40F1092F50F82EF9FE00E9430ED1BA5B7
:1081B000112309F4F5C020E030E040E751E460917C
:1081C000CD0F7091CE0F8091CF0F9091D00F0F9463
:1081D000E65721966CAF7DAF8EAF9FAF21971F3FC3
:1081E00009F0F9C481E08093FD0463E687ED9AE02D
:1081F0000E9499B368E873E182E090E00E94847E77
:1082000080E1E6EEFFE0A1E3B8E001900D928A95EF
:10821000E1F7CE0101960F94C42BC12CD12C76012D
:1082200080915C0982FDB1C068E873E182E090E072
:108230000E94847E20E030E040E85EE360913D08EB
:1082400070913E0880913F08909140080F94EC5641
:1082500060933D0870933E0880933F0890934008D8
:1082600020E030E040E85EE3C701B6010F94EC5631
:108270006B017C0120E030E84BE354E40F944C594F
:1082800087FD73C01092FD0428C08090EA0F909083
:10829000EB0FA090EC0FB090ED0FFBCEC090E60F6F
:1082A000D090E70FE090E80FF090E90F06CF85EF50
:1082B0009AE06DCD63E682E99AE00E9499B30F944B
:1082C000B7321093FD0489899A890E94AA3161E02E
:1082D00081E00F947608811147CF6FEF89EE9AE025
:1082E0000E9499B38CA5811112C081E08CA78D8169
:1082F0009E81AF81B885B0588DA79EA7AFA7B8ABB8
:10830000BE01635D7F4F81E398E00E94842E80E090
:1083100090E0A0EAB0E48093390890933A08A093E3
:108320003B08B0933C081DA61EA61FA618AABE01B6
:10833000635D7F4F81E398E00E94842EEC965FADF1
:10834000EC97509381080E940CC51092FD048AA1FD
:1083500081111FCD10926F0810926E080E945BC7AA
:1083600090E080E00E947CDC14CDCE01CD960E948E
:10837000D8F780E1E6EEFFE0A1E3B8E001900D92CE
:108380008A95E1F70E94FADC4BCF0E9464BA63E65B
:108390008AEC9AE00E9499B30F94B7321092FD04D0
:1083A000E2EBF4E085E0DF011D928A95E9F780E1D8
:1083B000E6EEFFE0A1E3B8E001900D928A95E1F7C7
:1083C00089859A85AB85BC858093390890933A0856
:1083D000A0933B08B0933C081DA61EA61FA618AA92
:1083E000BE01635D7F4F81E398E00E94842EBE0151
:1083F000635E7F4F81E398E00E94842E81E080934A
:10840000FD0489A1882309F43CC42091E60F309132
:10841000E70F4091E80F5091E90FAC962CAF3DAFBC
:108420004EAF5FAFAC978091EA0F9091EB0FA091A8
:10843000EC0FB091ED0FE0968CAF9DAFAEAFBFAF3C
:10844000E097ADEBB5E1A196BFAFAEAFA197312CF0
:10845000212CBFEF6C96BFAF6C97EFEFA496EFAFF8
:10846000A497FFEFE396FFAFE3972FE4EA962FAFD1
:10847000EA9733ECEB963FAFEB9707E481E090E0AF
:10848000A0E0B0E0022C04C0880F991FAA1FBB1FF8
:108490000A94D2F7C458DF4F88839983AA83BB8399
:1084A000CC57D040A2EBB4E0E296BFAFAEAFE297BC
:1084B000E9EAF5E1A396FFAFEEAFA39710E0C0584D
:1084C000DF4F2882C058D040E296AEADBFADE297F4
:1084D0008D91E296BFAFAEAFE29790E0B0E0A0E042
:1084E000C458DF4F288139814A815B81CC57D04005
:1084F00082239323A423B523892B8A2B8B2B09F06A
:10850000E5C0A196AEADBFADA197CD90DD90ED9049
:10851000FC90A396AEADBFADA3972D913D914D912B
:108520005C91A8962CAF3DAF4EAF5FAFA897A70167
:108530009601AC966CAD7DAD8EAD9FADAC970F94B2
:10854000EB562B013C01A8962CAD3DAD4EAD5FAD79
:10855000A897E0966CAD7DAD8EAD9FADE0970F9482
:10856000EB564B015C01A3019201C301B2010F94D0
:1085700060502B013C01A5019401C501B4010F9489
:1085800060509B01AC01C301B2010F94EC560F94F3
:108590009A594B015C01A70196016BA17CA18DA1A9
:1085A0009EA10F94EB566B017C01A8962CAD3DADBE
:1085B0004EAD5FADA8976FA178A589A59AA50F9438
:1085C000EB562B013C01A7019601C701B6010F94A0
:1085D00060506B017C01A3019201C301B2010F94B1
:1085E00060509B01AC01C701B6010F94EC560F948B
:1085F0009A5920E030E040E751E40F94E657A50196
:1086000094010F94EC566B017C018090B70490901C
:10861000B804A090B904B090BA0420E030E040E87B
:108620005FE3C501B4010F944C591816F4F4C50169
:10863000B4010F9458584B015C0160E070E0CB012D
:10864000181419041A041B0434F40F94314BA501B7
:1086500094010F9460560F9401509B01AC01B60138
:10866000C7010F94EC566B017C01E3962FADE397A5
:10867000EA963FADEA97EB964FADEB97502FB601D8
:10868000C7010F94FA4F87FF21C06C961FAF6C97FC
:10869000C058DF4FB881C058D040A496BFAFA49750
:1086A000E696CFAEE697E796DFAEE797E896EFAEB1
:1086B000E897E996FFAEE997E396CFAEE397EA969F
:1086C000DFAEEA97EB96EFAEEB970F2D1F5FA39609
:1086D000EEADFFADA3973496A396FFAFEEAFA39791
:1086E000153009F0F1CEFFEF2F1A3F0AA1962EADFB
:1086F0003FADA1972C5F3F4FA1963FAF2EAFA19703
:1087000035E02316310409F0B9CE6C964FAD6C9765
:10871000E42FF0E0EE54FB4F208181E090E0A0E0F8
:10872000B0E0A4960FACA49704C0880F991FAA1FAD
:10873000BB1F0A94D2F7822B8083A4965FADA497C7
:1087400062965FAF629763964FAF6397E6968FAD81
:10875000E697E7969FADE797E896AFADE897E9967D
:10876000BFADE99767968CAF9DAFAEAFBFAF6797D0
:108770005F3F09F414C24F3F09F411C284E048027C
:10878000F0011124E755FA4E1081018132802380D7
:1087900027E137EB41ED58EB612F702F832D922DA0
:1087A0000F944C5987FDFFC123E030E04BE953E4BF
:1087B000612F702F832D922D0F94FA4F18160CF401
:1087C000F2C1A4969FADA497A4E09A02F0011124EF
:1087D000E354FA4EC080D180E280F38027E137EB8A
:1087E00041ED58EBB601C7010F944C5987FDDBC131
:1087F00023E030E84DE953E4B601C7010F94FA4F86
:1088000018160CF4D0C120E030E040EA50E4B60184
:10881000C7010F94EC56A0966FAFA097A2967FAFBA
:10882000A297A5968FAFA597A9969FAFA997CB01C1
:10883000A596AFADA597A996BFADA99721968CAF88
:108840009DAFAEAFBFAF2197812F902FA32DB22D3B
:1088500025968CAF9DAFAEAFBFAF2597A496BFADA9
:10886000A497B11150C26C96EFAD6C97E11118C28C
:1088700020E030E040EA50E4612F702F832D922DEC
:108880000F94EC56A4966FAFA497AD967FAFAD97BB
:10889000E1968FAFE197E3969FAFE3976C96FFADBC
:1088A0006C97FF2309F4F1C26C963FAD6C97A096CC
:1088B000CFAEA097A296DFAEA297A596EFAEA597F2
:1088C000A996FFAEA99734300CF014C222ED822E87
:1088D00023E5922E2BE7A22E21E4B22E21964CAC5A
:1088E0005DAC6EAC7FAC219725962CAD3DAD4EAD09
:1088F0005FAD25976F962CAF3DAF4EAF5FAF6F97D3
:10890000A3019201B601C7010F94EB562D966CAFEF
:108910007DAF8EAF9FAF2D976F962CAD3DAD4EAD19
:108920005FAD6F97612F702F832D922D0F94EB56B3
:1089300061966CAF7DAF8EAF9FAF6197A30192013F
:108940006091E60F7091E70F8091E80F9091E90F29
:108950000F94EB562B013C016F962CAD3DAD4EAD07
:108960005FAD6F976091EA0F7091EB0F8091EC0F04
:108970009091ED0F0F94EB566F966CAF7DAF8EAF6D
:108980009FAF6F97A0968FADA097A2969FADA2972D
:10899000A596AFADA597A996BFADA9978DA79EA7A0
:1089A000AFA7B8ABA4968FADA497AD969FADAD978A
:1089B000E196AFADE197E396BFADE39789AB9AAB94
:1089C000ABABBCABC984DA84EB84FC84CDAADEAA51
:1089D000EFAAF8AE2DEC3CEC4CEC5CE3C501B40125
:1089E0000F94605029813A814B815C810F946050D3
:1089F0002091F20F3091F30F4091F40F5091F50F49
:108A00000F94EC5669AF7AAF8BAF9CAFA301920184
:108A1000C301B2010F9460502B013C016F962CAD45
:108A20003DAD4EAD5FAD6F97CA01B9010F94605077
:108A30009B01AC01C301B2010F94EC5620E030E081
:108A400040E050E40F944C591816ACF420E030E0AC
:108A500040E05FE3C701B6010F94EC5629966CAF76
:108A60007DAF8EAF9FAF2997BE01635C7F4FCE0174
:108A700001960E948D2E89859A85AB85BC852996A5
:108A80008CAF9DAFAEAFBFAF29976B961CAE1DAE3E
:108A90001EAE1FAE6B97BE01695A7F4FCE01CD96B9
:108AA0000E94842ECE0101960F94C42BA090C50F76
:108AB000B090C60FC090C70FD090C80FE090C10F04
:108AC000F090C20F0091C30F1091C40F9701A8013D
:108AD000B501C6010F944C59181614F075018601A2
:108AE0008090740290907502A0907602B090770208
:108AF0002DEC3CEC4CEC5DE3B701C8010F946050E9
:108B0000609374027093750280937602909377025B
:108B100040E0BE01675B7F4FCE018D960F947833A6
:108B200080E1E6EEFFE0A1E3B8E001900D928A95C6
:108B3000E1F78092740290927502A0927602B09250
:108B400077020E9496278111C8CB20E04FEFBE012B
:108B50006F5A7F4FCE0101960E94503020E041E0D5
:108B6000BE016F5A7F4FCE0101960E9450302FEF09
:108B700040E0BE016F5A7F4FCE0101960E945030F7
:108B800021E040E0BE016F5A7F4FCE0101960E9466
:108B900050300E94FADC0E94962781119ECB809172
:108BA000F60F8093F70FE5964EAD5FADE597415018
:108BB0005109E5965FAF4EAFE597452B09F48DCB94
:108BC00062968FAD629787FD88CB63968FAD639772
:108BD00087FF17CC82CB63E687EB9AE00E9499B3BC
:108BE0000F94B73280E1E6EEFFE0A1E3B8E0019038
:108BF0000D928A95E1F72D853E854F8558896091C4
:108C00003D0870913E0880913F08909140080F9474
:108C1000EC5660933D0870933E0880933F08909314
:108C20004008CE01CD960E94D8F72D853E854F8510
:108C3000588960913D0870913E0880913F0890915D
:108C400040080F94EB5660933D0870933E08809364
:108C50003F08909340088CA58111A2CB81E08CA79E
:108C60008D819E81AF81B885B0588DA79EA7AFA793
:108C7000B8ABBE01635D7F4F81E398E00E94842E14
:108C80008FCB2BA13CA14DA15EA1AC962CAF3DAFEB
:108C90004EAF5FAFAC978FA198A5A9A5BAA5CBCBD6
:108CA000C601D70121968CAF9DAFAEAFBFAF219764
:108CB00020E030E040EA50E4612F702F832D922DA8
:108CC0000F94EB5625966CAF7DAF8EAF9FAF259777
:108CD0006C962FAD6C9724300CF4CACDA4961FAFC0
:108CE000A497AD960FAFAD97E1963FAEE197E396AF
:108CF0002FAEE39792ED892E93E5992E9BEFA92E47
:108D000090E4B92EEBCDA4964FADA49744300CF46B
:108D10006EC06C965FAD6C975430BCF120E030E0D3
:108D200040EA50E4B601C7010F94EB5621966CAFB0
:108D30007DAF8EAF9FAF219720E030E040EA50E456
:108D4000612F702F832D922D0F94EB56A4966FAF49
:108D5000A497AD967FAFAD97E1968FAFE197E3967D
:108D60009FAFE3976C969FAD6C97A096CFAEA09700
:108D7000A296DFAEA297A596EFAEA597A996FFAEF5
:108D8000A99794300CF0B6CFA1CDC601D70121969A
:108D90008CAF9DAFAEAFBFAF219720E030E040EA8F
:108DA00050E4612F702F832D922D0F94EC56259651
:108DB0006CAF7DAF8EAF9FAF25976C968FAD6C97E4
:108DC0008111BACF20E030E040EA50E4B601C7019B
:108DD0000F94EB56A0966FAFA097A2967FAFA29785
:108DE000A5968FAFA597A9969FAFA99777CF6C96B9
:108DF000AFAD6C97A1112BC020E030E040E251E410
:108E0000A0966FADA097A2967FADA297A5968FADC5
:108E1000A597A9969FADA9970F94EB56A0966FAF13
:108E2000A097A2967FAFA297A5968FAFA597A99678
:108E30009FAFA997A4961FAFA497AD960FAFAD971C
:108E4000E1963FAEE197E3962FAEE3973FCD6C9668
:108E5000BFAD6C97B43034F120E030E040E251E433
:108E6000A0966FADA097A2967FADA297A5968FAD65
:108E7000A597A9969FADA9970F94EB5621966CAF35
:108E80007DAF8EAF9FAF2197D5CFA096CFAEA097E5
:108E9000A296DFAEA297A596EFAEA597A996FFAED4
:108EA000A99728CFA4961FAFA497AD960FAFAD9703
:108EB000E1963FAEE197E3962FAEE39782ED882EE1
:108EC00083E5982E8BEFA82E81E4B82E07CD87E599
:108ED00099E00C940237CF92DF92EF92FF920F93BA
:108EE0001F93CF93DF9388E50E940732D82E89E441
:108EF0000E940732C82E8823D1F10E94D931D82F81
:108F000089E50E940732182F8AE40E940732082F51
:108F1000882309F455C00E94D931C82F8AE50E94E0
:108F20000732E82EF12C811104C081E50E9407323E
:108F3000F82EC11001C000E0802F90E0D11001C0D8
:108F400010E0810F911D019721F4E11062C0F11032
:108F500060C00E94674783E49EE0DF91CF911F913C
:108F60000F91FF90EF90DF90CF900C940237D110CB
:108F700002C0DFEFC5CF0E94DD3120914C09309156
:108F80004D0940914E0950914F090F94EB5620E046
:108F900030E040EF51E40F94EB5620E030E040EF3A
:108FA00051E40F94EC5629E838E848E85CE30F9464
:108FB00060500F945858D62F653008F4A1CFD9CF00
:108FC000111102C0CFEFAACF0E94DD3120915009CC
:108FD0003091510940915209509153090F94EB5629
:108FE00020E030E040EF51E40F94EB5620E030E019
:108FF00040EF51E40F94EC5629E838E848E85CE388
:109000000F9460500F945858C62F653008F486CFDF
:10901000D9CFD7FD02C0C7FF05C00E9467478AE2CB
:109020009EE09BCF0E94DD319B01AC010D2FDD0F37
:10903000110BAC2FCC0FBB0B60E070E0CB01FF201D
:1090400091F065E0609FF001619FF00D1124EA0F3F
:10905000FB1FEE0FFF1FEE0FFF1FE453FA4F60815F
:10906000718182819381E5E0E09FE001E19FD00D75
:109070001124CA0FDB1FCC0FDD1FCC0FDD1FC45323
:10908000DA4F0F94EC56688379838A839B83DF9150
:10909000CF911F910F91FF90EF90DF90CF900895A7
:1090A00081E599E00C940237CF9384E50E94553214
:1090B000C0E08823D9F00E94B531C82F1816B4F447
:1090C0000E9450488DE40E94C9368091F10490912D
:1090D000F2040F944C3C6C2FCC0F770B8BE29FE08B
:1090E0000E940D3E8AE00E94C936CFEF8C2FCF91AF
:1090F00008954F925F926F927F928F929F92AF925C
:10910000BF92CF92DF92EF92FF92CF93DF93CDB7D2
:10911000DEB72C970FB6F894DEBF0FBECDBF4090E0
:109120004C0950904D0960904E0970904F09209164
:10913000390230913A0240913B0250913C02C30106
:10914000B2010F94EC5669837A838B839C83809061
:10915000500990905109A0905209B0905309209164
:109160003D0230913E0240913F0250914002C501C4
:10917000B4010F94EC566D837E838F839887C090E3
:109180005409D0905509E0905609F0905709209164
:109190004102309142024091430250914402C70182
:1091A000B6010F94EC5669877A878B879C8720914C
:1091B0004502309146024091470250914802C30156
:1091C000B2010F94EC562B013C01209149023091E1
:1091D0004A0240914B0250914C02C501B4010F94D8
:1091E000EC564B015C0120914D0230914E024091B2
:1091F0004F0250915002C701B6010F94EC566B011B
:109200007C010E9450488CE79EE00E94023783E573
:109210000E940732882321F00E94C93180933702CF
:1092200080913702811151C083E69EE00E9402378F
:1092300084E79EE00E94023749815A816B817C81DC
:109240008EED9BE20E94F7384D815E816F817885BB
:1092500081EF90E40E94F73849855A856B857C85BB
:109260008EEE90E40E94F73882E79EE00E9402377B
:109270008AE69EE00E940237B301A2018EED9BE2D6
:109280000E94F738B501A40181EF90E40E94F738FD
:10929000B701A6018EEE90E40E94F7388AE02C9682
:1092A0000FB6F894DEBF0FBECDBFDF91CF91FF9018
:1092B000EF90DF90CF90BF90AF909F908F907F9076
:1092C0006F905F904F900C94C93687E69EE0AECFCA
:1092D0002F923F924F925F926F927F928F929F92C6
:1092E000AF92BF92CF92DF92EF92FF920F931F93B4
:1092F000CF93DF93CDB7DEB76A970FB6F894DEBF92
:109300000FBECDBF83E50E940732182F3090E50FC6
:10931000882319F00E94C931382E4090E60F5090F2
:10932000E70F6090E80F7090E90F8091EA0F90913D
:10933000EB0FA091EC0FB091ED0F8B8B9C8BAD8B55
:10934000BE8B8091EE0F9091EF0FA091F00FB09136
:10935000F10F8F8B988FA98FBA8F112329F03110BD
:1093600003C080E00E94BE3486E50E940732888BED
:109370000E94B935882309F4BFC083E40E940732F4
:10938000882309F498C00E94DD316B017C01ACECAC
:10939000B5E0BF83AE83B987A887F5E0FD831D865E
:1093A0001E8628EC2F8702EC1A86212C88EC8B87EE
:1093B00092E49C87A885B985BA8BA98B15E0E989C9
:1093C000FA8981909190A190B190FA8BE98B2A85CE
:1093D000322D4B855C85C501B4010F94FA4F87FF90
:1093E00004C08A86292CAB86BC862D853E854F8598
:1093F000502FC501B4010F944C59181624F48D86D2
:109400009E86AF860B2D1150D1F6FD81F150FD8364
:1094100088859985449699878887F111CBCF2D85CA
:109420003E854F85502F6A85722D8B859C850F94C4
:10943000EC5620E030E040E05FE30F946050A7017D
:1094400096010F94EC566B017C012DEB37E346E857
:1094500055EB0F944C5987FD0AC02DEB37E346E8D6
:1094600055E3C701B6010F94FA4F181624F580E0B2
:109470000E94BE3415E0AE80BF8005E0D5016D913D
:109480007D918D919D915D014D01B4E08B1A910804
:10949000A70196010F94EB56F401608371838283D8
:1094A0009383015059F711508E819F8144969F8379
:1094B0008E831111E0CFA889AA2351F00E94B935FB
:1094C000882331F080E09DE00E9402370E945A38E4
:1094D0008AE50E940732882359F00E94DD316983B2
:1094E0007A838B839C8360E0CE0101960E94D934FD
:1094F000832D0E94BE340BC0311003C0988999237C
:1095000039F30E94504886E19DE00E9402373320E3
:1095100051F08091E50F811106C00E94674781EEEE
:109520009CE00E9402370E94504883ED9CE00E941C
:1095300002378091E50F0E94D9380E94504886EC8E
:109540009CE00E940237C0906408D0906508E090CB
:109550006608F090670820E030E0A901C701B60175
:109560000F944C5918160CF053C042E0C701B601D5
:109570000F945F078DE00E94C9368AE00E94C936C9
:10958000A30192016091E60F7091E70F8091E80FBF
:109590009091E90F0F94FA4F81111FC02B893C89DC
:1095A0004D895E896091EA0F7091EB0F8091EC0F0D
:1095B0009091ED0F0F94FA4F81110FC02F89388DC4
:1095C000498D5A8D6091EE0F7091EF0F8091F00FE1
:1095D0009091F10F0F94FA4F81110E9490F96A96C1
:1095E0000FB6F894DEBF0FBECDBFDF91CF911F91B4
:1095F0000F91FF90EF90DF90CF90BF90AF909F9032
:109600008F907F906F905F904F903F902F90089534
:1096100081EC9CE00E940237B3CFCF93C82F82E049
:10962000C11184E040E060E00E94D9850E9450486A
:1096300089EC99E0CC2311F08EED99E0CF910C9458
:109640000237FF920F931F93CF93DF93EC018B01AF
:10965000F42E0E944BD50E94674781E399E00E9457
:1096600002370115110511F401E81FE3209711F4E9
:10967000C8E2D9E00E9455BA1F930F93DF93CF93AE
:1096800088E199E09F938F9381E08F930E947EB34E
:109690000E94F084C0916F15C695C6958AE695E143
:1096A0000E948929DC2FDD0F1D2F1C0FEDB7FEB79F
:1096B00037960FB6F894FEBF0FBEEDBF83E00E9451
:1096C00007294DEA52E16C2F80E00E94342C109261
:1096D000A515D093A61589E099E00E94192A109249
:1096E000A5151093A6158CEF98E00E94192A8EE616
:1096F00095E10F94713A8111E1CF61E08FE199E03A
:109700000E94CA3789EE93E030E6019729F0232FB3
:109710002A950000E9F7F9CFF89489EE93E038EE46
:10972000019729F0232F2A950000E9F7F9CF0E942D
:109730004BD5FF2041F00E9434360E944922909977
:1097400005C0A895FCCF0E944722F7CF909B02C08E
:10975000A895FCCFF0E0E0E0DF91CF911F910F9151
:10976000FF9019945F926F927F928F929F92AF9227
:10977000BF92CF92DF92EF92FF920F931F93CF93FE
:10978000DF931F92CDB7DEB77C0139018B015B01FE
:10979000A40EB51ED12CC12CA016B10609F450C0E0
:1097A000F70180809180F80151908F015982C401A6
:1097B0000F9418565816B9F1652DC4010F94205610
:1097C000FFEFCF1ADF0AC6018F779927892B21F186
:1097D00062E070E080E090E00F944B32C4010F949F
:1097E000185699818917F9F00E9450488BE596E048
:1097F0000E94023781E00F90DF91CF911F910F916E
:10980000FF90EF90DF90CF90BF90AF909F908F90A0
:109810007F906F905F90089562E070E080E090E04C
:109820000E94FE35DBCFBE016F5F7F4FC3010F94F7
:109830001F24F70180819181019691838083ACCFB1
:1098400080E0D9CF8091F60F9091F70F2FEF3FEF87
:10985000981751F0E92FF0E0EA50F04F228130E004
:109860009F5F9F779093F70FC90108951F920F9202
:109870000FB60F9211240F900FBE0F901F901895E6
:109880001F920F920FB60F9211240BB60F920F93E7
:109890001F932F933F934F935F936F937F938F9378
:1098A0009F93AF93BF93CF93DF93EF93FF93C091B9
:1098B000C6000091F70FD091F60F11E01D0F1F7732
:1098C00090917904913108F09FC0E92FF0E088274A
:1098D000E359F34B8F4F0D94E3567E4CAD4CBC4C8B
:1098E000CB4CD24C044DD64C044DDA4CDE4C044DDE
:1098F000E24CE64CEA4CF14C044DFC4CC03229F0F1
:1099000028F5CA3011F0CD3031F5011731F0ED2FC7
:10991000F0E0EA50F04FC283D12FD093F60FFF91C1
:10992000EF91DF91CF91BF91AF919F918F917F91F7
:109930006F915F914F913F912F911F910F910F90D8
:109940000BBE0F900FBE0F901F901895CD3481F075
:1099500081E0CE3471F080E10CC0CA3338F4C033FA
:10996000A0F6C03291F2CD32B1F7CFCFCD3499F716
:1099700082E080937904C9CFC13359F018F4C03222
:1099800021F2E9CF88E0C433A1F38BE0C83389F337
:10999000E2CF83E0EECF84E0C03359F386E0C133F9
:1099A00041F3D9CF85E0C833B1F6E3CF87E0C233C6
:1099B00091F6DFCF89E0C13371F6DBCF8AE0C033A7
:1099C00051F6D7CF8CE0C73331F6D3CF8DE0C63315
:1099D00011F6CFCFC03209F498CF8EE0C33549F2EB
:1099E000BACF80ED8C0F8A3008F08FCF9FE0909334
:1099F00079048093780489CFCA3019F0CD3009F00A
:109A000084CF1092790481CFCA3019F0CD3009F09B
:109A10007CCF8091A8158823A1F3973041F138F4C9
:109A2000953079F710926C0210924C08EACF9A3078
:109A300011F19F3031F7909178048091490810928C
:109A40004908823089F38430E9F08130D1F69923D6
:109A5000B1F09130B1F682E080934B0880914A08D2
:109A6000882379F2109255020E943422CACF81E0F5
:109A700080934206C6CF81E080934106C2CF809397
:109A80004B08BFCF8BE09EE19093C2078093C10744
:109A9000B8CF8EBD0DB407FEFDCF08958FEF8EBDFC
:109AA0000DB407FEFDCF8EB50895909164009B7FA5
:109AB00090936400982F906A96959CBD80FD03C09A
:109AC00091E0863009F490E09DBD0895CF93DF9337
:109AD000EB010E940237CE01DF91CF910C9433CF7E
:109AE000AF92BF92CF92DF92EF92FF920F931F93AC
:109AF000CF93DF93CDB7DEB7E6970FB6F894DEBF0E
:109B00000FBECDBF0091F4041091F504F80101904F
:109B10000020E9F731976F01C01AD10AF801CF018F
:109B2000801B910B8C159D053CF481918F32B9F708
:109B3000DF0111971C92F3CF8BE1EBEFF5E1DE0132
:109B40005C9601900D928A95E1F7F12CE12CEC14D2
:109B5000FD040CF05DC0F801EE0DFF1D8081811148
:109B600003C08FEFE81AF80A5801AE0CBF1CF501CC
:109B70008081882309F44CC0FFEFEF1AFF0AF80137
:109B8000EE0DFF1D7F01E01AF10A81918111FACFDC
:109B9000CE014C960E942ED38BE1FE017C96DE0115
:109BA000119601900D928A95E1F7B501CE010196CB
:109BB0000E94F5CBCE0101960E9407348FE20E94ED
:109BC000C93680916A1281113BC087E593E00E94FB
:109BD00033CF8091DC1584FF1BC019821C8221E0E9
:109BE000A501BE01645E7F4FCE0101960F948005F2
:109BF000811129C08AE00E94C9360E945048B501EF
:109C000081EE94E10E94664DCE0101960E940734D8
:109C10008AE00E94C936CE014C960E940734E6962F
:109C20000FB6F894DEBF0FBECDBFDF91CF911F916D
:109C30000F91FF90EF90DF90CF90BF90AF9008957D
:109C40008AE692E1C4CFCE014C960E94EBD28BE122
:109C5000FE013196DE015C9601900D928A95E1F746
:109C6000CE0101960E94073472CF2F923F924F92FD
:109C70005F926F927F928F929F92AF92BF92CF929C
:109C8000DF92EF92FF920F931F93CF93DF9300D059
:109C900000D000D01F921F92CDB7DEB7B82E8091B2
:109CA000E310843008F0D1C10F947E326B017C0147
:109CB0008091E310811108C08091F60F9091F70F09
:109CC000891B8F7709F4D9C681E6A82E13C08A3084
:109CD00019F08D3009F0F6C01092DE1080917C10E2
:109CE00090917D10FC01E858FF4E1682892BF1F40B
:109CF0000E94EAF08091E310843008F0ECC080917B
:109D0000F60F9091F70F891B8F7709F4E4C00E943A
:109D1000224C97FFDCCF0E94674781EA97E00E94C0
:109D200002378091F60F8093F70FE4CF10927D10E9
:109D300010927C100EE710E1F8018191803209F455
:109D400046C08E3409F0A9C06CE977E0C8010F94D1
:109D5000774F4C01892B41F06EE470E0C801049606
:109D60000F94415A009709F4C8014AE050E070E0AE
:109D700060E001960F94E74C2B013C018091781034
:109D800090917910A0917A10B0917B100196A11D4D
:109D9000B11D481659066A067B0629F060E089E67F
:109DA00097E0892851F16AE270E0C8010F94705A77
:109DB0009C01009729F1982F901B912C992349F031
:109DC0009150F801E90FF11D80819826F7CF8F019E
:109DD000B3CF4AE050E070E060E0C90101960F9413
:109DE000E74C292D30E050E040E06217730784070C
:109DF000950751F060E08AE497E00F9486277ACFC8
:109E000060E080E297E0F9CF4092781050927910AC
:109E100060927A1070927B10809104088130E1F09A
:109E200067E470E0C8010F94415A0097A9F04AE036
:109E300050E070E060E001960F94E74C64307105EB
:109E40008105910548F48FE796E00E94023760E0B3
:109E500085E796E00E9499B3C0925108D0925208CB
:109E6000E0925308F092540880917E108B3309F4ED
:109E700041CF8091E310843008F03CCF8091E51011
:109E80008A9DC00111246EE770E18A519F4E0F94A4
:109E90004C5A80E00F9440272DCF8091DC1580FF35
:109EA000BBCF64E07FE3C8010F94774F009731F098
:109EB000FC01838180538A3008F0AECF60E086EFEA
:109EC00096E09BCF2CE730E14EE750E16EED70E17C
:109ED0000E94C3210FCF8091DC1582FFB6C01A8289
:109EE000198271E6F72EE0E1EE2EF9E6DF2E809181
:109EF000E310843008F0A9C00E94FB218111A5C0A5
:109F000041E050E0BE016B5F7F4F8FE397E10E941D
:109F1000D3CF0D8110E0019711F00FEF1FEF80916B
:109F2000471790914817A0914917B0914A1780930D
:109F3000D8159093D915A093DA15B093DB150E942C
:109F4000FB210F3F100749F4811107C00E946747AA
:109F50008FEB97E00E940237CACF4091E510242F83
:109F600030E00A3061F00D3051F0882309F45FC011
:109F700089819A81009719F001969A8389831092BA
:109F80007A0489819A81F29EF001F39EF00D1124EA
:109F9000ED51FF4EE80FF91F1382892B69F50E94DE
:109FA000EAF00E94FB21882309F4A1CF0E94FADC89
:109FB0008FE397E10E94EBD28091D315882391F132
:109FC00081508093D3158D9DC001112462E0805D86
:109FD000984F0F94DB40E091D31524E0E29FF0010D
:109FE0001124E45DF84F60817181828193810E9428
:109FF000DA250F94DB3D7BCF1A82198281E00F9422
:10A0000040278091D8159091D915A091DA15B0917B
:10A01000DB158093DF109093E010A093E110B093D4
:10A02000E210BFCF0F94CA3DE092040860CF4F9D6D
:10A03000A00111244A515F4E9E012F5F3F4F6AE7F6
:10A0400074E0802F0E94C32152CF0F947E326B01A7
:10A050007C01B11004C080912B07882351F0C0927D
:10A060004108D0924208E0924308F0924408BB2491
:10A07000B3948091CD049091CE04A091CF04B0917F
:10A08000D0040097A105B10551F1409141085091CC
:10A0900042086091430870914408840F951FA61FE1
:10A0A000B71FA7019601281B390B4A0B5B0BDA017E
:10A0B000C901B7FD14C00E94674760914F087091B5
:10A0C00050088AE198E00E94664D8AE00E94C936F5
:10A0D00040E070E060E090E080E00E94214B8091E1
:10A0E000100290911102A0911202B0911302892BDB
:10A0F0008A2B8B2B79F090914215809143159817FC
:10A1000009F4ACC1C0924108D0924208E0924308E1
:10A11000F092440880918B0490918C049099E0C156
:10A12000019690938C0480938B0480918B04909182
:10A130008C048E3E92406CF00E94674787EF97E058
:10A140000E94023740E070E060E090E080E00E9412
:10A15000214B0F947E324B015C0180914C088111A0
:10A1600008C0209142159091431581E0291301C048
:10A1700080E020911C1530911D1591E089272A3A25
:10A1800031050CF480E091E040917F04509180040F
:10A190006091810470918204452B462B472B09F472
:10A1A00090E0981789F0882309F4A0C1D501C40173
:10A1B00080569444A24FBF4F80937F0490938004B5
:10A1C000A0938104B09382044090F20F5090F30F5B
:10A1D0006090F40F7090F50F20917B0430917C0417
:10A1E00040917D0450917E04C301B2010F94FA4F57
:10A1F000882319F180917F0490918004A0918104BB
:10A20000B091820440927B0450927C0460927D0461
:10A2100070927E04892B8A2B8B2B09F449C0D501BF
:10A22000C40180569444A24FBF4F80937F04909303
:10A230008004A0938104B093820480917F04909164
:10A240008004A0918104B09182040097A105B1051A
:10A2500079F1881A990AAA0ABB0AB7FC29C0109298
:10A260007F0410928004109281041092820482EE86
:10A2700097E00E94023760E08EEC97E00E9499B36D
:10A2800080911E1590911F151816190624F490E060
:10A2900080E00E947CDC80916E0890916F08181617
:10A2A000190634F410926F0810926E080E945BC772
:10A2B0008091870490918804A0918904B0918A04C8
:10A2C00046015701881A990AAA0ABB0AD501C40196
:10A2D000B7FD9CC1209142159091431540915C02BD
:10A2E00080915B02291306C190918609899FC00164
:10A2F0001124880F892F881F990B91958D83809148
:10A300008709489FC0011124880F892F881F990B46
:10A3100091958E830F947E3269837A838B839C839D
:10A3200040E0BE016F5F7F4FCE0105960E944EDD7B
:10A330006D8170E089E00F94753141E0BE016F5F7F
:10A340007F4FCE0105960E944EDD6E8170E087E062
:10A350000F94753180914E06882309F44AC100910B
:10A36000330210913402C801029720911E153091DA
:10A370001F15281739070CF43CC1809043158F82B4
:10A38000188619861A861B86809142159F8089152A
:10A3900009F4CAC0892D90E030E6A32EA89EF001F2
:10A3A000A99EF00D1124E556F64F45895689678917
:10A3B000708D452B462B472B81F4418D528D638D3B
:10A3C000748D452B462B472B41F4458D568D678D5B
:10A3D00070A1452B462B472BE1F120E6B22EB89E0B
:10A3E0009001B99E300D1124A9014556564F1A010E
:10A3F000FA0161817281838194810F949A594B0192
:10A400005C01F10161A172A183A194A10F94FF4F9E
:10A410002B013C01F10165A176A187A190A50F94C4
:10A42000FF4F9B01AC01C301B2010F94E657A50198
:10A4300094010F9460504B015C01288539854A8551
:10A440005B850F944C59181624F488869986AA8641
:10A45000BB868F818F5F8F708F8396CFBB2019F063
:10A4600010928D0457CE0F947E32009141081091C6
:10A470004208209143083091440880901002909047
:10A480001102A0901202B0901302080D191D2A1D8E
:10A490003B1D601B710B820B930B97FDE1CF8091ED
:10A4A0008D04811137CE81E080938D045F9A809175
:10A4B000BF078E7F8093BF078A9A8091BF078D7FE9
:10A4C0008093BF0780910801809581708093060179
:10A4D0008091BF078B7F8093BF070E9447221ACECF
:10A4E000181619060CF021CE01971BCE80E090E0E3
:10A4F000DC0162CE2091431550E6259F9001112486
:10A500002556364FF901EA5AFF4F9081899FC001C5
:10A510001124880F892F881F990B91958D83295AB3
:10A520003F4FF9018081EDCE20912D0230912E0216
:10A5300040912F0250913002688579858A859B85EC
:10A540000F9460504B015C01B801012E000C880B88
:10A55000990B0F9401509B01AC01C501B4010F94FC
:10A56000EC5669837A838B839C83409131025091AE
:10A570003202B801CE0101960E9416D689809A80D7
:10A58000AB80BC804090830450908404609085042C
:10A5900070908604A3019201C501B4010F94FA4F93
:10A5A00087FF16C028E431EE4AE75FE3C301B2013A
:10A5B0000F94605020E037ED43EA5CE30F94EC56D3
:10A5C000A50194010F94605069837A838B839C83E7
:10A5D00069817A818B819C81609383047093840468
:10A5E00080938504909386040F945858CB010E9461
:10A5F0007CDCF4E6CF0ED11CE11CF11CC092870478
:10A60000D0928804E0928904F0928A040E94EAF0D1
:10A6100080910408882309F4F0C1809155028823B1
:10A6200009F471C080914A0881116DC00E942236E0
:10A63000811105C080912B07882309F464C0F89428
:10A64000649B10C08091510290915202A0915302DC
:10A65000B09154028093390690933A06A0933B063A
:10A66000B0933C066091390670913A0680913B06A2
:10A6700090913C06789420E030E0A9010F94FA4FC5
:10A6800087FF41C001E000934A0880912B078111A8
:10A6900038C00E94FB370093490840E366E878E041
:10A6A00083E490E40E94003861E087E390E40E9434
:10A6B000E2371091D10460E0102784E59AE069F454
:10A6C00084E798E00E94CA3780E30E94C9368AE096
:10A6D0000E94C93660E087E598E00E94CA3782E6AA
:10A6E00098E00E94023780E30E94C9368AE00E9407
:10A6F000C936112331F08DE598E09093C20780931D
:10A70000C1070E94FADC90910901892F8095817020
:10A7100010910802181709F45AC02091DC15206224
:10A720002093DC158093080290FD10C064EF71E067
:10A7300080E090E00E94FE350F94523E8091DC153F
:10A7400083FDBEC1112309F442C002C00F94413EF3
:10A75000123008F46BC100E00E949F2883E08093D0
:10A7600078020F947E326C597F4F8F4F9F4F6093CA
:10A77000F9047093FA048093FB049093FC04002383
:10A7800031F1123021F58091DC1583FF20C00F9448
:10A79000363D882379F081E00F94523C42EB50E043
:10A7A0006AE978E080EE95E10E94D3CF80EE95E1F2
:10A7B0000E94EBD20E94F533811144C10E94DF3325
:10A7C0000F94203F81E08093D2150F94623F0F9445
:10A7D0007E326B017C0110910F021123F1F0809108
:10A7E0004D088823D1F040918E0450918F046091E0
:10A7F00090047091910446015701841A950AA60AA3
:10A80000B70AB501A40177FD1AC0833009F430C13D
:10A810000CF01FC181300CF024C1212F30E0A8EED4
:10A82000B3E00F949256C60ED71EE81EF91EC092D2
:10A830008E04D0928F04E0929004F0929104809163
:10A840006208813009F073C00F947E326B017C0185
:10A850008091960490919704A0919804B0919904E6
:10A86000A7019601281B390B4A0B5B0BDA01C901C2
:10A87000B7FD3AC0D701C601805F984DAF4FBF4FBB
:10A880008093960490939704A0939804B0939904AE
:10A890008090BF059090C005A090C105B090C20502
:10A8A0000E941DFCAB01BC014093BF055093C00545
:10A8B0006093C1057093C2058091B0079091B10774
:10A8C000A091B207B091B30788199909AA09BB09E9
:10A8D000840F951FA61FB71F8093B0079093B107F1
:10A8E000A093B207B093B307809192049091930420
:10A8F000A0919404B091950446015701881A990AD1
:10A90000AA0ABB0AD501C401B7FD11C020E8C20ED6
:10A910002EEED21E26E3E21EF11CC0929204D092CB
:10A920009304E0929404F09295040E94FEDB0F944D
:10A93000E8010E94A5B78091CC04882379F10F9497
:10A940007E326B017C018091C8049091C904A09172
:10A95000CA04B091CB0446015701881A990AAA0A81
:10A96000BB0AD501C401B7FD19C02091CC0430E069
:10A97000A8EEB3E00F949256C60ED71EE81EF91E3D
:10A98000C092C804D092C904E092CA04F092CB04E9
:10A9900080E00F9403088AE00E94C9368091C704C2
:10A9A000882359F10F947E326B017C018091C3049E
:10A9B0009091C404A091C504B091C604A70196016A
:10A9C000281B390B4A0B5B0BDA01C901B7FD15C017
:10A9D0002091C70430E0A8EEB3E00F949256C60E63
:10A9E000D71EE81EF91EC092C304D092C404E092A0
:10A9F000C504F092C6040F944A3D2B960FB6F89406
:10AA0000DEBF0FBECDBFDF91CF911F910F91FF90A1
:10AA1000EF90DF90CF90BF90AF909F908F907F90FE
:10AA20006F905F904F903F902F90089560E087E97E
:10AA300098E00E9499B38091070581118CCE0E9405
:10AA4000F08489CE84EB98E09093C2078093C1078D
:10AA5000BECE843009F0E1CE0E9450488BEB98E0E6
:10AA600004C00E9450488AEE98E00E940237D5CE7A
:10AA70000E94504883ED98E0F8CF80915108909162
:10AA80005208A0915308B0915408A7019601281BC1
:10AA9000390B4A0B5B0BDA01C901885E9340A109AF
:10AAA000B109B7FD11C989EB97E00E940237C09246
:10AAB0005108D0925208E0925308F092540804C909
:10AAC000123028F460E085EA98E00E9499B301E032
:10AAD00043CECF93DF93C82FD62F80919C0F83FD59
:10AAE00014C080919809811110C080917D029091CD
:10AAF0007E02AC014150510920911E1530911F1565
:10AB00002417350714F40E947CDC40E06D2F8BE0A5
:10AB10000E94D985CC2339F040E061E080E0DF91EC
:10AB2000CF910D94FB098091980991E0892780933A
:10AB30006C0280916C02882389F080911C159091A1
:10AB40001D1520911E1530911F15821B930B97FF29
:10AB500003C0919581959109029744F410926C027B
:10AB600080919C0F83FF06C0C1E01AC080E00E9464
:10AB7000354EDFCFC0919809C11112C080917D027E
:10AB800090917E02019720911E1530911F15281774
:10AB9000390754F70E94504888EB99E00E94023729
:10ABA0008C2FDF91CF910895AF92BF92CF92DF9219
:10ABB000EF92FF920F931F93CF93DF93CDB7DEB742
:10ABC00064970FB6F894DEBF0FBECDBF0E94544805
:10ABD000D82E87FDB5C08AE50E945532882309F436
:10ABE000C0C040E050E0BA018AE50E9470327B01AB
:10ABF0008C014D2D63E085E00E94D9852091EE0FF8
:10AC00003091EF0F4091F00F5091F10F60E070E044
:10AC100088EC93E40F94EB565B016C019701A8015B
:10AC20000F944C59181614F07501860120E030E09D
:10AC3000A901B701C8010F944C59181624F4E12C4E
:10AC4000F12C00E010E0B701C8010F945858072E0E
:10AC5000000C880B990B0F9401506D837E838F83BA
:10AC6000988720E030E0A9010F94FA4F882321F063
:10AC7000CE0105960E94282680E090E0A0EAB1E48B
:10AC800089879A87AB87BC871D861E861F86188A90
:10AC90008CE40E940732882309F468C00E94DD31E9
:10ACA0006B017C0120E030E0A901C701B6010F94DF
:10ACB0004C5987FF04C0F7FAF094F7F8F094C98A6A
:10ACC000DA8AEB8AFC8A20911E1530911F152430F8
:10ACD000310574F080911C1590911D15821B930B0A
:10ACE00097FF03C091958195910901E004970CF4B9
:10ACF00000E063E080E00E946955811140C083E07C
:10AD000080932402109206050E94F0846D817E815A
:10AD10008F8198858B019C01305809831A832B837E
:10AD20003C8320E030E0A9010F94FA4F882321F002
:10AD3000CE0101960E942826109206050E94F084FA
:10AD400064960FB6F894DEBF0FBECDBFDF91CF91F2
:10AD50001F910F91FF90EF90DF90CF90BF90AF9039
:10AD60000895E12CF12C00E211E443CFC090C70517
:10AD7000D090C805E090C905F090CA0593CF83E054
:10AD8000E82E22E0AE01475F5F4FBE016F5E7F4F4E
:10AD9000CE010D960F948A29B9CF6F927F928F9230
:10ADA0009F92AF92BF92CF92DF92EF92FF920F935A
:10ADB0001F93CF93DF9300D000D01F921F92CDB787
:10ADC000DEB75C014B013A01F22E680100914706A3
:10ADD00010924306109244061092450610924606C1
:10ADE000109247060F948A3280911E1590911F157C
:10ADF0008C159D051CF4C6010E947CDC60E080E09F
:10AE00000E94695581112FC1109206050E94F0849D
:10AE10001C141D0444F4C6010E947CDC40E060E088
:10AE200080E00F94FB0940E060E088E00E94D98553
:10AE300060E081E00E94695580E090E0A0E7B2E424
:10AE400089839A83AB83BC8380E090E0A0E8B0EC78
:10AE50008D839E83AF83B887BE016F5F7F4FCE0126
:10AE600005960E94B8F087E00E94F8EE811158C064
:10AE70008091EE0F9091EF0FA091F00FB091F10F34
:10AE80004091A6045091A7046091A8047091A90470
:10AE9000C090A204D090A304E090A404F090A50474
:10AEA000C0923108D0923208E0923308F092340810
:10AEB00040933508509336086093370870933808EC
:10AEC0008093390890933A08A0933B08B0933C08CC
:10AED00080E090E0A8E4B2E489839A83AB83BC83EA
:10AEE000CE0101960E94D8F78091AA049091AB04FC
:10AEF000A091AC04B091AD048093390890933A08C6
:10AF0000A0933B08B0933C0880E090E0A0EAB0E456
:10AF100089839A83AB83BC83CE0101960E94D8F7C4
:10AF2000C12CD12C80E7E82E82E4F82EC982DA8287
:10AF3000EB82FC8280E090E0A0E8B0E48D839E8309
:10AF4000AF83B887BE016F5F7F4FCE0105960E9429
:10AF5000B8F020E030E0A9016091AE047091AF0438
:10AF60008091B0049091B1040F94FA4F87FF0BC009
:10AF7000C982DA82EB82FC82BE016F5F7F4F8EEA6C
:10AF800094E00E94B8F08091AE049091AF04A0913B
:10AF9000B004B091B1048093F20F9093F30FA0939B
:10AFA000F40FB093F50F80933D0890933E08A09363
:10AFB0003F08B09340088DE398E00E9430ED809107
:10AFC000CB0581110F947C3C109206050E94F08401
:10AFD00061E081E69AE00E94CA3780912B07815098
:10AFE00080932B074CEC5DE169E67AE085E00F94F5
:10AFF000942A80912B07882339F00F94DB3D8091B0
:10B000002B07815080932B078091A104882351F056
:10B010001092A10480919F04809386098091A004DE
:10B02000809387090E94342280916208823011F453
:10B030000E94DFFC0F941B400E94F08428960FB6FC
:10B04000F894DEBF0FBECDBFDF91CF911F910F915E
:10B05000FF90EF90DF90CF90BF90AF909F908F9038
:10B060007F906F900895E12C2F2DA301B401C501AD
:10B070000F948A29CDCE4F925F926F927F92AF92BA
:10B08000BF92CF92DF92EF92FF921F93CF93DF9305
:10B0900000D000D01F921F92CDB7DEB75C01E62E24
:10B0A000F42E642F80E00E946955182F81111BC077
:10B0B000EE2021F0109206050E94F084812F289640
:10B0C0000FB6F894DEBF0FBECDBFDF91CF911F91B9
:10B0D000FF90EF90DF90CF90BF90AF907F906F90F8
:10B0E0005F904F900895EE2029F040E06F2D83E0AF
:10B0F0000E94D98580E090E0A0E7B2E48D839E8332
:10B10000AF83B88780E090E0A0E8B0EC89839A83B1
:10B11000AB83BC83BE016B5F7F4FCE0101960E9463
:10B12000B8F068E873E180E090E00E94FE35C12C41
:10B13000D12C88ECE82E81E4F82ECD82DE82EF82DD
:10B14000F88680E090E0A0E8B0E489839A83AB833E
:10B15000BC83BE016B5F7F4FCE0101960E94B8F0A9
:10B160004090D50F5090D60F6090D70F7090D80FA9
:10B17000C092D50FD092D60FE092D70FF092D80F91
:10B1800080E090E0A0E2B2E48D839E83AF83B88735
:10B19000F50180819181A281B38189839A83AB83F8
:10B1A000BC83BE016B5F7F4FCE0101960E94B8F059
:10B1B0004092D50F5092D60F6092D70F7092D80F51
:10B1C000129A64E670E080E090E00E94FE3576CF4F
:10B1D000BF92CF92DF92EF92FF920F931F93CF9384
:10B1E000DF9300D01F92CDB7DEB77C016B018A01DF
:10B1F000B22E61E084E59AE00E94CA374CEC5DE132
:10B200006BE57AE085E00F94942A90912B0781E01A
:10B21000890F80932B078091DC1582FF06C08B7FFE
:10B220008093DC159E5F90932B070E9417FD80E1B1
:10B23000E6EEFFE0A2EAB4E001900D928A95E1F714
:10B240000E94FADC8091A10481110FC081E08093FB
:10B25000A1048091860980939F04109286098091B1
:10B2600087098093A0041092870920E030E0A901AB
:10B27000F70160817181828193810F94FA4F882355
:10B28000F1F08091980981110CC080917D0290911C
:10B290007E02019720911C1530911D152817390742
:10B2A00074F080E090E0A0E7B2E489839A83AB83F6
:10B2B000BC83BE016F5F7F4FC7010E94B8F087E07B
:10B2C0000E94F8EE811103C0B6010F942D0120E019
:10B2D00030E0A901F80160817181828193810F942E
:10B2E000FA4F882329F042E06B2DC8010E943B5899
:10B2F000129A64E670E080E090E00E94FE3581E002
:10B300000F900F900F900F90DF91CF911F910F91A1
:10B31000FF90EF90DF90CF90BF900895CF92DF9293
:10B32000EF92FF92CF93DF936B017C01D42FC091FA
:10B330004D0883E080934D0881E080934C08C11450
:10B34000D104E104F10431F00F947E32C60ED71E11
:10B35000E81EF91E80914C08882389F0C114D1049D
:10B36000E104F10421F48D2F0E94354EF3CF0F94A8
:10B370007E326C197D098E099F0997FDF4CF1092DA
:10B380004C08C0934D08DF91CF91FF90EF90DF9074
:10B39000CF9008951F93CF93DF93D82FC62F0E948D
:10B3A0000D4B61E08C2F0E940D340F947E32685358
:10B3B00070458F4F9F4F6093430670934406809370
:10B3C0004506909346061092470610914D0883E07B
:10B3D00080934D0830E020E048E650E466E47AE0EF
:10B3E00082E00E94233881E080934C0880914C08D1
:10B3F000882309F463C060E08C2F0E940D34809193
:10B400004706882309F456C040E060E08AE00E94C5
:10B41000D9850E9450488CE29AE00E94023730E0C1
:10B4200020E046E15AE06DE17AE082E00E942338B4
:10B4300041E060E070E0CB010E948E5930E020E0F6
:10B4400050E040E069E07AE085E00E942338109205
:10B45000430610924406109245061092460610923A
:10B4600047060F948A3260E080E00E9469558D2F74
:10B470000E940D4B0F947E32685370458F4F9F4F43
:10B480006093430670934406809345069093460666
:10B490001092470630E020E048E650E46DEF79E096
:10B4A00082E00E94233881E080934C0861E08C2F79
:10B4B0000E940D3481E00E94354E98CF10934D08C4
:10B4C000DF91CF911F910895CF92DF92EF92FF927B
:10B4D0000F931F93CF93DF93CDB7DEB7A0970FB62F
:10B4E000F894DEBF0FBECDBF0E94544887FDD1C087
:10B4F000482F61E081E00E94D98585E40E940732EF
:10B50000882309F4D5C00E94DD316B017C0120E065
:10B5100030E0A9010F944C5987FF04C0F7FAF0946A
:10B52000F7F8F094F7FAF094F7F8F094C98ADA8A09
:10B53000EB8AFC8A8CE0E3E8F2E0DE0111960190F0
:10B540000D928A95E1F78AE50E945532882351F0E1
:10B5500040E050E0BA018AE50E94703269877A873C
:10B560008B879C8788E50E945532882351F040E004
:10B5700050E0BA0188E50E94703269837A838B8338
:10B580009C8389E50E945532882351F040E050E0C9
:10B59000BA0189E50E9470326D837E838F8398871C
:10B5A00085E50E940732882309F489C00E94DD31B5
:10B5B0006B017C0120E030E0A901C701B6010F94C6
:10B5C0004C5987FF04C0F7FAF094F7F8F094F7FAB3
:10B5D000F094F7F8F094CD8ADE8AEF8AF88E198E0F
:10B5E0001A8E1B8E1C8E8CE40E940732882309F46D
:10B5F0006FC00E94DD316B017C0120E030E0A901C9
:10B60000C701B6010F944C5987FF04C0F7FAF094B4
:10B61000F7F8F094CD8EDE8EEF8EF8A262E070E047
:10B6200082E40E94BB33F82E80912B07811131C038
:10B6300021E0AE014B5E5F4FBE016F5F7F4FCE01D9
:10B6400041960E94E858882321F16F2D81E00E94E5
:10B65000CA5982E50E945532882309F442C00E94EB
:10B66000D93140E050E060EA71E44D875E876F8732
:10B67000788B20912B07222361F08C012F2DAE01B6
:10B68000435F5F4FBE01635E7F4FCE0149960E94CC
:10B69000CD56A0960FB6F894DEBF0FBECDBFDF919A
:10B6A000CF911F910F91FF90EF90DF90CF90089571
:10B6B000C12CD12C80E8E82E80E4F82E33CFC09046
:10B6C000C305D090C405E090C505F090C60572CFC3
:10B6D000C090C705D090C805E090C905F090CA0594
:10B6E0008CCF90E080E0BDCFCF92DF92EF92FF92BF
:10B6F0000F931F93CF93DF93CDB7DEB76C970FB641
:10B70000F894DEBF0FBECDBF8CE40E9407328823C1
:10B7100009F4C3C00E94DD316B017C0120E030E000
:10B72000A9010F944C5987FF04C0F7FAF094F7F879
:10B73000F094F7FAF094F7F8F094C98EDA8EEB8E65
:10B74000FC8E8CE0E3E8F2E0DE01119601900D92B0
:10B750008A95E1F788E50E9455328823A1F040E000
:10B7600050E0BA0188E50E94703220914C09309176
:10B770004D0940914E0950914F090F94EB56698342
:10B780007A838B839C8389E50E9455328823A1F0BC
:10B7900040E050E0BA0189E50E94703220914C09E6
:10B7A00030914D0940914E0950914F090F94EB563D
:10B7B0006D837E838F8398878AE50E945532882324
:10B7C00051F040E050E0BA018AE50E94703269878A
:10B7D0007A878B879C87F090DC15F2FAFF24F0F8CB
:10B7E00040E061E080E00E94D98560E080E50E9451
:10B7F000CA33E82E1D861E861F86188A80912B0765
:10B8000081113CC02E2DAE01435F5F4FBE016F5FC3
:10B810007F4FCE0149960E94E858882379F18091A4
:10B82000CB0581110F947C3CFF2011F0EE2031F10B
:10B8300060E080E00E94CA59898D9A8DAB8DBC8DE5
:10B84000B0588D8B9E8BAF8BB88F198A1A8A1B8A42
:10B850001C8A1D861E861F86188A80912B078823C6
:10B8600069F010E000E020E0AE014B5E5F4FBE01EA
:10B870006F5E7F4FCE010D960E94CD566C960FB62F
:10B88000F894DEBF0FBECDBFDF91CF911F910F9116
:10B89000FF90EF90DF90CF900895C12CD12C80E8DD
:10B8A000E82E80E4F82E45CF2F923F924F925F9280
:10B8B0006F927F928F929F92AF92BF92CF92DF92C0
:10B8C000EF92FF920F931F93CF93DF93CDB7DEB725
:10B8D000E1970FB6F894DEBF0FBECDBF89AB2091C4
:10B8E0004D0828AB11E010934D088091F3048D347E
:10B8F00009F463C4843511F40C941271873409F08F
:10B9000044C18091F1049091F2048A31910509F4C7
:10B91000D7C108F03DC18430910508F030C12091B5
:10B9200004088230910508F451C1213009F054C156
:10B9300011E0029709F010E00E94873219821A8202
:10B940001B821C821D821E821F82188682E50E9435
:10B950005532882309F453C10E94DD316B017C010B
:10B9600020E030E0A9010F94FA4F882309F4EAC0DF
:10B970004090E60F5090E70F6090E80F7090E90F4D
:10B980008091EA0F9091EB0FA091EC0FB091ED0F29
:10B9900088A799A7AAA7BBA78090310890903208E2
:10B9A000A0903308B0903408809135089091360803
:10B9B000A0913708B09138088CA79DA7AEA7BFA764
:10B9C000A5019401C301B2010F94FA4F81110DC07A
:10B9D0002CA53DA54EA55FA568A579A58AA59BA523
:10B9E0000F94FA4F882309F4ADC0A3019201C50159
:10B9F000B4010F94EB5620E030E040E05FE30F9499
:10BA000060506CA37DA38EA39FA328A539A54AA54A
:10BA10005BA56CA57DA58EA59FA50F94EB5620E098
:10BA200030E040E05FE30F9460502B013C0120E0E8
:10BA300030E0A901C701B6010F94FA4F881F88278B
:10BA4000881F181709F4D2C080E090E0A0E8BFEB8F
:10BA500088A799A7AAA7BBA72CA13DA14EA15FA12A
:10BA6000CA01B9010F9460504B015C01A30192011E
:10BA7000C301B2010F9460509B01AC01C501B40138
:10BA80000F94EC560F949A594B015C01AC019B0149
:10BA9000C701B6010F94EB566CA77DA78EA79FA791
:10BAA000A5019401C701B6010F94EC569B01AC01AE
:10BAB0006CA57DA58EA59FA50F9460506B017C01A0
:10BAC00020E030E0A9010F944C5987FD94C0C701D4
:10BAD000B6010F949A596B017C01C301B2019058D1
:10BAE000A50194010F94E65728A539A54AA55BA5A1
:10BAF0000F946050A70196010F9460502CA13DA1B6
:10BB00004EA15FA10F94EC5669837A838B839C834B
:10BB1000A50194016CA17DA18EA19FA10F94E65770
:10BB200028A539A54AA55BA50F946050A7019601E9
:10BB30000F946050A30192010F94EC566D837E83A5
:10BB40008F83988720E030E0A90169817A818B8119
:10BB50009C810F94FA4F811166C020E030E0A9016A
:10BB60006D817E818F8198850F94FA4F81115BC022
:10BB70000E9467478EE39FE00E9402372DC0843009
:10BB8000910509F463C0459739F10F947C2924C0CD
:10BB90008A32910509F4ECC158F48C31910509F40D
:10BBA000AAC008F490C04D9781F70E94237414C076
:10BBB0008B35910509F459C28C35910509F459C2A8
:10BBC0008A35910511F71092630806C0213021F4DF
:10BBD0000E9487320E9425F539A9311102C00F94C5
:10BBE000DF3288A980934D080C94A46980E090E02E
:10BBF000A0E8BFE32DCFC12CD12C76016ECF89E414
:10BC00000E945532882331F00E94DD3169837A83A6
:10BC10008B839C838AE40E945532882309F492CF57
:10BC20000E94DD318BCF412FBE016F5F7F4F81E3DB
:10BC300098E00F9478330F947E32609341087093AC
:10BC400042088093430890934408C6CF80E50E9441
:10BC50005532C12CD12C7601882321F00E948627F1
:10BC60006B017C0183E50E945532882361F00E94BC
:10BC7000DD3120E030E04AE754E40F9460500F9447
:10BC80005F586B017C010E94FADC8091AD1281113A
:10BC900005C060E084E59FE00E9499B30F947E3276
:10BCA000C60ED71EE81EF91E0F947E326C197D0950
:10BCB0008E099F0997FF90CF80E00E94354EF4CF08
:10BCC0000E94173E89CF0F943D40811185CF8CE0B3
:10BCD000EFE8F2E0DE01119601900D928A95E1F70E
:10BCE00070E060E080E50E946232BE016F5F7F4FCE
:10BCF0000F942D0171CF87E00E94F8EE811106C0EC
:10BD000060E08FE40E94CA33811166CF0E94FADCA2
:10BD1000109238026091E50F8CE40E94CA33982E8D
:10BD200080E00E94BE340F947E326093410870938D
:10BD30004208809343089093440880917402909144
:10BD40007502A0917602B09177028093BF04909320
:10BD5000C004A093C104B093C20480916E0290917C
:10BD60006F029093BE048093BD0484E690E09093AC
:10BD70006F0280936E0281E08093BD070E9499FA62
:10BD80008AE50E940732A82E88E50E940732182F04
:10BD900089E50E940732B82E181308C0B12EA112EF
:10BDA00005C011E0BB24B394AA24A39482E50E94A9
:10BDB0005532882309F4D2C00E94DD316C8F7D8F0B
:10BDC0008E8F9F8F20E030E0A9010F94FA4F8823D7
:10BDD00049F0111103C0BB2009F494C0CE014C9668
:10BDE0000F94692B112309F488C0BB2009F482C089
:10BDF0001092E60F1092E70F1092E80F1092E90FE1
:10BE00001092EA0F1092EB0F1092EC0F1092ED0FC0
:10BE10000E94E8F0ECEBF7E2C590D590E590F49045
:10BE2000E0ECF7E24590559065907490A70196017B
:10BE3000C301B2010F94FA4F87FF95C0A701960185
:10BE4000C301B2010F94E6579B01AC010F946050FF
:10BE500020E030E040E85FE30F94EC560F949A59ED
:10BE600020E030E048E452E40F94605069837A8324
:10BE70008B839C838091EE0F9091EF0FA091F00F38
:10BE8000B091F10F8CA39DA3AEA3BFA320E030E03F
:10BE900040EC5FE3C301B2010F9460502B013C0101
:10BEA00077FA709477F8709420E030E040EC5FE32C
:10BEB000C701B6010F9460509058DE0111966D01D4
:10BEC000ECA0FDA00EA11FA1A30192010E94E1EF31
:10BED0000E940FFC1092E60F1092E70F1092E80FED
:10BEE0001092E90F1092EA0F1092EB0F1092EC0FE4
:10BEF0001092ED0F80E00E943FF8BB2019F081E026
:10BF00000E943FF8AA2019F082E00E943FF80E94A8
:10BF1000E8F08091BC078093BD07892D0E94BE3454
:10BF20008091BF049091C004A091C104B091C2045B
:10BF30008093740290937502A0937602B093770277
:10BF40008091BD049091BE0490936F0280936E0225
:10BF500083E0809378020E9490F93ECE60E070E02A
:10BF600080E890E42BCFA3019201C701B6016ACF0C
:10BF700080910408813009F02FCE89E40E94553267
:10BF8000082F10E0882319F00E94D931182F8AE475
:10BF90000E945532F82E882339F00E94D9310111C0
:10BFA00006C0853068F005C080E0002349F01530F8
:10BFB00028F08DE59FE00E9402370ECEF110F1CF00
:10BFC00090E1E6EEFFE0A1E3B8E001900D929A95D2
:10BFD000E1F7002391F0B4E01B02F0011124E354D7
:10BFE000FA4E4081518162817381409331085093B0
:10BFF00032086093330870933408FF2091F024E0F6
:10C000008202F0011124E755FA4E80819181A281CC
:10C01000B3818093350890933608A0933708B09386
:10C02000380840E050E0BA0186E40E9470326B01AB
:10C030007C0120E030E0A9010F944C5918168CF4D3
:10C0400020E030E040E752E4C701B6010F94E65724
:10C0500069837A838B839C83CE0101960E94D8F7F3
:10C06000BBCD60E070E0CB01F3CF8FE0809363083D
:10C07000B3CD8091F004882381F1893009F0ACCDF3
:10C080006BE9A62E62E0B62E76EEC72E7FE0D72EA5
:10C09000E12C00E010E0D5018D915D010E94553248
:10C0A000F82E882361F0133011F4082FFE2C0E9423
:10C0B000DD31F6016083718382839383EF2C1F5FF0
:10C0C000F4E0CF0ED11C143031F7EE2009F457C044
:10C0D0000E94E8F00E9490F97FCD5BE9C52E52E006
:10C0E000D52EF12CE12C00E010E0D6018D916D01F0
:10C0F0000E945532382E8823D9F10E94DD314B0140
:10C100005C01133059F0F701E45BF64F2081318177
:10C11000428153810F94EB564B015C01F701EA51C8
:10C12000F04F2081318142815381C501B4010F94C8
:10C13000EB562B013C012DEB37E346E855EB0F9412
:10C140004C5987FD0AC02DEB37E346E855E3C301A0
:10C15000B2010F94FA4F18165CF41330C1F48092B8
:10C16000F20F9092F30FA092F40FB092F50F032DFF
:10C170001F5FB4E0EB0EF11C143009F0B6CF0023C2
:10C1800009F4A8CF82EF9FE00E9430EDA3CFF70122
:10C19000EE57F74F5F01A3019201608171818281A7
:10C1A00093810F94EC56D5016D937D938D939C9361
:10C1B0001397812F0E94D8EEDBCF8091F1049091EC
:10C1C000F2048837910511F40C94B26B08F07BC22D
:10C1D0008D34910509F4E6C708F0D3C08A31910582
:10C1E00009F408C708F094C08431910509F44EC6DB
:10C1F00008F071C08131910509F40FC608F044C000
:10C20000029708F0C2CC80E50E945532C12CD12C97
:10C210007601882321F00E9486276B017C0183E54B
:10C220000E945532882361F00E94DD3120E030E029
:10C230004AE754E40F9460500F945F586B017C01FF
:10C240000E94FADC8091F4049091F504009709F4BF
:10C25000DEC50F94E93F8091F1049091F2046EE7FE
:10C260007FE0892B11F466E77FE030E020E048E6CC
:10C2700050E482E00E94233840E0C701B6010E94EA
:10C280008E590F941B40A8CC429709F07ECC83E5D1
:10C290000E945532882311F40C94E96A0F947E327F
:10C2A0006093410870934208809343089093440838
:10C2B0000E94DD3120E030E04AE754E40F94605002
:10C2C0000F945F58609310027093110280931202D2
:10C2D0009093130281CC8731910509F40CC670F458
:10C2E0008531910509F403C6469709F04ECC80913B
:10C2F000DC1582FD71CC0F94413E6ECC88319105E6
:10C3000009F40EC6499709F040CC0E94745B64CCD6
:10C310008F31910509F413C7D0F48C31910509F4DC
:10C32000D6C608F47AC68D31910509F4D8C64E9761
:10C3300009F02BCC8091DC1583FF4ECC0F94622941
:10C340008091F4049091F5040F94B83E45CC893463
:10C35000910509F413C750F48032910509F4C6C65B
:10C36000819709F012CC0E94704D36CC8B34910528
:10C3700009F414C78C34910509F007CC0E9417FD0D
:10C380002BCC8B36910511F40C94BD6908F00FC1CC
:10C390008435910509F47BCF40F58135910511F481
:10C3A0000C94C96A90F48E34910509F0EECB70E0DC
:10C3B00060E083E50E94BB338E34910509F0F7C637
:10C3C0000E9420DC0F941B4007CC8235910511F4AC
:10C3D0000C94E16A8335910509F0D7CB809163080D
:10C3E0008F7E806280936308F7CB8836910509F4CD
:10C3F00062C708F09CC08535910511F40C942C6B34
:10C400008C35910509F0C1CB0E94544887FDE4CBDF
:10C410008091EC0484FD0AC08091EE0487FD06C083
:10C420008091EF04837011F40C945A6B2BE9C22EA7
:10C4300022E0D22E3DE9E32E3FE0F32E10E0D601BC
:10C440008D916D010E945532882309F466C0133026
:10C4500011F00C94516B0E94DD314B015C0120E026
:10C4600030E040EA51E40F94FA4F87FF4EC0A50137
:10C4700094016091BD0F7091BE0F8091BF0F90919C
:10C48000C00F0F94E6572B013C01AC019B0160915A
:10C490006A0970916B0980916C0990916D090F94F4
:10C4A000605060936A0970936B0980936C09909354
:10C4B0006D09A30192016091CD0F7091CE0F809113
:10C4C000CF0F9091D00F0F9460506093CD0F709369
:10C4D000CE0F8093CF0F9093D00F60917A09709117
:10C4E0007B0980917C0990917D090F94FF4FA301F6
:10C4F00092010F9460500F945F5860937A09709383
:10C500007B0980937C0990937D098092BD0F909266
:10C51000BE0FA092BF0FB092C00F1F5FF4E0EF0EEE
:10C52000F11C143009F08BCF0E94D6DC55CB893634
:10C53000910509F4F7C68A36910509F026CB80E506
:10C540000F949D2AF82E81E08F1508F445CB81E4E5
:10C550000E94073260918609062F10E0811102C007
:10C560000FEF10E089E40E945532882311F40C94F7
:10C5700041710E94B53190E01816190614F481E05B
:10C5800090E026E0289FF001299FF00D1124EB5F39
:10C59000F74F04811581EF2DF0E0EA57F64F0F3F7A
:10C5A000110519F010F00FEF10E0008315CB813763
:10C5B000910509F444C708F068C08E36910509F466
:10C5C000EAC608F059C08C36910509F405CB8D36C2
:10C5D000910509F0DACA80919C0F83FDFDCA0E9483
:10C5E0005448F82E87FDF8CA89E40E945532882302
:10C5F00011F40C9430710E94B53190E018161906B0
:10C6000014F481E090E026E0289FF001299FF00DCE
:10C610001124EB5FF74F8081918110E00E947CDC58
:10C6200061E081E00F942A4420911E1530911F157E
:10C6300080911C1590911D15821793070CF069C607
:10C640008FE690E19F938F938AE790E19F938F937A
:10C650001F920E947EB30F900F900F900F900F903B
:10C6600001E00F94F343002309F4B6CA40E0612FC0
:10C670008F2D0F94FB09B0CA8F36910509F49EC621
:10C680008037910509F4A8CA80CA8537910511F44D
:10C690000C94676B60F48237910511F40C945F6B16
:10C6A0008337910509F071CA0E94293795CA8637E8
:10C6B000910511F40C94796B8737910509F065CADF
:10C6C0000E9476FA89CA8039E1E09E0711F40C9441
:10C6D000686E08F059C28D3C910511F40C94BC6C45
:10C6E00008F0A6C08B39910509F42CC740F58D37A9
:10C6F000910509F40ACE58F48937910509F045CA25
:10C700001092BD071092BC070E9499FA65CA8C3836
:10C71000910509F4B3C68139910509F036CA70E074
:10C7200060E083E50E94BB33823010F40C94BA6B56
:10C730000E94674780ED90E10E9402374DCA893C14
:10C74000910511F40C94276CB0F58E3B910509F41A
:10C75000BBC6883C910509F018CA0E945448182F9E
:10C7600087FD3ACA0091810884E40E945532F82E70
:10C770008823C1F00E94DD314B015C0120E030E0F4
:10C78000A9010F94FA4F882311F40C94246C24E02F
:10C790001202F0011124E358F74F80829182A282A5
:10C7A000B3820F2D602F83E50E94CA3380938108E6
:10C7B0000E940CC511CA8B3C910511F40C94516C6C
:10C7C0008C3C910509F0E1C98091ED0487FF02C01E
:10C7D0000C94746C8091EE048E7011F00C94746C57
:10C7E0004091D10F5091D20F6091D30F7091D40F1F
:10C7F00085EF90E10E94F7384091D50F5091D60F08
:10C800006091D70F7091D80F82EF90E10E94F738B6
:10C810004091D90F5091DA0F6091DB0F7091DC0FCE
:10C820008DE69CE20E94F7388AE00E94C936D4C99E
:10C83000823221E0920711F40C94A46D08F09CC0A0
:10C84000833D910511F40C94436D08F050C0AEE89F
:10C85000EA2EA8E0FA2E10E08E3C910509F095C969
:10C8600088E5810F0E940732882351F00E94DD3154
:10C87000F7016083718382839383812F0E94D8EEB6
:10C880001F5FF4E0EF0EF11C133051F78091EE04BE
:10C8900087FD20CC8091EF04837009F01BCC409180
:10C8A0008E0850918F08609190087091910887E3ED
:10C8B00091E10E94F738409192085091930860915D
:10C8C00094087091950881EF90E40E94F7384091A8
:10C8D00096085091970860919808709199088EEE8B
:10C8E00090E40E94F7388AE00E94C93675C98C3DF1
:10C8F000910511F40C94476D8D3D910509F045C9E2
:10C900000E945448082F87FD67C983E50E9455326D
:10C91000002E000C110B7801EE0CFF1C882311F483
:10C920000C948A6D0E94D931F701EB5CFD4F918325
:10C930008083000F111F000F111F980127583D4FD2
:10C940007901BC01990F880B990B0F9401502AE0D3
:10C9500037ED43E25CE30F94605009541A4FD8015D
:10C960002D913D914D915C910F946050F701608342
:10C9700071838283938330C98E32A1E09A0711F4C8
:10C980000C941E6E08F083C08C32E1E09E0711F417
:10C990000C94006E8D32914009F0F7C885E40F9435
:10C9A0009D2A81110C94166E80E50E94073288231F
:10C9B00051F00E94DD316093211570932215809310
:10C9C00023159093241589E40E940732882381F06F
:10C9D0000E94DD312CEA35EC47E25EE30F946050B3
:10C9E000609325157093261580932715909328152D
:10C9F00084E40E940732882381F00E94DD312CEA12
:10CA000035EC47E25EE30F94E65760932915709387
:10CA10002A1580932B1590932C150E945048409115
:10CA200021155091221560912315709124158FE5E1
:10CA300091E10E94F7382CEA35EC47E25EE3609121
:10CA400025157091261580912715909128150F9422
:10CA5000E657AB01BC018BE591E10E94F7382CEA67
:10CA600035EC47E25EE36091291570912A158091BB
:10CA70002B1590912C150F946050AB01BC0187E5EC
:10CA800091E10E94F7388AE00E94C936A5C88F322A
:10CA900021E0920711F40C94646E8033914009F008
:10CAA00074C880E50E940732882351F00E94DD316E
:10CAB0006093710870937208809373089093740860
:10CAC00089E40E940732882381F00E94DD312CEA3C
:10CAD00035EC47E25EE30F94605060937508709305
:10CAE0007608809377089093780884E40E94073250
:10CAF000882381F00E94DD312CEA35EC47E25EE3C9
:10CB00000F94E6576093790870937A0880937B08B6
:10CB100090937C080E94504840917108509172088F
:10CB200060917308709174088DE791E10E94F73865
:10CB30002CEA35EC47E25EE3609175087091760867
:10CB400080917708909178080F94E657AB01BC016B
:10CB500089E791E10E94F7382CEA35EC47E25EE381
:10CB60006091790870917A0880917B0890917C0897
:10CB70000F946050AB01BC0185E791E10E94F7384A
:10CB80008AE00E94C93628C8873FA1E09A0711F4BD
:10CB90000C947C6F08F0B8C0853AE1E09E0711F470
:10CBA0000C94BF6EE8F48C3921E0920711F40C94D8
:10CBB0006C6E38F48A39914011F40C94EC5D0C944D
:10CBC000C55D8D39B1E09B0711F40C94F570843A82
:10CBD000914011F00C94C55D0E9468490C94EC5D85
:10CBE000843FF1E09F0711F40C94746F08F07DC04E
:10CBF0008C3A31E0930711F40C94C36E863E914059
:10CC000011F00C94C55D84E50E9407328823A1F0E1
:10CC10001092000510920105109202051092030572
:10CC2000109204058FEF0E94E82561E070E084E532
:10CC30000E94BB338093040583E50E94073288235A
:10CC400021F00E94D9310E94E82583E40E94073236
:10CC5000882331F080912302803210F40E948234C4
:10CC600080E50E940732882331F00E94D93180325A
:10CC700010F40E94823485E50E940732882311F463
:10CC80000C94EC5D0E94D931803210F00C94EC5D74
:10CC900041E050E060E070E0082E04C0440F551FF2
:10CCA000661F771F0A94D2F740955095609570954E
:10CCB00000910005109101052091020530910305B6
:10CCC00040235123622373234093000550930105B1
:10CCD00060930205709303059091230289130C94CD
:10CCE000EC5D10929B0F0C94EC5D853FB1E09B07CF
:10CCF00011F40C94786F863F914011F00C94C55D4F
:10CD00000E94A4FA0C94EC5D8E3BF2E09F0711F4B4
:10CD10000C94247060F5883532E0930711F40C947C
:10CD2000A06FB0F4883FB1E09B0711F40C94856FBD
:10CD30008C30924011F00C94C55D8091DC1582FD21
:10CD400002C00C94986F80648093DC150C94EC5DA9
:10CD50008B35F2E09F0711F40C94A46F8D3B924049
:10CD600011F00C94C55D0E94D4550C94EC5D873E87
:10CD700033E0930711F40C94E570C8F48C36B3E0FB
:10CD80009B0711F40C94EC5D803A934011F00C94E5
:10CD9000C55D2091F4043091F5049091DC1592600A
:10CDA0009093DC15C9010F9492400C94EC5D883E81
:10CDB000F3E09F0711F40C940E71893E934011F03B
:10CDC0000C94C55D0F94623F81110C94EC5D0E9440
:10CDD000DF330F94203F0E941DFC6D3371058105E8
:10CDE000910520F089E592E10E94957185E592E137
:10CDF0000E94957184EE8093FE0481E492E10E948A
:10CE000002378DE392E10E9495710C94EC5D60E035
:10CE100086E89FE00E9499B31ECA8091EC0484FDCD
:10CE200017C08091EE0487FD13C08091EF048370DA
:10CE300079F460E089E99FE00E9499B35F988A984D
:10CE40008091080181708093060112980C94EC5D2A
:10CE500088E50E94073281115F9889E50E940732B8
:10CE600081118A988AE50E940732882329F08091EF
:10CE7000080181708093060185E40E9407328823AF
:10CE800011F40C94EC5D12980C94EC5D8091DC151F
:10CE900083FF25C081EB9FE00E9402378091DC1563
:10CEA00083FF17C08BEF95E10E942ED38BE1EBEF50
:10CEB000F5E1DE01119601900D928A95E1F770E09F
:10CEC00060E0CE0101960F947806CE0101960E9493
:10CED000073482EA9FE00E9402370C94EC5D0E94C6
:10CEE000504882EC9FE00E9402370C94EC5D0F9456
:10CEF000523E0C94EC5D8091F4049091F504FC0199
:10CF00002191222331F02032D9F7DF0111971C92B1
:10CF1000F7CF60E00F94DB401092FE040C94EC5DC0
:10CF200083E50E945532882321F00E94A7270E94A2
:10CF3000DA2584E50E9455328823A9F00E94A727AC
:10CF40006B017C010E94C4FCC092BB05D092BC0561
:10CF5000E092BD05F092BE05CD28CE28CF2819F06D
:10CF600081E08093620880912B078823F9F080E0AC
:10CF700090E0A0EAB1E489839A83AB83BC831C8EE2
:10CF80001D8E1E8E1F8E18A219A21AA21BA210E0BF
:10CF900000E020E0AE014F5F5F4FBE01645E7F4F57
:10CFA000CE0180960E94CD560C94EC5D0E944D36C9
:10CFB000882381F00F94DB3D0E94713688ED98E064
:10CFC0000F94833D1092DF101092E0101092E11048
:10CFD0001092E21061E084E09EE10E94CA374CECBE
:10CFE0005DE16CEC7FE085E00F94942A0F941B4088
:10CFF0000C94EC5D8091DC1583FD02C00C94EC5D1B
:10D0000083E50E945532882311F40C94EC5D0E9454
:10D01000A7270E94DA250C94EC5D83E40E94073276
:10D02000882361F182EE9FE00E94023780914217CF
:10D030008823F9F0BE016F5F7F4F8FE397E10E9475
:10D04000F4D2CE0101960E9433CFCE0101960F9407
:10D05000BB3F80916A12882339F080E20E94C93672
:10D060008AE692E10E9433CF8AE00E94C9360C948E
:10D07000EC5D88ED9FE00E940237F6CF83E50E94C9
:10D080005532882301F10E94B531182F8C3308F0F6
:10D090008CE38093C7040F947E326B017C01212FB7
:10D0A00030E0A8EEB3E00F949256C60ED71EE81EED
:10D0B000F91EC092C304D092C404E092C504F09259
:10D0C000C6040C94EC5D0F944A3D0C94EC5D809189
:10D0D000F4049091F5040F9492400C94EC5D8091CF
:10D0E000DC158E7F8093DC150C94EC5D8091DC1553
:10D0F00082FD0E94FADC8091DC1583FD02C00C9455
:10D10000EC5D60E080E50E94CA33182F682F8091A3
:10D11000F4049091F5040F94DB4083E50E945532AE
:10D12000882321F00E94A7270E94DA250F94DB3D77
:10D1300011110C94EC5D0E9471360C94EC5D0E9410
:10D140001DFC6C8F7D8F8E8F9F8FBE016F5F7F4F19
:10D15000CE014C960E943B2CCE0101960F94E93FE4
:10D160000E945048BE016F5F7F4F81EF9FE00E9499
:10D17000664D8AE00E94C9360C94EC5D80E50E9401
:10D180000732882311F40C94EC5D0E94B53185368A
:10D1900008F084E68093FE040C94EC5D0E947136E6
:10D1A0000C94EC5D81E00E944FFC0C94EC5D8CE5EE
:10D1B00090E10E9402376091AC077091AD0783E562
:10D1C00090E10E94E5386091AE077091AF0786E468
:10D1D00090E10E94E5386091AC077091AD078091B5
:10D1E000AE079091AF07681B790B80916208815060
:10D1F00021E030E0823010F030E020E0621B730B61
:10D200008BE390E10E94E5388AE00E94C93683E30F
:10D2100090E10E9402378091B0079091B107A091F0
:10D22000B207B091B3078C8F9D8FAE8FBF8FBE01B9
:10D230006F5F7F4FCE014C960E943B2CBE016F5F0B
:10D240007F4F86E290E10E94664D8091B4079091F5
:10D25000B507A091B607B091B7078C8F9D8FAE8FA1
:10D26000BF8FBE016F5F7F4FCE014C960E943B2C5B
:10D27000BE016F5F7F4F86E190E10E94664D20E026
:10D2800030E04AE754E46091B8077091B9078091A3
:10D29000BA079091BB070F94E657AB01BC018EEF24
:10D2A0009FE00E94F7388DE60E94C9368AE00E940E
:10D2B000C9360C94EC5D80919C0F83FF02C00C94E6
:10D2C000EC5D0E94544887FF02C00C94EC5D89E439
:10D2D0000E945532882309F4BAC70E94B53190E004
:10D2E0001816190614F481E090E026E0289FF0015A
:10D2F000299FF00D1124EB5FF74F808191810E94EF
:10D300007CDC61E080E00F942A440F94F3430C949A
:10D31000EC5D84E690E1112309F494C9012FA1C9C1
:10D32000182F9FC90E945448182F87FD0AC08FE705
:10D3300090E10E940237812F0F9403088AE00E9437
:10D34000C93638A930934D08E1960FB6F894DEBF80
:10D350000FBECDBFDF91CF911F910F91FF90EF9046
:10D36000DF90CF90BF90AF909F908F907F906F9005
:10D370005F904F903F902F90089580E50F949D2AE5
:10D38000823010F00C94EC5DE82FF0E0EA57F64F95
:10D3900010820C94EC5D8EE40E945532882311F4C7
:10D3A0000C94EC5D0E94A72760937810709379101D
:10D3B00080937A1090937B100C94EC5D83E50E942F
:10D3C0000732882329F083E50F949D2A80939C0FD0
:10D3D0000E94504880E990E10E94023780919C0FA2
:10D3E000882351F110E000E020E080919C0F90E054
:10D3F000B0E0A0E0002E04C0B695A795979587955C
:10D400000A94D2F780FF12C0FF24F394F20E222375
:10D4100019F08CE20E94C936F801EE0FFF1FEA579F
:10D42000FF4E859194910E9402372F2D0F5F1F4F61
:10D4300005301105D1F618CE82E890E11CCE83E5C7
:10D440000E945532882369F00E94B5318D3320F453
:10D4500080930F020C94EC5D8CE380930F020C948C
:10D46000EC5D0E94504860910F0287E990E10E94B4
:10D47000EF388AE00E94C9360C94EC5D80919C0FD5
:10D4800083FF02C00C94EC5D89E40E94553288232E
:10D4900009F403C70E94B53190E01816190614F478
:10D4A00081E090E026E0289FF001299FF00D1124F3
:10D4B000EB5FF74F828193810E94AA3161E080E0A7
:10D4C0000F942A440C94EC5D80919C0F83FF02C062
:10D4D0000C94EC5D89E40E945532882309F4E7C678
:10D4E0000E94B53190E01816190614F481E090E01E
:10D4F00026E0289FF001299FF00D1124EB5FF74FE4
:10D500008281938110E00E94AA3160E081E00F9453
:10D510002A4420916E0830916F0880916C08909198
:10D520006D08821793071CF48DEA90E102C08EE922
:10D5300090E160E00E9499B360E0812F0F9476083B
:10D540000C94EC5D83E50E945532882311F40C9411
:10D55000EC5D0E94B531182F8C3308F08CE380937A
:10D56000CC040F947E326B017C01212F30E0A8EEB9
:10D57000B3E00F949256C60ED71EE81EF91EC09255
:10D58000C804D092C904E092CA04F092CB040C946F
:10D59000EC5D0E944BD50E940BDD81E00E944FFCA8
:10D5A0000E94843668EE73E080E090E00E94FE35D1
:10D5B0000E94492260E08CEB90E10E9499B30C94A8
:10D5C000EC5D809163088F7D8061809363080C948B
:10D5D000EC5D8091EC0484FD0CC08091EE0487FD2D
:10D5E00008C08091EF04837021F40E940BDD0C943D
:10D5F000EC5D0E94FADC88E50E940732882331F056
:10D600005F9A8091BF078E7F8093BF0789E50E9454
:10D610000732882331F08A9A8091BF078D7F8093EB
:10D62000BF078AE50E940732882359F080910801DC
:10D6300080958170809306018091BF078B7F8093D6
:10D64000BF0785E40E940732882311F40C94EC5D37
:10D650000E9447220C94EC5D83E50E9407328823E8
:10D6600011F40C94EC5D0F947E326093410870933A
:10D67000420880934308909344080E94DD3120E0E3
:10D6800030E04AE754E40F9460500F945F58609381
:10D69000CD047093CE048093CF049093D0040C9467
:10D6A000EC5D0E94DD31F701648B758B868B978B67
:10D6B0000C948D6281E00F9427290C94EC5D0F94FB
:10D6C000C22884E495E10E9418D80C94EC5D809106
:10D6D000F4049091F504009741F0DC012C91222391
:10D6E00021F00F94E93F0C94EC5D0F941B400C94D7
:10D6F000EC5D0091F4041091F50494E0F12C40E00D
:10D700009150F9F0F8018081282F2B7F213499F472
:10D7100021812133B1F4813411F1853409F441E0E0
:10D7200098012E5F3F4F89012F5F3F4FF8018081A5
:10D730008032C9F3E5CF803521F4818180538A306E
:10D7400078F341110E945048FF2021F08DEC90E1C8
:10D750000E940237C8010E94D0360C94EC5DFF2471
:10D76000F394DECF1093BD071093BC070E9499FA83
:10D770000C94EC5D8C01112788E40E9455328823BB
:10D78000C1F00E94D9318A3A91050CF44BC00E9435
:10D79000D9318D3291400CF048C00E94D93126E039
:10D7A000209FF001219FF00D1124EB5FF74F918333
:10D7B000808382E40E9455328823A9F00E94D931E7
:10D7C0000597B4F10E94D9318D389105A4F50E94D6
:10D7D000D93126E0209FF001219FF00D1124EB5F4D
:10D7E000F74F9383828386E40E945532882311F495
:10D7F0000C94EC5D0E94D93197FD20C00E94D93174
:10D800008F3F910509F0ECF40E94D93126E0209F6A
:10D81000F001219FF00D1124EB5FF74F9583848376
:10D820000C94EC5D8AEA90E0BACF8CE291E0B7CF3D
:10D8300085E090E0CECF8CE890E0CBCF90E080E028
:10D84000E5CF8FEF90E0E2CF80E00C94D6630E94AA
:10D85000544887FF02C00C94EC5D0BE912E08DE99F
:10D86000E82E8FE0F82E9FE9C92E92E0D92ED8013C
:10D870008D918D010E940732882359F00E94DD317D
:10D880000F945F58F70160837183828393830E94B2
:10D8900088DCF4E0EF0EF11CC016D10641F70C94C1
:10D8A000EC5D0E94544887FF02C00C94EC5DBBE91C
:10D8B000EB2EB2E0FB2E10E000E0D7018D917D0150
:10D8C0000E940732882349F00E94DD31F801E356B7
:10D8D000F04F64A375A386A397A30C5F1F4F00317D
:10D8E000110559F70C94EC5D83E50E9455328823AD
:10D8F00091F00E94DD316093D10F7093D20F80932D
:10D90000D30F9093D40F6093D90F7093DA0F809355
:10D91000DB0F9093DC0F80E50E945532882351F095
:10D920000E94DD316093D10F7093D20F8093D30F9B
:10D930009093D40F82E50E945532882351F00E94C3
:10D94000DD316093D50F7093D60F8093D70F9093EE
:10D95000D80F84E50E945532882311F40C94EC5DB5
:10D960000E94DD316093D90F7093DA0F8093DB0F43
:10D970009093DC0F0C94EC5D8091EC04827151F477
:10D980008091EE048C7831F48091EF04837011F46F
:10D990000C94EC5D82E40E940732882351F00E94CF
:10D9A00086276093AD0F7093AE0F8093AF0F909367
:10D9B000B00F83E50E940732882351F00E94DD31C9
:10D9C0006093DD0F7093DE0F8093DF0F9093E00F75
:10D9D00084E50E940732882351F00E94DD31609374
:10D9E000E10F7093E20F8093E30F9093E40F88E5CB
:10D9F0000E940732882351F00E94DD3160935E0956
:10DA000070935F09809360099093610989E50E9492
:10DA10000732882351F00E94DD31609362097093D0
:10DA2000630980936409909365098AE50E9407322F
:10DA30008823B1F00E94DD31609366097093670915
:10DA400080936809909369092DEC3CEC4CEC5DE304
:10DA50000F94FA4F181624F085E091E10E940237E6
:10DA600085E40E940732882311F40C94EC5D0E9437
:10DA7000DD3160936A0970936B0980936C09909310
:10DA80006D090C94EC5D0E9479480C94EC5D82E485
:10DA90000E940732882341F080916E0290916F02BC
:10DAA000909315028093140282E50E940732882326
:10DAB00041F0809114029091150290936F0280932F
:10DAC0006E0283E50E945532882331F00E94D931DD
:10DAD00090936F0280936E028091EC049091ED041C
:10DAE000A091EE04B091EF04892B8A2B8B2B11F0BF
:10DAF0000C94EC5D60916E0270916F028EE391E187
:10DB00000E940D3E85E20E94C9368AE00E94C93615
:10DB10000C94EC5D0E94504885E40E94C93680E375
:10DB2000800F0E94C936F701EB5CFD4F6081718167
:10DB300082E491E10E940D3E85E20E94C9368AE0AE
:10DB40000E94C9360C94EC5D8AE50E945532882308
:10DB500031F10E94DD3120E030E040E050EC0F94E4
:10DB6000FA4F87FD3CC00E94DD3120E030E040E00C
:10DB700050E40F944C591816BCF10E94DD312091ED
:10DB8000B90F3091BA0F4091BB0F5091BC0F0F9459
:10DB900060500F945858CB010F94323305C083E581
:10DBA0000E9455328111D5CF8091EE0487FD21C0AE
:10DBB0008091EF048370E9F40E9450484091300650
:10DBC0005091310660913206709133068AE491E1FA
:10DBD0000E94F7388AE00E94C9360C94EC5D60E040
:10DBE00070E080E090ECCBCF60E070E080E090E40B
:10DBF000C6CF82E50E9407328111DECF0C94EC5D26
:10DC000064E071E083E50E9462328C0168EE73E0AB
:10DC100080E50E9462328938F3E19F0710F088E8BE
:10DC200093E1B8010E94847E0C94EC5D0E946747EA
:10DC300083E691E10E9402370C94EC5D83E50E943B
:10DC40000732182F882369F00E94D9319C019093E4
:10DC50007E0280937D0291E0232B09F090E0909367
:10DC6000980980E50E940732882361F020917D02A7
:10DC700030917E02232B11F00E94C93180939809C4
:10DC80000C94EC5D11110C94EC5D0E9450488DE9F0
:10DC900091E10E94023780919809882391F085E8EC
:10DCA00091E10E94023760917D0270917E028CE8C2
:10DCB00091E10E940D3E88E891E10E9402370C94A8
:10DCC000EC5D81E891E1EDCF0E9419390C94EC5D97
:10DCD0000E94FADC0C94EC5D8091EC048878F9F4F5
:10DCE0008091EE048670D9F40E94504880ED91E155
:10DCF0000E940237809155020E94D938409151020A
:10DD000050915202609153027091540280EB91E164
:10DD10000E94F7388AE00E94C9360C94EC5D88E4D2
:10DD20000E940732882321F00E94C9318093D104D8
:10DD300082E50E940732082F83E50E940732182FE0
:10DD4000011102C0882341F00E943422112321F0E6
:10DD50000E94C9318093550284E40E9407328823CF
:10DD600011F40C94EC5D0E94DD31609351027093CC
:10DD7000520280935302909354020C94EC5D0E94E3
:10DD80006B470C94EC5D0F943D4081110C94EC5D5D
:10DD90007BE8C72E77E2D72E26EE3FE03DA32CA3EB
:10DDA000CE0101961C017C0110E000E0F6016591B6
:10DDB000759185919491ACA1BDA18D909D90AD90F0
:10DDC000BD90BDA3ACA3A50194010F94EB562B010C
:10DDD0003C01F701408251826282738220E030E090
:10DDE00040EA51EC0F944C5987FD0AC020E030E026
:10DDF00040EA51E4C301B2010F94FA4F181684F4BB
:10DE0000F801EE5DFF4BE4911E1654F4B7FAB0949E
:10DE1000B7F8B094D7018D929D92AD92BC921397B2
:10DE2000F70181909190A190B1907F0120E030E0C6
:10DE300040EA51ECC501B4010F944C5987FD3FC035
:10DE400020E030E040EA51E4C501B4010F94FA4FFC
:10DE50001816ACF10F5F1F4FF4E0CF0ED11C03304A
:10DE6000110509F0A3CF6EE8E62E68E0F62E10E06B
:10DE7000F10181919191A191B1911F01F7018193DC
:10DE80009193A193B1937F01812F0E94D8EE1F5FE0
:10DE9000133071F70E9490F960E081EE91E10E94E9
:10DEA00099B363E972E084E690E00E94847E6AEBB5
:10DEB00072E084E690E00E94847E0C94EC5D0E9407
:10DEC00067478FEF91E10E94023761E081EF91E1B6
:10DED0000E9499B30E94F08468E270E088EC90E0C0
:10DEE0000E94847E0C94EC5D0E94CAD80C94EC5D78
:10DEF0000F94A5120C94EC5D61E083E50E94CA3397
:10DF000081270F94890B0C94EC5D81E0809334069B
:10DF10000F94991210923406882311F40C94EC5D3E
:10DF20000E9450488DE192E10E9402370C94EC5D12
:10DF300083FD02C00C94EC5D0F9462290C94EC5D9F
:10DF40000E94645A0C94EC5D0E945448082F87FF8D
:10DF500002C00C94EC5D85E50E940732882359F1DC
:10DF60000E94DD314B015C01E02E002E000CFF0809
:10DF700020E030E0A9010F944C5987FF04C0B7FAA4
:10DF8000B094B7F8B09420E030E84BE354E4C50116
:10DF9000B4010F944C59970153E0220F331F5A9547
:10DFA000E1F72D533A4F1816D4F1D9018D929D9275
:10DFB000AD92BC9213978CE40E940732882311F42F
:10DFC0000C94EC5D0E94DD316B017C01002E000C95
:10DFD000110B20E030E0A9010F944C5987FF04C0D9
:10DFE000F7FAF094F7F8F09420E030E84BE354E4CB
:10DFF000C701B6010F944C59980143E0220F331F1B
:10E000004A95E1F72D533A4F18169CF0D901149612
:10E01000CD92DD92ED92FC9217970C94EC5D80E02E
:10E0200090E8ABE3B4E4F90180839183A283B383E6
:10E03000C2CF80E090E8ABE3B4E4F9018483958338
:10E04000A683B7830C94EC5D0E945448182F87FF79
:10E0500002C00C94EC5D8AE50E945532812C912C13
:10E0600090E2A92E91E4B92E882341F040E050E0DF
:10E07000BA018AE50E9470324B015C01412F64E0D5
:10E0800083E00E94D98520E030E0A901C501B401F8
:10E090000F944C5918167CF580E090E0A0EAB0E4AB
:10E0A00089839A83AB83BC832091EE0F3091EF0F6D
:10E0B0004091F00F5091F10FC501B4010F94EC564F
:10E0C0006B017C0120E030E048EC53E40F94FA4F00
:10E0D00087FD06C0C12CD12C88ECE82E83E4F82EF5
:10E0E000CC8EDD8EEE8EFF8EBE016F5F7F4FCE0138
:10E0F0004C960E9499F085E50E940732882309F426
:10E1000059C00E94DD316B017C0120E030E0A901A3
:10E11000C701B6010F944C5987FF04C0F7FAF09479
:10E12000F7F8F094F7FAF094F7F8F094C982DA82ED
:10E13000EB82FC8244E061E0CE0101960E943B58F4
:10E1400020E030E0A901C501B4010F944C59181624
:10E150005CF580E090E0A0EAB0E489839A83AB8329
:10E16000BC83A50194016091EE0F7091EF0F809137
:10E17000F00F9091F10F0F94EB566B017C0120E0B2
:10E1800030E0A9010F944C5918161CF0C12CD12C69
:10E190007601CC8EDD8EEE8EFF8EBE016F5F7F4FDF
:10E1A000CE014C960E9499F0109206050E94F084D0
:10E1B0000C94EC5D28E01202F0011124ED53FA4FAB
:10E1C000C080D180E280F380A0CF81E080930408FA
:10E1D0001092021360E083E50E94CA3381110C940F
:10E1E000EC5D0F9469270C94EC5D83E50E94073287
:10E1F000882341F00E94C9318093CB050E94E73308
:10E200000C94EC5D0E94504888E292E10E94023733
:10E210008091CB050E94D9380C94EC5D0E94077266
:10E220000C94EC5D1091F1040F947E3260934108E0
:10E23000709342088093430890934408112311F48B
:10E240000C94EC5D812F0E9401D50C94EC5D83E56C
:10E250000E945532882309F458C80E94D9314FC80A
:10E2600083E50E945532182F811107C082E50E9474
:10E270005532082F882309F453C80E94D9310C94D1
:10E280000E6383E50E945532882311F40C94CB620F
:10E290000E94A7278B010C94CB6283E50E94553224
:10E2A000882311F40C94EC5D0E94D93105C983E5F3
:10E2B0000E945532182F811107C082E50E94553205
:10E2C000882311F40C94EC5D0E94D9311CC9DF92B3
:10E2D000EF92FF920F931F93CF93DF93EC01E090A7
:10E2E0004F08F09050088AE0D82E6AE070E0CE0126
:10E2F0000F94415A8C01009711F0FC011082CE015D
:10E300000E941A2D81E00E94545C0115110519F03C
:10E31000E801D992EACFC701DF91CF911F910F9108
:10E32000FF90EF90DF900C941A2D4F925F926F92B6
:10E330007F928F929F92AF92BF92CF92DF92EF9295
:10E34000FF920F931F93CF93DF93CDB7DEB77C017E
:10E350004DB65EB660904F08709050088DB69EB670
:10E360006AE070E0C7010F94354F6C018C010E1903
:10E370001F09892B21F4C7010F94474F8C01C80155
:10E3800001962DB73EB7281B390B0FB6F8943EBF48
:10E390000FBE2DBF8DB79EB701965C01A801B701D6
:10E3A0000F94684FF501E00FF11F1082C5010E9424
:10E3B0001A2D81E00E94545CC114D10451F0760101
:10E3C0009FEFE91AF90A0FB6F8949EBE0FBE8DBEF4
:10E3D000C5CF0FB6F8949EBE0FBE8DBEC3010E947E
:10E3E0001A2D0FB6F8945EBE0FBE4DBEDF91CF91D1
:10E3F0001F910F91FF90EF90DF90CF90BF90AF9063
:10E400009F908F907F906F905F904F9008954F9264
:10E410005F926F927F928F929F92AF92BF92CF92B4
:10E42000DF92EF92FF920F931F93CF93DF93CDB7BD
:10E43000DEB7C059D1090FB6F894DEBF0FBECDBF0D
:10E440000E94F533882369F083E50E940732882310
:10E4500001F120E040E070E060E08AE195E80E9490
:10E460008A81C057DF4F0FB6F894DEBF0FBECDBF15
:10E47000DF91CF911F910F91FF90EF90DF90CF90A0
:10E48000BF90AF909F908F907F906F905F904F90D4
:10E49000089583E40E940732882319F00E940F85B3
:10E4A000E0CF8090410990904209A0904309B0903C
:10E4B000440980914A0980FF05C090919C0F9860A3
:10E4C00090939C0F869581708093980980E29FE0DD
:10E4D0000E9495718091D0089091D1089E012F5F84
:10E4E0003F4F7901009799F09F938F9387E19FE0C9
:10E4F0009F938F933F932F930F94914FC7010E9447
:10E5000067710F900F900F900F900F900F90809168
:10E51000CE089091CF08009799F09F938F938EE04B
:10E520009FE09F938F93FF92EF920F94914FC701BB
:10E530000E9467710F900F900F900F900F900F90A7
:10E540006E0131E8C30ED11C6091AD087091AE0828
:10E550008091AF089091B008860123E041E00F94CC
:10E56000C74A9F938F938CEF9EE09F938F93FF9268
:10E57000EF920F94914FC7010E94677184EF9EE064
:10E580000E94957187E08093BF078093AE050F903E
:10E590000F900F900F900F900F908091C9088823D3
:10E5A000F9F06091CA087091CB088091CC089091E5
:10E5B000CD0823E041E00F94C74A9F938F938BEEE1
:10E5C0009EE09F938F93FF92EF920F94914FC7011C
:10E5D0000E9467710F900F900F900F900F900F9007
:10E5E0008091D2088823A1F01F928F931F921F92CF
:10E5F0008EED9EE09F938F93FF92EF920F94914F39
:10E60000C7010E9467710FB6F894DEBF0FBECDBF81
:10E610008091D3088823A9F01F928F931F9281E0E5
:10E620008F938EED9EE09F938F93FF92EF920F94C6
:10E63000914FC7010E9467710FB6F894DEBF0FBEFD
:10E64000CDBF4090D4085090D5086090D608709007
:10E65000D70820E030E0A901C301B2010F94FA4FBE
:10E66000811104C080914A0982FF20C0860121E007
:10E6700041E0C301B2010F94C74A9F938F938091E9
:10E680004A0982FB882780F91F928F9381ED9EE0D3
:10E690009F938F93FF92EF920F94914FC7010E9427
:10E6A00067710FB6F894DEBF0FBECDBF60919F08B3
:10E6B0007091A0088091A1089091A2088E010F5836
:10E6C0001F4F23E041E00F94C74A782E692E6091D6
:10E6D0009B0870919C0880919D0890919E088601EE
:10E6E00023E041E00F94C74A6F927F929F938F93EC
:10E6F00080EC9EE09F938F93FF92EF920F94914F47
:10E70000C7010E9467716091A3087091A40880916D
:10E71000A5089091A60823E041E00F94C74A85EB35
:10E720009EE00E949571DF92CF928BEA9EE09F93CC
:10E730008F93FF92EF920F94914FC7010E946771E0
:10E740008091AC088F938091AB088F9384EA9EE010
:10E750009F938F93FF92EF920F94914FC7010E9466
:10E7600067716091A7087091A8088091A90890919D
:10E77000AA0823E041E00F94C74A9F938F938AE948
:10E780009EE09F938F93FF92EF920F94914FC7015A
:10E790000E9467718CE0E1EBF8E0AEE8B8E0019030
:10E7A0000D928A95E1F78CE0EDEBF8E0A2E8B8E095
:10E7B00001900D928A95E1F780E00E94D8EE81E009
:10E7C0000E94D8EE82E00E94D8EE809149098093A1
:10E7D000630881E08093CB050E94E73388ED98E0E1
:10E7E0009F938F9387EB97E39F938F93FF92EF9283
:10E7F0000F94914F0FB6F894DEBF0FBECDBFC70187
:10E800000E946771809148098F93809147098F9387
:10E81000809146098F93809145098F93BF92AF9263
:10E820009F928F928CE89EE09F938F93FF92EF923E
:10E830000F94914FC7010E9467710FB6F894DEBF25
:10E840000FBECDBF0ECE4F925F926F927F928F928E
:10E850009F92AF92BF92CF92DF92EF92FF920F936F
:10E860001F93CF93DF9300D000D01F921F92CDB79C
:10E87000DEB783E50F949D2A863028F083E19EE081
:10E880000E9402373FC0833009F464C1B0F4813084
:10E8900021F1823009F450C080E09EE00E940237EE
:10E8A0000E94B9358823A1F08091E50F0E94D938E4
:10E8B0000E945A380E9490F925C0843009F490C112
:10E8C000853051F780E00E94BE340E94AE34F2CF12
:10E8D00082EF9DE00E940237EDCF0E94AE3410928D
:10E8E0000E0210920D028091FF04811125C08EE46A
:10E8F0000E94073281111DC080EE9DE09093C207F7
:10E900008093C10728960FB6F894DEBF0FBECDBF27
:10E91000DF91CF911F910F91FF90EF90DF90CF90FB
:10E92000BF90AF909F908F907F906F905F904F902F
:10E93000089586EE9DE0E2CF80910D0290910E0247
:10E9400097FF03C087EB9DE09BCF009709F0A8C01D
:10E950001D821E821F8218868DEC9CECACE4BEE307
:10E9600089839A83AB83BC83BE016B5F7F4FCE01EB
:10E9700001960E9499F080910D0290910E028931CA
:10E9800091050CF0B3C021E0209338029C012F5F69
:10E990003F4F30930E0220930D0265E00F94AD5669
:10E9A00080FF03C024E0291B922F24E09202F00193
:10E9B0001124E354FA4E80809180A280B38094E0C9
:10E9C0008902F0011124E755FA4E4080518062809F
:10E9D00073808DEC9CECACE4BEE38D839E83AF83AF
:10E9E000B88719821A821B821C82CE0101966C01A3
:10E9F000E12CF12C00EA10E4A3019201C501B4015D
:10EA00000E94E1EF19821A821B821C82B601CE019C
:10EA100005960E9499F08092E60F9092E70FA092DF
:10EA2000E80FB092E90F4092EA0F5092EB0F60921C
:10EA3000EC0F7092ED0F1092FF0400910D021091F7
:10EA40000E0289E1E82EF12C093111050CF4780150
:10EA5000B70180E59DE00E940D3E69E170E08BE426
:10EA60009DE00E940D3E8AE00E94C93610161106F4
:10EA70000CF020CF1F9289E18F93FF92EF9284E3F5
:10EA80009DE09F938F9382E49DE09F938F931F92CD
:10EA90000E947EB30FB6F894DEBF0FBECDBF0ACF83
:10EAA000815065E00F94AD5680FF03C024E0291B20
:10EAB000922F25E09202F0011124E80FF11D87FD4D
:10EAC000FA95EE0FFF1FEE0FFF1FE453FA4F8091F0
:10EAD000EE0F9091EF0FA091F00FB091F10F8083A6
:10EAE0009183A283B3831092380245CF80E090E0F7
:10EAF000A0EAB0E48093EE0F9093EF0FA093F00F95
:10EB0000B093F10F84E792E00E94C6EF0E94FADC16
:10EB10008FEF9FEF90930E0280930D0283EA9DE0AA
:10EB20000E94023781E99DE00F94E93F63E972E0BA
:10EB300084E690E00E94847E6AEB72E084E690E0D6
:10EB40000E94847E8BE89DE00E94957181E00E9486
:10EB5000BE3471CF89E40E945532882371F00E943F
:10EB6000D931182F853068F064E070E088E79DE0C7
:10EB70000E940D3E85E79DE083CE8AE40E94C43763
:10EB8000C1CE8AE40E9455328823B9F30E94D9315C
:10EB9000082F853048F064E070E082E69DE00E9436
:10EBA0000D3E8FE59DE06CCE8AE50E9455328823AC
:10EBB000A9F00E94DD3125E01202F0011124E00FDE
:10EBC000F11D07FDFA95EE0FFF1FEE0FFF1FE45337
:10EBD000FA4F60837183828393836CCE8AE5CECFB4
:10EBE0008AE50E9455328823C9F30E94DD31609383
:10EBF00030067093310680933206909333065ACED6
:10EC0000CF93DF93C091E410C0935D0981E6C89F64
:10EC1000E0011124CA51DF4E80919C0F80FF05C096
:10EC20000E945048CE010E94D036CE010E941A2D7B
:10EC300080E0DF91CF910C94545C6091350270912B
:10EC40003602072E000C880B990B0F9401502AE016
:10EC500037ED43E25CE30F9460502091B7053091AB
:10EC6000B8054091B9055091BA050F946050609372
:10EC7000790270937A0280937B0290937C020895CC
:10EC8000E0912C08E23030F4F0E0EA57F64F809142
:10EC90002208808308958091D1158823C1F0815086
:10ECA0008093D115EBEFF5E1882351F08150990B5A
:10ECB0002BE1289FF001299FF00D1124EF5CF94E04
:10ECC0008BE1A6E1B6E101900D928A95E1F72091E2
:10ECD000D115211105C08091DC1580628093DC156F
:10ECE00081E090E0A0E0B0E0211103C080E090E07E
:10ECF000DC0180931A0890931B08A0931C08B09322
:10ED00001D0810921F0881E08093190883E080930A
:10ED100078020895CF93DF93EC01CB01BA010F94F1
:10ED2000015029EC38EC48EC5EE30F94E65720E004
:10ED300030E040E05FE30F94EC560F945F58688337
:10ED4000DF91CF910895E0912C0886E0E802F00170
:10ED50001124EB5FF74F8091220890E09583848324
:10ED60000895CF93DF93EC01CB01BA010F940150CA
:10ED700020E030E0A9010F94EC560F945F586883AF
:10ED8000DF91CF9108958F929F92AF92BF92CF92D1
:10ED9000DF92EF92FF92CF936B017C0120E030E095
:10EDA000A9010F94FA4F87FD9FC06DEB77E386E0D2
:10EDB00095E3A70196010F94EC566B017C0120E0CE
:10EDC00030E040E251E40F94605020E030E048EC45
:10EDD00052E40F9460504B015C0120E030E0A90147
:10EDE000C701B6010F94FA4F20E030E040EA50E44A
:10EDF00087FF04C020E030E040EA50ECC501B401D8
:10EE00000F94EC5620E030E040E251E40F94E657D6
:10EE10000F9458586B017C018BE2F7FE09C0F09407
:10EE2000E094D094C094C11CD11CE11CF11C8DE273
:10EE30008093A605C701B60120E137E240E050E02B
:10EE40000F9460568AE0882E912CA12CB12CCA0117
:10EE5000B901A50194010F946056605D6093A70508
:10EE6000C701B60128EE33E040E050E00F94605651
:10EE7000CA01B901A50194010F946056605D6093C9
:10EE8000A805C701B60124E630E040E050E00F9449
:10EE90006056CA01B901A50194010F946056605DE6
:10EEA0006093A9058EE28093AA05C701B601A5016A
:10EEB00094010F946056C62FCA01B901A5019401AF
:10EEC0000F946056605D6093AB05C05DC093AC0568
:10EED00086EA95E0CF91FF90EF90DF90CF90BF90C2
:10EEE000AF909F908F9008956DEB77E386E095EB60
:10EEF00060CF8F929F92AF92BF92CF92DF92EF92AC
:10EF0000FF92CF936B017C0120E030E0A9010F94C8
:10EF1000FA4F87FDAAC06DEB77E386E095E3A70182
:10EF200096010F94EC566B017C0120E030E0A901C2
:10EF30000F94FA4F87FF9EC0C701B601905820E09A
:10EF400030E040E251E40F94605020E030E040E2D5
:10EF500051E40F94605020E030E040EA50E40F9418
:10EF6000EC5620E030E040E251E40F94E6570F9475
:10EF700058586B017C0180E28093A60560E280E135
:10EF8000C81687E2D806E104F1048CF0C701B60187
:10EF900020E137E240E050E00F946056CA01B90129
:10EFA0002AE030E040E050E00F946056605D6093EE
:10EFB000A70560E288EEC81683E0D806E104F104F4
:10EFC0008CF0C701B60128EE33E040E050E00F942A
:10EFD0006056CA01B9012AE030E040E050E00F94E9
:10EFE0006056605D6093A80560E284E6C816D104AF
:10EFF000E104F1048CF0C701B60124E630E040E002
:10F0000050E00F946056CA01B9012AE030E040E0B8
:10F0100050E00F946056605D6093A9058AE0882EE9
:10F02000912CA12CB12CC701B601A50194010F941C
:10F030006056C62FCA01B901A50194010F9460560C
:10F04000605D6093AA058EE28093AB05C05DC093BE
:10F05000AC0586EA95E0CF91FF90EF90DF90CF90DE
:10F06000BF90AF909F908F9008956DEB77E386E00F
:10F0700095EB55CF20E030E040E251E4C701B60106
:10F0800062CFCF93DF93EC01CB01BA010F94015013
:10F0900020E030E040E251E40F94E65720E030E019
:10F0A000A9010F94EC56688379838A839B83DF914F
:10F0B000CF910895CF93DF93EC01CB01BA010F9468
:10F0C000015020E030E040E251E40F94E65720E0A8
:10F0D00030E0A9010F94EC56688379838A839B837F
:10F0E000DF91CF9108950F94015020E030E040E28D
:10F0F00051E40F94E65720E030E0A9010F94EC565C
:10F100000C947977CF93DF93EC01CB01BA010F9484
:10F1100001502AE037ED43E25DE30F94E65720E02B
:10F1200030E0A9010F94EC560F945F5868837983FF
:10F130008A839B83DF91CF910895CF93DF93EC0176
:10F14000CB01BA010F9401502AE037ED43E25DE3B1
:10F150000F94E65720E030E0A9010F94EC56688345
:10F1600079838A839B83DF91CF910895CF93DF9337
:10F17000EC01CB01BA010F94015020E030E0A9016D
:10F180000F94EC56688379838A839B83DF91CF91B8
:10F190000895CF93DF93EC01CB01BA010F94015096
:10F1A00020E030E0A9010F94EC56688379838A83CC
:10F1B0009B83DF91CF910895CF93DF93EC01CB0137
:10F1C000BA010F94015020E030E048EC52E40F9473
:10F1D000E65720E030E0A9010F94EC56688379836C
:10F1E0008A839B83DF91CF910895CF93DF93EC01C6
:10F1F000CB01BA010F94015020E030E048EC52E41A
:10F200000F94E65720E030E0A9010F94EC56688394
:10F2100079838A839B83DF91CF9108950F94015066
:10F2200020E030E048EC52E40F94E65720E030E074
:10F23000A9010F94EC560C94C376CF93DF93EC01A5
:10F24000CB01BA010F94015020E030E0A9010F94E6
:10F25000EC560F94585879836883DF91CF910895C5
:10F26000CF93DF93EC01CB01BA010F94015020E062
:10F2700030E0A9010F94EC56688379838A839B83DD
:10F28000DF91CF910895CF93DF93EC01CB01BA01C9
:10F290000F94015020E030E04AE754E40F94E65721
:10F2A00020E030E0A9010F94EC56688379838A83CB
:10F2B0009B83DF91CF9108952CEA35EC47E25EE322
:10F2C00060919405709195058091960590919705B0
:10F2D0000F94E6576093291570932A1580932B1588
:10F2E00090932C1508952CEA35EC47E25EE360918B
:10F2F00098057091990580919A0590919B050F94BE
:10F300006050609325157093261580932715909370
:10F31000281508952CEA35EC47E25EE360919405E8
:10F320007091950580919605909197050F94E657F9
:10F330006093291570932A1580932B1590932C15A3
:10F3400008952CEA35EC47E25EE3609198057091F0
:10F35000990580919A0590919B050F946050609358
:10F3600025157093261580932715909328150895D9
:10F370008091220890912308A0912408B09125083B
:10F380008093510290935202A0935302B09354027F
:10F390000895E0918D05E63010F581E08E0F8093A1
:10F3A0008D0540911A0850911B0860911C087091BE
:10F3B0001D0890911F088091180828E0E29FF00135
:10F3C0001124E25BFA4F2091681530916915318361
:10F3D0002083428353836483758396838783089550
:10F3E000FC01A081B1811C92A281B3818C918F5FBD
:10F3F0008C930280F381E02D90818CE0989F800DAA
:10F400001124EAE6F5E113AE84AF0895CF92DF92BE
:10F41000EF92FF92CF93DF9300D01F92CDB7DEB76C
:10F420006B017C0120E030E0A9010F94FA4F87FDC9
:10F430001CC06DEB77E386E095E3A70196010F947E
:10F44000EC5669837A838B839C8360E2CE010196BC
:10F450000E94AFFD0F900F900F900F90DF91CF9112
:10F46000FF90EF90DF90CF9008956DEB77E386E00B
:10F4700095EBE3CF0F94015020E030E04AE754E4ED
:10F480000F94E65720E030E0A9010F94EC560C945D
:10F49000067ACF92DF92EF92FF926B017C0120E01F
:10F4A00030E0A9010F94FA4F87FD26C06DEB77E39A
:10F4B00086E095E3A70196010F94EC566B017C0161
:10F4C00020E030E0A9010F94FA4F20E030E040E066
:10F4D0005FE387FF04C020E030E040E05FEBC7015E
:10F4E000B6010F94EC560F945858CB01FF90EF9053
:10F4F000DF90CF900D94AB006DEB77E386E095EB5A
:10F50000D9CF0F94015020E030E0A9010F94EC56C0
:10F510000C94497A0F94015020E030E0A9010F9437
:10F52000EC560F945858CB010D94AB000F9401503A
:10F5300029EC38EC48EC5EE30F94E65720E030E02D
:10F5400040E05FE30F94EC560F945F58862F0D94C4
:10F5500002010D948A320D948A326FEF8091220855
:10F560000D94A83061E473EB82E00D94CF4166E422
:10F5700073EB81E00D94CF416BE473EB80E00D946D
:10F58000CF416CEF70EB83E00D94CF41CF92DF92CF
:10F59000EF92FF92CF93DF9300D01F92CDB7DEB7EB
:10F5A0006B017C0120E030E0A9010F94FA4F87FD48
:10F5B0001BC06DEB77E386E095E3A70196010F94FE
:10F5C000EC5669837A838B839C83CE0101960E94DB
:10F5D0004BFE0F900F900F900F90DF91CF91FF9007
:10F5E000EF90DF90CF9008956DEB77E386E095EB99
:10F5F000E4CF0F94015020E030E040E251E40F945A
:10F60000E65720E030E0A9010F94EC560C94C67A3E
:10F610008091421590914315891B8F7011F40C94C1
:10F62000223681E0089580917802882351F060911C
:10F6300092057091930530E020E041E081E00C9468
:10F640007B2A089584E00D947B2F83E00D947B2F1B
:10F6500082E00D947B2F0F94015020E030E0A9014F
:10F660000F94EC560F945F58862F0D94E000909104
:10F67000E50F81E089270C94BE3461E082E298E0D6
:10F680000C94D9340F94AA270C94E8F080E090E011
:10F69000A0E8B0E48093EE0F9093EF0FA093F00FEB
:10F6A000B093F10F87ED92E00E94C6EFE0919D05C7
:10F6B00080E090E0A6E1B3E4E43009F44AC080E0E1
:10F6C00090E0A0EBB1E48093E60F9093E70FA09356
:10F6D000E80FB093E90F8093EA0F9093EB0FA0939C
:10F6E000EC0FB093ED0FEE0FFF0BE954FD4F80814F
:10F6F00091818330910549F184309105D9F10297C8
:10F7000061F480E090E0ABE8B3E48093E60F90937F
:10F71000E70FA093E80FB093E90F8FEB92E00E9400
:10F72000C6EF1092EE0F1092EF0F1092F00F1092A2
:10F73000F10F87ED92E00E94C6EF80919D058F5FEB
:10F740008530ECF480939D05089580E090E0ABE86F
:10F75000B3E48093E60F9093E70FA093E80FB09384
:10F76000E90F8093EA0F9093EB0FA093EC0FB09307
:10F77000ED0FD3CF80E090E0ABE8B3E4F2CF10928E
:10F780009D050895CF93DF9300D01F92CDB7DEB7CC
:10F790000F945F580F94FF4F69837A838B839C8308
:10F7A000CE0101960E942CFD0F900F900F900F90AC
:10F7B000DF91CF9108950F9401502AE037ED43E295
:10F7C0005DE30F94E65720E030E0A9010F94EC567A
:10F7D0000C94C27BCF92DF92EF92FF92CF93DF9394
:10F7E00000D01F92CDB7DEB76B017C0120E030E086
:10F7F000A9010F94FA4F87FD1BC06DEB77E386E0FC
:10F8000095E3A70196010F94EC5669837A838B8365
:10F810009C83CE0101960E942CFD0F900F900F90BB
:10F820000F90DF91CF91FF90EF90DF90CF900895F0
:10F830006DEB77E386E095EBE4CF0F9401502AE07F
:10F8400037ED43E25DE30F94E65720E030E0A90195
:10F850000F94EC560C94EA7B0F94015020E030E0BA
:10F86000A9010F94EC560C94EA7BCF92DF92EF92B1
:10F87000FF926B017C0120E030E0A9010F94FA4F68
:10F8800087FD26C06DEB77E386E095E3A70196013F
:10F890000F94EC566B017C0120E030E0A9010F943D
:10F8A000FA4F20E030E040E05FE387FF04C020E053
:10F8B00030E040E05FEBC701B6010F94EC560F94C7
:10F8C0005858CB01FF90EF90DF90CF900D9401003E
:10F8D0006DEB77E386E095EBD9CF0F94015020E0F4
:10F8E00030E0A9010F94EC560C94357CCF92DF9256
:10F8F000EF92FF92CF93DF9300D01F92CDB7DEB788
:10F900000F94015020E030E048EC52E40F94E657A9
:10F9100020E030E0A9010F94EC566B017C0120E05F
:10F9200030E0A9010F94FA4F2DEB37E346E055E3A1
:10F9300087FF04C02DEB37E346E055EBC701B60166
:10F940000F94EC5669837A838B839C83CE01019656
:10F950000E94C7FE0F900F900F900F90DF91CF91F4
:10F96000FF90EF90DF90CF9008950C94D6DC0C942C
:10F97000D6DC0C94D6DC0C94D6DC0C9488DC0C948D
:10F9800088DC0C9488DC0C9488DCCF92DF92EF92B8
:10F99000FF92CF93C82F0F947E326B017C0124EA33
:10F9A00030E74DE75FE36091250270912602809178
:10F9B0002702909128020F94FA4F87FD18C08AEF12
:10F9C00090E0A0E0B0E08C0D9D1DAE1DBF1D8093AA
:10F9D000380590933905A0933A05B0933B05C09341
:10F9E0001E02CF91FF90EF90DF90CF90089580E0BE
:10F9F00090E0DC01E8CFCF92DF92EF92FF920F937D
:10FA00001F930F947E320091090510910A052091F1
:10FA10000B0530910C056B017C01C01AD10AE20A7A
:10FA2000F30A9701860137FD11C020910805209542
:10FA3000209308056A547C4F8F4F9F4F60930905B0
:10FA400070930A0580930B0590930C0581E09091CB
:10FA50000805911101C080E01F910F91FF90EF9078
:10FA6000DF90CF9008950F941B4010924C08109295
:10FA70006C020E944D36882351F08091DC1582FD86
:10FA800006C08BE09EE19093C2078093C10761E0BE
:10FA900084E09EE10E94CA370C94DFFC4F925F9293
:10FAA0006F927F928F929F92BF92CF92DF92EF924E
:10FAB000FF920F931F93CF93DF9300D000D01F923C
:10FAC0001F92CDB7DEB77C016A014901FB0190812D
:10FAD0008CE0989F800D1124982FF7012081822FB0
:10FAE000880F820F880F8093A5159093A615411556
:10FAF000510571F1FA82E9827C836B83011121C087
:10FB0000AE014B5F5F4FB401C6010E94B7276C0185
:10FB10006D817E818F8198856115710581059105C3
:10FB2000B9F00E941829F70180818F5F80838531A9
:10FB300038F3CE0101960E94F079E2CFB12C860114
:10FB400029C08A01B12C26C0452846284728B1F78C
:10FB500028960FB6F894DEBF0FBECDBFDF91CF91D0
:10FB60001F910F91FF90EF90DF90CF90BF909F90EB
:10FB70008F907F906F905F904F900895B39407C0DF
:10FB8000B1102EC001151105C9F20F5F1F4F0115ED
:10FB90001105A9F2AE014B5F5F4FB401C6010E948F
:10FBA000B7276C014D805E806F80788441145104CA
:10FBB00061047104A9F0F0E24F165104610471046C
:10FBC000F9F2D301C2018D97A109B1090297A105EC
:10FBD000B10530F04BE2441651046104710471F632
:10FBE000F7018081482F4B0D5527551F4631510590
:10FBF00034F0853020F0CE0101960E94F07981E04A
:10FC0000411451046104710409F480E0B80EF70155
:10FC100080818B0D8083BB2009F496CFBA94AE010E
:10FC20004B5F5F4FB401C8010E94B7278C016D8103
:10FC30007E818F8198850E941829EDCFEF92FF92E7
:10FC40000F931F93CF93DF9300D000D000D01F926B
:10FC50001F92CDB7DEB77C0120912008422F022EE3
:10FC6000000C550B80912108833099F1843051F1BB
:10FC70008AE991E25F932F939F938F938E010F5F99
:10FC80001F4F1F930F930F94914FC7010E947CDC6D
:10FC90004FE350E0B80183EC97E00F94615A0F9066
:10FCA0000F900F900F900F900F902B960FB6F89427
:10FCB000DEBF0FBECDBFDF91CF911F910F91FF909F
:10FCC000EF90089586EA91E227FDD4CF81E991E291
:10FCD000D1CF8FEA91E2CECFE0912C0885E1E80206
:10FCE000F0011124E85EFA4E868197810C941E7E05
:10FCF000E0912C0886E0E802F0011124EB5FF74F59
:10FD0000808191810C941E7E0F931F93CF93DF937C
:10FD10008C01EB019091561520915715921305C057
:10FD20000F94E8010E94EAF0F5CF8091551534E078
:10FD3000839FF0011124E85AFA4E11830083D38384
:10FD4000C2839F5F909356158F5F281739F0809379
:10FD50005515DF91CF911F910F9108951092551570
:10FD6000F8CF63E972E084E690E00E94847E6AEB5B
:10FD700072E084E690E00C94847E81110C94B17E54
:10FD800068EB71E084E190E00C94847E0E94CAD814
:10FD90000C94BD7E0F94A5120C94BD7E0E94A4FA13
:10FDA0000C94B17ECF93DF93CDB7DEB720E24885C8
:10FDB00059856F818E810F94512CDF91CF910895D9
:10FDC000282F10922A0880911A0890911B08A09160
:10FDD0001C08B0911D08B7FF08C010921A081092B5
:10FDE0001B0810921C0810921D088091A5058823FD
:10FDF00031F080911A0880931E08109219088091A2
:10FE000018081816FCF4082E000C990B821B910997
:10FE100020911E08022E000C330B2817390794F08E
:10FE200097FF02C090E080E080931E08092E000C2E
:10FE3000AA0BBB0B80931A0890931B08A0931C0875
:10FE4000B0931D0880911E086623A9F090911F08A9
:10FE5000891714F480931F0820911F08022E000CAC
:10FE6000330B2C5F3F4F482F082E000C550B2417E7
:10FE700035071CF4845080931F0808955F926F9299
:10FE80007F928F929F92AF92BF92CF92DF92EF922A
:10FE9000FF920F931F93CF93DF9361E081E00E9465
:10FEA000E07EC0911F0885E0982E9C0ED1E09DEE6B
:10FEB000E92E91E2F92E882483947D2E7C1A6C2EF3
:10FEC00061942FECC22E21E2D22E12E01C1B33E0F3
:10FED000532E44E3A42E42E2B42EC11141C0DD23CF
:10FEE000D9F080911E081816BCF040911A08509164
:10FEF0001B0860911C0870911D084F5F5F4F6F4F8A
:10FF00007F4F40931A0850931B0860931C0870930E
:10FF10001D088F5F80931E0880917802882341F02E
:10FF200030E020E041E068EF71E2862D0E947B2AFC
:10FF300080914A08882309F487C0C23051F4809127
:10FF40001E08823009F445C08091780281115AC0A0
:10FF5000D0E0CF5F9C12C1CF83E08093180818C017
:10FF6000C13031F790911E08913031F080917802C4
:10FF700081111EC0D0E0DCCF8091170810921708C5
:10FF80008823A1F3C0934B0880911908882371F34B
:10FF9000DF91CF911F910F91FF90EF90DF90CF9065
:10FFA000BF90AF909F908F907F906F905F900895DB
:10FFB0001F92FF92EF927F9281E0913009F080E0F2
:10FFC0008F930E94D27E0F900F900F900F900F9002
:10FFD000D1CF8091170810921708882309F4B4CF65
:10FFE0008091550288258093550250927802A11481
:10FFF000B10411F00E94342280911908882309F479
:020000021000EC
:10000000A3CFC6CF81E090911E08923009F080E026
:10001000909155022CED31E2911102C028ED31E2B0
:1000200001E04FED51E2612F0E94762B91CF80913C
:10003000170810921708882371F0C0934B0880911D
:100040001908882341F0A4CFC23009F082CF9091E3
:100050001E08923061F380917802882309F478CFEA
:100060001F92DF92CF921F9381E0923009F080E0DF
:100070008F930E94D27E0F900F900F900F900F9051
:1000800067CF2F923F924F925F926F927F928F92A3
:100090009F92AF92BF92CF92DF92EF92FF920F9317
:1000A0001F93CF93DF934C010F94474F0196840128
:1000B000080F191FC8010F94474F01966801C80E19
:1000C000D91EF8016080C1E0611001C0C0E0F601F6
:1000D0003080D1E0311001C0D0E0AA24A394611097
:1000E000A12C60E085E00E94E07E50901F08752CF6
:1000F0009EE0E92EF12C252C21948A2D90E001968A
:100100005C01AC0EB11CAD0EB11C71101DC0809114
:1001100078028823A1F0E0912402E25068E072E2C4
:10012000E33038F4F0E0EE0FFF1FE152FD4F608145
:10013000718130E020E043E0822D0E947B2AD1E0F3
:10014000611013C0D2E011C0D2E06110D1E0D7112C
:100150000CC080917802882341F030E020E041E03B
:10016000B4018D2F85190E947B2AC1E0CD0F472C49
:100170004518662079F0C7110BC08091780288235A
:1001800039F030E020E041E0B801842D0E947B2A64
:10019000C2E0CD0F332071F0C7110BC080917802FF
:1001A000882339F030E020E041E0B601842D0E9440
:1001B0007B2ACF5FF3E0AF16B1040CF4CF5FC71119
:1001C00062C080917802882309F45AC030E020E0B0
:1001D00042E065E172E2842D0E947B2AD0910605FF
:1001E00093EF9E0D909305058EEF8E0D80932B0857
:1001F0002091A2152E151F0411F00CF041C0209182
:10020000A4159217E8F59EE39093A5158093A61583
:1002100065E470E080E090E00E94182961E36D0FD2
:10022000062E000C770B880B990B0E94182960E2B0
:1002300070E080E090E00E94182980911C15909158
:100240001D150F94AB000E94F32A6FE270E080E06E
:1002500090E00E9418290E94FB7C811109C085E072
:100260008D9FF0011124ED5BF94F8481811108C04D
:1002700080911E1590911F150F94AB000E94F32AD8
:1002800092E090937802ECE0EE0EF11C7394FAE4A5
:10029000EF16F10409F039CFCF5FC0931808DF9152
:1002A000CF911F910F91FF90EF90DF90CF90BF9073
:1002B000AF909F908F907F906F905F904F903F9006
:1002C0002F90089580E292E20C9441808DE292E2B8
:1002D0000C9441808FE492E20C9441808AEE92E289
:1002E0000C94418085EA92E20C94418082ED92E286
:1002F0000C94418085E293E20C94418088E093E283
:100300000C94418088E892E20C94418089E692E264
:100310000C9441808F929F92AF92BF92EF92FF9286
:100320000F931F93CF93DF93EC018B01E42EF22EFA
:1003300080916815909169158C179D0709F43EC04E
:100340002091FE0427FD1092FE0424EBC731D20752
:1003500009F03FC08B529D4B71F40F947E326E5169
:100360007B4F8F4F9F4F60938E0570938F058093C7
:10037000900590939105D0936915C093681530E06E
:1003800020E000931A0810931B0820931C08309358
:100390001D08E0921F08F0921808CB52DD4B21F4A3
:1003A0001092070510928D0582E08093780281E01B
:1003B000809319081092A20510929C05DF91CF91AD
:1003C0001F910F91FF90EF90BF90AF909F908F90F3
:1003D00008952DEBCB32D20771F68751944B19F06B
:1003E000CBE2DDEBC8CF0F947E3280908E059090EB
:1003F0008F05A0909005B0909105681979098A0938
:100400009B0997FFEDCF8091BF078770873041F739
:10041000C9E1D2E8B0CFCF93DF93EC010E94C97954
:1004200020E040E070E060E0CE01DF91CF910C94DD
:100430008A8120E040E070E060E085E090EB0E947F
:100440008A8181E08093070510924808109247083E
:10045000089520E040E070E060E081EC9AE70C94C1
:100460008A8180919809811114C080917D029091B8
:100470007E02019720911C1530911D152817390710
:1004800044F420E040E070E060E080E19CEB0C94FC
:100490008A810C94298221E020930705FC01808148
:1004A0009181A281B3818093250290932602A0932B
:1004B0002702B093280220E040E070E060E08091E5
:1004C0001508909116080C948A81CF93DF9300D081
:1004D0001F92CDB7DEB78DEC9CECACECBCE389830E
:1004E0009A83AB83BC83CE0101960E944B820F900E
:1004F0000F900F900F90DF91CF910895CF93DF93DE
:1005000000D01F92CDB7DEB78DEC9CECACECBDE318
:1005100089839A83AB83BC83CE0101960E944B8270
:100520000F900F900F900F90DF91CF910895CF9380
:10053000DF9300D01F92CDB7DEB780E090E0A0E857
:10054000BFE389839A83AB83BC83CE0101960E946B
:100550004B820F900F900F900F90DF91CF910895E5
:10056000CF93DF9300D01F92CDB7DEB780E090E04D
:10057000A0E2B1E489839A83AB83BC83CE01019668
:100580000E944B820F900F900F900F90DF91CF91B0
:1005900008958FEF8093220820E040E070E060E053
:1005A00086E297E90C948A8181E080930705109296
:1005B000BF071092AE0520E040E070E060E08BE005
:1005C00093E80E948A8184E696E29093C207809322
:1005D000C107089581E0809307058091BF07877068
:1005E000873051F01092BF071092AE0584E696E274
:1005F0009093C2078093C1078091E50F80939E0579
:1006000080E00E94BE3420E040E070E060E08CE5D5
:1006100094E80C948A8180917802882341F030E03C
:1006200020E041E06DE370E282E00E947B2A80914D
:10063000AE058770873041F420E040E070E060E074
:100640008EE393E80C948A81089520E040E070E006
:1006500060E085E593E80E948A8181E08093FF0451
:1006600080919F05811107C082E290E29093C207BA
:100670008093C107089588E290E2F8CF80917802D4
:10068000882341F030E020E041E06EE270E281E05A
:100690000E947B2A8091170810921708882321F066
:1006A00010929F050C94258308950F931F93CF9369
:1006B000DF9300D000D000D01F92CDB7DEB780917D
:1006C00078028823F1F01F9289E18F9380919F0532
:1006D00090E001969F938F938AE190E29F938F938E
:1006E0008E010F5F1F4F1F930F930F94914FB8010F
:1006F0008FE090E20E94F72A0FB6F894DEBF0FBE9B
:10070000CDBF84E0809378028091FF04811108C0FE
:1007100020E040E070E060E08BE993E80E948A818D
:100720002A960FB6F894DEBF0FBECDBFDF91CF91F2
:100730001F910F910895CF92DF92EF92FF92CF9386
:10074000DF9300D01F92CDB7DEB7809117081092CB
:100750001708882331F180919F058F5F80939F0553
:100760008931E0F081E08093FF0420E040E070E018
:1007700060E080E593EB0E948A8189E090E29093AB
:10078000C2078093C1070F900F900F900F90DF91D9
:10079000CF91FF90EF90DF90CF9008950E94258336
:1007A000F2CF60911A0870911B0880911C089091FB
:1007B0001D08611571058105910509F43EC00F946E
:1007C00001502DEC3CEC4CEC5CE30F94605020911C
:1007D000EE0F3091EF0F4091F00F5091F10F0F9409
:1007E000EC566B017C0120E030E040E850EC0F94C7
:1007F000FA4F87FD53C020E030E040E850E4C701E5
:10080000B6010F944C5918160CF44FC0C092EE0F5D
:10081000D092EF0FE092F00FF092F10F87ED92E09F
:100820000E94C6EF82E08093780210921A0810921C
:100830001B0810921C0810921D08809178028823D2
:1008400009F4A1CFC090EE0FD090EF0FE090F00F21
:10085000F090F10F20E030E0A901C701B6010F943C
:10086000FA4F27E137EB41ED58E387FF04C027E15A
:1008700037EB41ED58EBC701B6010F94EC56698395
:100880007A838B839C836BE2CE0101960E94AFFD3D
:10089000BC0182E090E20E94F72A75CFC12CD12CD6
:1008A00090E8E92E90ECF92EB1CFC12CD12C80E844
:1008B000E82E80E4F82EAACF80917802882341F0B8
:1008C00030E020E041E06DE370E282E00E947B2AAC
:1008D0008091AE058770873079F410929D0520E0F5
:1008E00040E070E060E082EE9CEB0E948A8181E053
:1008F00080939C050C94467B08952F923F924F92D3
:100900005F926F927F928F929F92AF92BF92CF929F
:10091000DF92EF92FF920F931F93CF93DF9300D05C
:1009200000D0CDB7DEB71C017A8369832B833C836B
:100930004D835E832701380181E0809319080E946E
:10094000C97983E08093780230928C0520928B05E0
:1009500089819A8190938A05809389058B819C81F6
:10096000AD81BE818093850590938605A093870510
:10097000B09388054092810550928205609283056C
:1009800070928405F12CE12CC0921A08D0921B08B9
:10099000E0921C08F0921D08B0926915A0926815AB
:1009A0009092800580927F058C8D80937E0526969F
:1009B0000FB6F894DEBF0FBECDBFDF91CF911F9170
:1009C0000F91FF90EF90DF90CF90BF90AF909F90EE
:1009D0008F907F906F905F904F903F902F900895F1
:1009E00020E040E070E060E08BE29DEB0C948A81B7
:1009F0000E9484360E944BD50C94F08485E598E0E3
:100A00000F94E33D0E94F0840D941B400E94F084FB
:100A100080EB94E29093C2078093C10708950E94EF
:100A2000DF330F94203F81E08093D2150F94623F13
:100A30000C94F0846F927F928F929F92AF92BF92AC
:100A4000CF92DF92EF92FF920F931F93CF93DF939A
:100A500081E08093070561E00E94E07EC0911F085D
:100A600085E0882E8C0ED1E00FE015E896EBE92E9C
:100A700094E2F92E82E0982E9C1A26E0C22E25E8F8
:100A8000D22E31ECA32E34E2B32E7D2E7C1A6C2EA6
:100A90006194C11130C0DD23D9F080911E08181671
:100AA000BCF040911A0850911B0860911C0870918D
:100AB0001D084F5F5F4F6F4F7F4F40931A08509351
:100AC0001B0860931C0870931D088F5F80931E089D
:100AD00080917802882341F030E020E041E06EEC24
:100AE00074E2862D0E947B2ACF5F8C12D2CF83E0E6
:100AF0008093180823C0C13081F580911E08813091
:100B000089F080917802882309F444C0DF92CF9263
:100B1000BF92AF927F9281E090911E08913089F14F
:100B200080E02FC08091170810921708882349F39E
:100B30000E94068580911908882319F3DF91CF91CF
:100B40001F910F91FF90EF90DF90CF90BF90AF90EB
:100B50009F908F907F906F900895C23029F680917A
:100B60001E088230C9F080917802882399F01F9383
:100B70000F93FF92EF929F9281E090911E08923026
:100B800079F68F930E94D27E0F900F900F900F9066
:100B90000F900F90D0E0A8CF8091170810921708FF
:100BA000882309F30E940F85809119088823D9F2C0
:100BB000C5CF611160932402409306058C3008F084
:100BC0003AC0E82F880FFF0B8827E651FA478F4F6E
:100BD0000D94E3561D86F6850186208604860786D9
:100BE0000A8616860D861B861086138686E691E891
:100BF00021E02093070520E040E070E060E00C94E5
:100C00008A818EE691E8F4CF82E791E8F1CF86E71A
:100C100091E8EECF8AE791E8EBCF8EE791E8E8CF55
:100C200082E891E8E5CF86E891E8E2CF10924B08A0
:100C30008EE39FE7DDCF0C94F08482E691E8D8CF75
:100C40008AE691E8D5CFCF930E94A4FA0E94CAD831
:100C5000C82F882319F080E00F94890B8C2F0E94F5
:100C6000BD7ECF910C94F0840F931F93CF93DF93AD
:100C7000CDB7DEB76E970FB6F894DEBF0FBECDBF0F
:100C8000282F082E000C330B90911F024091200258
:100C90008F3F39F0F901EE0FFF1FEF5DFD4F90819F
:100CA00041814F939F933F938F9384E49EE19F9361
:100CB0008F938E010F5F1F4F1F930F930F94914FD0
:100CC0004FE350E0B80183EC97E00F94615A0E9423
:100CD000F0840FB6F894DEBF0FBECDBF6E960FB690
:100CE000F894DEBF0FBECDBFDF91CF911F910F9162
:100CF00008958FEF0C94348680912C080C943486E0
:100D0000E0918D05EE2389F0E150E0938D0588E0B8
:100D1000E89FF0011124E25BFA4F62817381278121
:100D20004681808191810C948A810C94F0842F9269
:100D30003F924F925F926F927F928F929F92AF926B
:100D4000BF92CF92DF92EF92FF920F931F93CF93B8
:100D5000DF9300D01F92CDB7DEB761E081E00E9443
:100D6000E07E80911F088B83382E8B5F898388E01B
:100D700083198A8397E093199C8386E0782E7318F1
:100D800085E0682E631884E0582E531882E0482EC0
:100D90004318232C21948B8181115BC080911E0804
:100DA000882399F180917802882359F081E090910D
:100DB0001E08911180E024E047EF56E2622D0F9467
:100DC000512C80918609809322089B81953009F0EF
:100DD0009EC010922C0880911E08853009F458C1DD
:100DE00080917802882309F4FEC111E080911E08E9
:100DF000853009F010E0809122080F94020100E094
:100E00009C0144ED56E2662D7FC080911708109238
:100E10001708882339F20E94808680911908882358
:100E200009F4C0CF0F900F900F900F90DF91CF91EA
:100E30001F910F91FF90EF90DF90CF90BF90AF90F8
:100E40009F908F907F906F905F904F903F902F90EA
:100E500008959B819130B1F580911E088130D9F0C1
:100E600080917802882309F4ACCF11E080911E08AC
:100E7000813009F010E080916E0290916F020F9422
:100E8000AB0061E0631900E09C0141EF56E2812F65
:100E90000E94762B96CF809117081092170888230E
:100EA000F9F210E000E027EE33E04AE050E06EE6B1
:100EB00072E081EF96E20F943E2E8091190888230C
:100EC00079F2B0CF8B81823009F06AC180911E081F
:100ED000823009F44CC0809178028823C1F011E07F
:100EE00080911E08823009F010E060913006709108
:100EF000310680913206909133060E94067A00E016
:100F00009C014BEE56E2642D812F0E94762B80913E
:100F10008709809322088B81863009F0E3C081E045
:100F200080932C0880911E08863009F4C6C08091F9
:100F30007802882391F011E080911E08863009F034
:100F400010E0809122080F94020100E09C0144ED22
:100F500056E2672D812F0E94762B9B819F5F9B839A
:100F60008981981318CF89E0809318085BCF80910E
:100F7000170810921708882309F4ADCF20E030E05D
:100F80004AE754E460913006709131068091320650
:100F9000909133060F94605020E030E0A9010F9447
:100FA000EC5620E030E04AE754E40F94EC560F94FE
:100FB0005F581F92912C812C83EBA82E8FEAB82EBC
:100FC0006B0110EDE12E17E0F12E00E010E028E1BA
:100FD0003CEF4FEF5FEF60E376E08BEE96E20E942E
:100FE0007D840F9080911908882309F474CF1ACF5B
:100FF00080911E088330C1F080917802882309F423
:1010000086CF11E080911E08833009F010E08091B6
:101010001E1590911F150F94AB0063E0631900E05B
:101020009C0144EE56E233CF8091170810921708C6
:10103000882311F30F94C62C0BEA1AE72CE231E057
:1010400050E040E06EE175E184EE96E20F943E2EB2
:1010500080911908882381F2E5CE809117081092BB
:101060001708882309F4A8C00F94C62C0BE517ECC9
:101070002CE830E050E040E06EE678E080EE96E26A
:101080000F943E2E80911908882309F495C0CACE8A
:101090008091170810921708882309F4A1CE0F94A5
:1010A000C62C60E476E784ED96E20F94372F8091AA
:1010B0001908882309F494CEB5CE809117081092B0
:1010C0001708882309F433CF0F94C62C60E476E721
:1010D00084ED96E20F94372F80911908882309F444
:1010E00026CFA0CE9B81973091F580911E08873046
:1010F000B9F080917802882309F42FCF11E0809114
:101100001E08873009F010E0809135029091360278
:101110000F94AB0000E09C014FEC56E26C811ACFBB
:101120008091170810921708882319F30DE116E72C
:1011300027EE33E04AE050E065E372E08FEC96E2A0
:101140000F943E2E80911908882399F26BCE8B81E3
:10115000883009F002CF80911E08883091F080918C
:101160007802882309F4F9CE81E090911E08983026
:1011700009F080E023E044EC56E26A810F94512CA0
:10118000ECCE8091170810921708882341F389E16B
:1011900092E80E940B8280911908882301F342CEC5
:1011A0009B81933009F424CF943009F00ACE8091CA
:1011B0001E08843009F451CF80917802882309F405
:1011C000A6CE11E080911E08843009F010E08091D5
:1011D0006E0890916F080F94AB0000E09C0140EE08
:1011E00056E2652D54CE8091870980932208B5CEB2
:1011F0005F926F927F928F929F92AF92BF92CF92A7
:10120000DF92EF92FF920F931F93CF93DF93FF2410
:10121000F39480911E1590911F15892B09F4F12CE0
:1012200061E081E00E94E07EC0911F088C2E95E075
:10123000992E9C0EAA24A39484E0E82EEC1A83E055
:10124000D82EDC1A82E0C82ECC1A7A2C7C1A6C2E8E
:10125000619487E0B82EBC1AC111B8C080911E08F5
:10126000882309F495C080917802882359F081E0A1
:1012700090911E08911180E024E04FEB56E2662D1C
:101280000F94512C8091870980932208C430E9F48F
:10129000A0922C0880911E08843009F445C18091E9
:1012A0007802882391F0D1E080911E08843009F003
:1012B000D0E0809122080F94020100E09C0148EAEE
:1012C00056E26E2D8D2F0E94762B10E000E0D5E0C7
:1012D0005C2E581800932208CD131FC0F801EE0FA2
:1012E000FF1FEE52F04C8591949190932E088093BD
:1012F0002D0880911E088C1709F42BC1809178026B
:10130000882359F081E090911E089D1380E023E02E
:101310004EE956E2652D0F94512C8D2F0F5F1F4F14
:10132000D6E08630B9F680916E0890916F08892BCF
:1013300019F4FF2009F42DC1C73009F580911E086A
:10134000873009F417C1809178028823C1F088EFB3
:1013500094E89F938F9385E996E29F938F93BF9232
:1013600081E090911E08973009F080E08F930E94F1
:10137000D27E0F900F900F900F900F900F9088E0FB
:10138000FF24F394CF5FC91167CF809318080EC074
:101390008091170810921708882309F464CF0E94DF
:1013A000808680911908882309F45DCFDF91CF9161
:1013B0001F910F91FF90EF90DF90CF90BF90AF9073
:1013C0009F908F907F906F905F900895C13009F04B
:1013D0005FC080911E08813009F43FC0809178027F
:1013E000882309F44FCFD1E080911E08813009F0A5
:1013F000D0E080911E1590911F150F94AB0000E076
:101400009C0148EB56E2672D8D2F0E94762B809130
:10141000860980932208C33009F034CF10922C083B
:1014200080911E08833009F46AC080917802882375
:1014300009F44BCFD1E080911E08833009F0D0E051
:10144000809122080F94020100E09C0148EA56E2D4
:101450006D2D8D2F0E94762B15CF8091170810923D
:101460001708882309F4BACF0F94C62C09EA1AE7A3
:101470002CE231E050E040E06EE175E188EB96E26D
:101480000F943E2E80911908882309F4A7CF8ECFA0
:10149000C23009F0BCCF80911E088230B9F0809133
:1014A0007802882309F4EECED1E080911E088230C4
:1014B00009F0D0E080916E0890916F080F94AB0016
:1014C00000E09C0144EB56E26C2D9ECF8091170802
:1014D00010921708882319F30F94C62C0BE517EC0C
:1014E0002CE830E050E040E06EE678E084EB96E2F5
:1014F0000F943E2E80911908882389F257CF80914E
:10150000170810921708882309F48FCF0F94C62C60
:1015100060E476E788EA96E20F94372F8091190805
:10152000882309F482CF42CF8091170810921708C0
:10153000882309F4B4CE0F94C62C60E476E788EAD9
:1015400096E20F94372F80911908882309F4A7CECB
:101550002DCF8091170810921708882309F4CECE5A
:101560008BEC9AE80E940B8280911908882309F479
:10157000C5CE1CCF8091170810921708882309F454
:10158000E2CE0E94F88480911908882309F4DBCE0A
:101590000DCF87E0F7CE4F925F926F927F928F923E
:1015A0009F92AF92BF92CF92DF92EF92FF920F93F2
:1015B0001F93CF93DF930091220861E081E00E94A6
:1015C000E07EC0911F0810E0000F111F0E52104C5A
:1015D00095E0592E5C0E2BE7E22E26E2F22ED3E0A8
:1015E000DC1B3DEAC32E3AE7D32E4DE6A42E46E29D
:1015F000B42E82E0782E7C1A5EE9852E56E2952E76
:1016000081E0682E6C1A4C2E4194C11137C0809134
:101610001E088823B1F080917802882359F081E078
:1016200090911E08911180E024E049E856E2642D73
:101630000F94512CCF5F5C12E8CF84E080931808A0
:101640000CC08091170810921708882321F30E947C
:101650008086809119088823F1F2DF91CF911F9144
:101660000F91FF90EF90DF90CF90BF90AF909F9041
:101670008F907F906F905F904F900895C13059F593
:10168000F8018591949190932E0880932D08809174
:101690001E08813081F080917802882359F21F92D0
:1016A0009F928F926F9281E090911E08913009F481
:1016B00074C080E072C080911708109217088823C8
:1016C00051F380912208682F0F94A8308091190857
:1016D000882309F3C2CFC23009F042C0F8018591D6
:1016E000949190932E0880932D0880911E0882304B
:1016F000D1F080917802882309F49CCFDF92CF92B9
:10170000BF92AF927F9281E090911E08923009F0D3
:1017100080E08F930E94D27E0F900F900F900F90D9
:101720000F900F9087CF8091170810921708882389
:1017300001F30E94AD7A809119088823D1F28DCFF0
:1017400080911708109217088823C1F06091220831
:101750008FEF0F94A83080911908882379F07DCFFE
:10176000C33009F067CFF8018591949190932E08CA
:1017700080932D0880911E08833011F380917802A8
:10178000882309F457CF1F92FF92EF92DF9381E0F5
:1017900090911E08933009F08CCF8F930E94D27ED7
:1017A0000F900F900F900F900F9044CF9F92AF9299
:1017B000BF92CF92DF92EF92FF920F931F93CF933E
:1017C000DF9361E081E00E94E07EC0911F08CC2E93
:1017D00085E0982E9C0E95E2A92E96E2B92ED7E0D0
:1017E000DC1B16E01C1B05E00C1B84E0F82EFC1A29
:1017F00082E0E82EEC1A81E0D82EDC1AC11133C049
:1018000080911E088823B9F080917802882361F0C6
:101810006C2D619581E090911E08911180E024E08B
:1018200048E656E20F94512CCF5FC911E7CF88E00C
:10183000809318080CC0809117081092170888230D
:1018400019F30E948086809119088823E9F2DF91BC
:10185000CF911F910F91FF90EF90DF90CF90BF90AD
:10186000AF909F900895C13011F580911E0881308E
:1018700079F0809178028823B9F281E090911E0876
:10188000913009F080E023E04AEA5FE36D2DCACF92
:101890008091170810921708882359F389E39DE86F
:1018A0000E940B8280911908882319F3D0CFC2308F
:1018B00009F0BFC090911E08923071F080917802BB
:1018C000882309F4B1CF81E0923009F080E020E272
:1018D0004AE556E26E2DA6CF8091170810921708A0
:1018E000882361F324E636E23093C2072093C107D0
:1018F00080911908882311F3AACF90911E08933084
:1019000079F080917802882309F48ECF63E06C1916
:1019100081E0933009F080E020E24EE456E282CF8D
:101920008091170810921708882359F325E536E2AD
:101930003093C2072093C10780911908882309F3C7
:1019400086CF90911E08943071F0809178028823A0
:1019500009F46ACF81E0943009F080E020E242E4AB
:1019600056E26F2D5FCF80911708109217088823D9
:1019700061F329E436E23093C2072093C1078091D6
:101980001908882311F363CF90911E08953071F0E8
:1019900080917802882309F447CF81E0953009F0DF
:1019A00080E020E246E356E2602F3CCF80911708AA
:1019B00010921708882361F32DE336E23093C207B3
:1019C0002093C10780911908882311F340CF80919B
:1019D0001E08863081F080917802882309F424CF94
:1019E00081E090911E08963009F080E023E049E202
:1019F00056E2612F17CF809117081092170888239D
:101A000051F385E59EE80E940B8280911908882396
:101A100011F31DCF80911708109217088823D9F071
:101A2000B092C207A092C10780911908882399F04B
:101A30000ECFC33009F461CFC43009F482CFC53072
:101A400009F4A2CFC63019F2C73009F0EDCE90915B
:101A50001E089730F9F280917802882309F4E4CEC9
:101A600081E0973009F080E020E244E156E26D2FFA
:101A7000D9CEAF92BF92CF92DF92EF92FF920F93A7
:101A80001F93CF93DF9361E081E00E94E07EC091DD
:101A90001F0885E0C82ECC0ED5E0DC1B93E0D92EC4
:101AA00014E01C1BBD2CBC1A82E0F82EFC1A81E04D
:101AB000E82EEC1AAC2EA194C1112BC080911E0807
:101AC000882381F080917802882369F181E09091E8
:101AD0001E08911180E024E04DE056E26A2D0F943B
:101AE000512C21C08091170810921708882351F3B8
:101AF0000E94808680911908882321F3DF91CF917D
:101B00001F910F91FF90EF90DF90CF90BF90AF901B
:101B10000895C130A1F590911E08913059F080913F
:101B20007802811119C0CF5FCC11C6CF86E08093B7
:101B30001808E4CF8091170810921708882379F3CA
:101B4000809137028C2780933702D092780280915F
:101B50001908882321F3D2CF81E0913009F080E089
:101B6000909137022CEF35E2911102C028EF35E257
:101B700001E04FEF55E26E2D0E94762BD4CFC2309C
:101B800009F077C080911E08823079F08091780248
:101B9000882349F281E090911E08923009F080E09C
:101BA00023E04BEC5FE36F2D9ACF809117081092E2
:101BB0001708882359F38CEB9AE70E940B828091D7
:101BC0001908882319F39ACF80911E08833081F079
:101BD00080917802882309F4A6CF81E090911E08B5
:101BE000933009F080E023E044EC5FE36B2D77CF86
:101BF0008091170810921708882351F387EB9AE712
:101C00000E940B8280911908882311F377CF80916D
